:020000040800F2
:10800000C8C20020A1810008A9810008DD9F0008E6
:10801000AD810008AF810008B181000800000000B8
:10802000000000000000000000000000B381000814
:10803000B581000800000000B7810008B981000880
:10804000BB810008BB810008BB810008BB81000820
:10805000BB810008BB810008BB810008BB81000810
:10806000BB810008BB810008BB810008BB81000800
:10807000BB810008BB810008979200089B92000812
:10808000BB8100089F920008BB810008BB810008EB
:10809000BB810008BB810008BB810008BB810008D0
:1080A000BB810008BB810008BB810008BB810008C0
:1080B00025BF0108BB810008BB810008BB81000807
:1080C000BB810008BB810008BB810008BB810008A0
:1080D000BB8100087DC8010881C8010885C8010866
:1080E00053960008BB810008BB810008BB810008D3
:1080F000BB810008BB810008BB810008A392000877
:10810000BB810008BB810008BB810008BB8100085F
:1081100075C8010879C80108BB810008BB81000847
:10812000BB810008BB810008BB810008BB8100083F
:10813000BB810008BB810008BB810008BB8100082F
:10814000BB810008BB810008BB810008BB8100081F
:10815000BB810008A7920008AB92000889C80108FB
:10816000BB810008BB810008BB810008BB810008FF
:10817000BB810008BB810008BB810008BB810008EF
:10818000BB810008BB810008DFF810D000F0BEFB07
:10819000004800474DE50108AFF30080C8C2002049
:1081A0000648804706480047FEE7FEE7FEE7FEE791
:1081B000FEE7FEE7FEE7FEE7FEE7FEE7C9BE0108D1
:1081C000898100082DE9F0410024061B254671F144
:1081D000000605DA01240027D0EB070067EB010158
:1081E000161E73F1000605DA0027D2EB07020125FF
:1081F00067EB030300F077FA86460E4617469C4667
:10820000AC4204D00025D0EB050E65EB010624B18D
:108210000020D2EB000760EB030C704631463A4673
:108220006346BDE8F081202A06DBCB17203A41FAED
:1082300002F043EAE07306E041FA02F3D040C2F1F3
:108240002002914008431946704740EA01039B070A
:1082500003D009E008C9121F08C0042AFAD203E0BB
:1082600011F8013B00F8013B521EF9D27047421E43
:1082700012F8013F002BFBD111F8013B02F8013B42
:10828000002BF9D17047421C10F8011B0029FBD1CB
:10829000801A704730B505460020034600E05B1C9D
:1082A000934205D2EC5CC85C201A01D1002CF6D1B7
:1082B00030BD2DE9FE4F804681EA0300C00F0C4619
:1082C000009021F0004123F00045B8EB0200A941E5
:1082D00005D24046214690461C460B46024623F0F6
:1082E0000040104347D0270DC7F30A00C3F30A51DB
:1082F0000290401A019040286BDAC3F3130040F457
:10830000801B0098924620B10023D2EB030A63EB56
:108310000B0B01985946C0F14002504600F014FA88
:1083200006460D4650465946019AFFF77CFF10EB72
:1083300008006141002487EA115284EAE7731A4376
:1083400040D0009A62B3019A012A4FEA075215DC25
:10835000001B61EB02014FF0004202EA0752CDE937
:108360000042001C41F5801132462B4600F051FAC4
:1083700003B0BDE8F08F40462146F9E7001B61EBF2
:108380000201001C41F5801300185B412018A2F582
:10839000001747EB030140EAD570B6196D4111E0B3
:1083A0006D084FEA360645EAC0754FEA0752001BD2
:1083B00061EB0201001C41F5801149084FEA3000D1
:1083C0000019514132462B4603B0BDE8F04F00F092
:1083D00011BA0098012240000023D0EB020263EBA7
:1083E000E073009821464FEAE074B8EB000061EBBF
:1083F0000401E9E783F000435BE781F0004158E7BF
:108400002DE9FE4F81EA030404F0004421F000410D
:1084100000944FF0000B23F0004350EA01045ED0BB
:1084200052EA03045BD0C3F30A54C1F30A552C4447
:10843000A4F2F3340194A0FB0254C1F3130141F4FC
:108440008011C3F3130343F4801301FB024400FBC8
:10845000034E840A970A44EA815447EA8357A4FBEF
:10846000076802958D0A05FB07854FEA932C04FBEC
:108470000C542705029D4FEA065847EA1637B5EB1C
:1084800008056EEB070C870E920E47EA811742EA49
:108490008312A7FB0201B6EB0B0164EB00042B0D6A
:1084A00043EA0C335E1844EB1C50DA465146E7FBB6
:1084B0000201C5F313044FEA0B3343EA14534FEAA6
:1084C0000432019C43EA0603A4F10C040294009CCC
:1084D000CDE900B400F09DF903B0BDE8F08F0020B5
:1084E0000146F9E72DE9F04D81EA030404F0004B61
:1084F00021F0004514464FF0000A23F0004150EAF5
:10850000050220D054EA01021DD0C5F30A570246E5
:10851000C5F31303C1F31300C1F30A5640F48015E9
:1085200043F48013A7EB0608101BD64608F2FD386B
:1085300073EB050002D308F1010801E092185B41DA
:10854000B8F1000F03DA00200146BDE8F08D0020ED
:108550004FF48011064684460EE0171B73EB0507A7
:1085600005D3121B63EB050306434CEA010C4908D3
:108570004FEA300092185B4150EA0107EDD152EA10
:10858000030012D082EA040083EA0501084305D003
:10859000101BAB4106D20122002306E000224FF05F
:1085A000004302E06FF0010253101AEB06004CEB9F
:1085B000085110EB0A0041EB0B01BDE8F04D00F053
:1085C00019B90EB5C10F80EAE0700844CA0700214E
:1085D00040F233438DE80E000A460B4600F019F9CD
:1085E00003B000BD0EB540F2334102910021CDE948
:1085F00000110A460B4600F00CF903B000BD3EB571
:10860000CA17CB0F002450405140C0186141DA070F
:1086100040F233430094CDE901232246234600F083
:10862000F8F803B030BD70B5C1F30A5201F000454F
:108630000024C1F3130140F2FF3341F480119A4248
:1086400001DA002070BD40F233439A42A2F2334275
:1086500003DC524200F087F800E090402C43F1D058
:10866000404270BD70B5C1F30A5201F000450024CC
:10867000C1F3130140F2FF3341F480119A4202DA50
:108680000020014670BD40F233439A42A2F23342C9
:1086900003DC524200F067F801E000F055F82C438B
:1086A000F0D00023D0EB030063EB010170BD01F0BB
:1086B000004330B421F0004150EA010206D00A0D17
:1086C000A2F56072C1F31301002A02DC30BC002065
:1086D0007047440F44EAC104C100E01830BC00EB0D
:1086E000C25000F050B82DE9F05F054600209246D8
:1086F0009B4688460646814640241BE02846414664
:108700004746224600F02FF853465A46C01A914178
:1087100010D311461846224600F016F82D1A67EBC2
:1087200001084F4622460120002100F00DF817EB0A
:1087300000094E41201EA4F10104DFDC4846314609
:108740002A464346BDE8F09F202A04DB203A00FA7F
:1087500002F1002070479140C2F1200320FA03F398
:10876000194390407047202A04DB203A21FA02F096
:108770000021704721FA02F3D040C2F1200291405B
:108780000843194670470029A8BF7047401C49009C
:1087900008BF20F00100704710B4B0FA80FC00FA66
:1087A0000CF050EA010404BF10BC704749B1CCF191
:1087B000200421FA04F411FA0CF118BF012121431D
:1087C0000843A3EB0C01CB1D4FEA00614FEA1020D8
:1087D00042BF002010BC704700EBC350104400297A
:1087E000A4BF10BC7047401C490008BF20F0010026
:1087F00010BC704710B5141E73F1000408DA401C59
:1088000041F1000192185B411A4301D120F00100AF
:1088100010BD2DE9F04D92469B4611B1B1FA81F29F
:1088200002E0B0FA80F220329046FFF78DFF044656
:108830000F4640EA0A0041EA0B0153465A460843F4
:1088400013D0114653EA010019D0C8F14002504636
:10885000FFF789FF05460E46504659464246FFF748
:1088600073FF084305D0012004E020463946BDE8E7
:10887000F08D0020054346EAE0762C4337430A9802
:108880006305E40AA0EB08000022FD0A44EA47540D
:108890000A3002D500200146E9E7010510196941B7
:1088A000DDE9084500196941BDE8F04DA2E770B562
:1088B00021F0004303430CD0C1F30A550024D5EB4B
:1088C000040564EB0403D617AD1AB34102DB0020A4
:1088D000014670BD201841EB025170BD30B5041E39
:1088E00071F1000404DB4FF00044404264EB0101ED
:1088F000141E73F1000405DB1C464FF00043524286
:1089000063EB0403994208BF904230BD064C074D0B
:1089100006E0E06840F0010394E80700984710344F
:10892000AC42F6D3FFF734FCA8140208C8140208BE
:108930002DE9F04D00231A461B1A8A4103DB002063
:108940000146BDE8F08DC1F30A52C1F3130141F4B1
:1089500080154FF0000BD10702D100186D41521E57
:108960000027044640F2FF11384601EB620A3E46FA
:108970008046024600204FF48011FFF7F4FEC21932
:108980007141BB1846EB0100B4EB030C75EB000C16
:1089900004D3E41A65EB000517460E46241908F1C6
:1089A00001006D4180463428E3DDF91946EB0600ED
:1089B000091BA84103D24FF0FF32134601E0002209
:1089C00013461BEB070046EB0A51BDE8F04DFFF7DD
:1089D00011BF000030B5041E71F1000404DB4FF03C
:1089E0000044404264EB0101141E73F1000405DBF6
:1089F0001C464FF00043524263EB04038B4208BF16
:108A0000824230BD70B58C1810F8015B15F0070379
:108A100001D110F8013B2A1106D110F8012B03E017
:108A200010F8016B01F8016B5B1EF9D12B0705D41F
:108A30000023521E0DD401F8013BFAE710F8013B68
:108A4000CB1A921C03E013F8015B01F8015B521E84
:108A5000F9D5A142D8D3002070BD027803E010F808
:108A6000013B1A44D2B2491E89B2F8D2104670476F
:108A700070B5ADF5287D00260D46ADF89462ADF8D1
:108A8000986200EB40012D4800EBC104608AA842C7
:108A900051D9ADF898624AE0A089228A284481B26F
:108AA000274800F0B1F8ADF894626A46208A0BE0DE
:108AB000BDF894326168C95CBDF89432D154BDF8F8
:108AC0009412491CADF89412BDF894128842EFD864
:108AD000401E81B21046FFF7C0FF1A498870228AF3
:108AE0000DF1FF31515C814219D1ADF894620CE077
:108AF000BDF894126068BDF89422405CA168885467
:108B0000BDF89402401CADF89402208ABDF894127E
:108B1000401E8842ECDC01200DF5287D70BD6420EC
:108B200015F0A4FBBDF89802401CADF89802BDF802
:108B300098020628B0D30020EEE7000088F2010872
:108B4000307C0020220A0020F0B50D46064600EBDE
:108B500046011C48002200EBC104ADF5257D608A6A
:108B6000A8422BD9694606E0A0686368805C9854E7
:108B70008854521C92B2208A401E9042F4DC208A13
:108B8000401E81B26846FFF768FF228A0DF1FF316F
:108B900000275054A089228A284481B2684600F0F8
:108BA0002FF929463046FFF763FF012807D06420DC
:108BB00015F05CFB7F1CBFB2062FEBD300200DF538
:108BC000257DF0BD88F2010838B50025ADF80050CC
:108BD00011F0E0F90A4C207000F088F8217809487B
:108BE000242907D0272908D0282902D1022180F87A
:108BF000E71138BD80F8E75138BD0121F7E70000E3
:108C0000220A0020A42200202DE9F0410646154644
:108C10000C46012080F31088254F0020B88011F009
:108C200099F9000609D4012015F020FBB888401CF2
:108C300080B2B880C828F2D335E0B888C82832D2CC
:108C40001C4F1021384601F0BCF90821384601F0CC
:108C5000BAF9E82000F030F8C4F3871000F02CF8DF
:108C6000A006000E00F028F8002000F025F80024EF
:108C7000002000F021F8641CA4B2042CF8D30024D6
:108C800005E0FF2000F018F83055641CA4B2AC4297
:108C9000F7D31021384601F096F9002080F31088B0
:108CA0000120BDE8F081002080F31088F9E7000082
:108CB000220A00200000024070B50B4C054602213C
:108CC000204611F061FA0028F9D02946204611F01B
:108CD00064FA0121204611F057FA0028F9D0204605
:108CE00011F059FAC0B270BD0030014010B501203A
:108CF00080F310881A4C0020A08011F02BF9000698
:108D000009D4012015F0B2FAA088401C80B2A080DE
:108D1000C828F2D320E0A088C8281DD2114C102109
:108D2000204601F04EF90821204601F04CF93D2083
:108D3000FFF7C2FF2A20FFF7BFFF8020FFF7BCFF2D
:108D4000A720FFF7B9FF1021204601F03CF90020D1
:108D500080F31088012010BD002080F3108810BD22
:108D6000220A0020000002402DE9F04106460D468F
:108D7000012080F31088204C0020A08011F0EAF838
:108D8000000609D4012015F071FAA088401C82B2B7
:108D9000A280C82AF2D32AE0A088C82827D2174F79
:108DA0001021384601F00DF90821384601F00BF981
:108DB0008420FFF781FF0020FFF77EFF0020FFF7F0
:108DC0007BFF0020FFF778FF002404E0305DFFF711
:108DD00073FF641CA4B2AC42F8D31021384601F0F2
:108DE000F2F8002080F310880120BDE8F081002017
:108DF00080F31088F9E70000220A002000000240FA
:108E000070B50D46012181F310881146FFF7ACFFC4
:108E1000002832D01B4C0020A08011F09BF80006E7
:108E200009D4012015F022FAA088401C80B2A0804D
:108E3000C828F2D322E0A088C8281FD2124C1021E3
:108E4000204601F0BEF80821204601F0BCF883203E
:108E5000FFF732FFC5F38710FFF72EFFA806000EBD
:108E6000FFF72AFF0020FFF727FF1021204601F01F
:108E7000AAF8002080F31088012070BD002080F344
:108E8000108870BD220A00200000024010B50023A7
:108E90001A4604E010F8014B6340521CD2B28A42D9
:108EA000F8D3184610BD000010B50446392015F05F
:108EB000DDFBE0B215F0FAFBC4F3072015F0F6FB7A
:108EC000C4F3074015F0F2FB200E15F0EFFB4FF452
:108ED0008051034801F077F8BDE8104013F0C6BD9B
:108EE000000402402DE9F041054614460E463A20A2
:108EF00015F0BCFBF0B215F0D9FB300A15F0D6FB2B
:108F0000104F4FF480563146384601F05CF8B046B9
:108F10003E4613F0ABFD1D2811D1284600F0A4F801
:108F200007463B2015F0A2FB4146304601F04BF8C6
:108F30003D44002CEDD0208838442080E9E7BDE88E
:108F4000F0810000000402402DE9F041054614467E
:108F50000E463C2015F08AFBF0B215F0A7FB300A54
:108F600015F0A4FB114F4FF480563146384601F0FE
:108F70002AF80CB100202080B0463E4613F076FD62
:108F80001E2811D1284600F017F907463D2015F09C
:108F90006DFB4146304601F016F83D44002CEDD003
:108FA000208838442080E9E7BDE8F08100040240D1
:108FB00010B510F017FF08B100F028F8BDE8104018
:108FC000302000F09FB80146362000F089B810B577
:108FD00008B100F0A5F8BDE81040342000F092B8C8
:108FE00010B5044600F09CF820785C2801D02F28AA
:108FF00003D10021642000F0FBF8BDE810403220CE
:1090000000F080B8682000F04BB8000010B52220B6
:1090100015F02CFB15F020FB04464FF4805102485C
:1090200000F0D1FF204610BD000402402DE9F041C0
:1090300015F012FB064615F00FFB054615F00CFB6C
:10904000044615F009FB07464FF48051054800F02F
:10905000BAFF46EA052040EA044040EA0760BDE85E
:10906000F08100000004024070B50546272015F08D
:10907000FDFA15F0F1FA0446260007D015F0ECFAD7
:10908000641E05F8010B14F0FF04F7D14FF4805172
:10909000024800F098FF304670BD00000004024016
:1090A00010B504460C2015F0E1FA204615F0FEFA42
:1090B000BDE81040FFF7BABF10B504460A2015F00E
:1090C000D5FA204615F0F2FA15F0C6FA04464FF428
:1090D0008051024800F077FF204610BD0004024096
:1090E00010B50C4615F0C2FA204615F0DFFA4FF421
:1090F0008051034800F067FFBDE8104013F0B6BC94
:109100000004024010B515F0B1FA4FF48051034845
:1091100000F059FFBDE8104013F0A8BC0004024065
:1091200070B50546012015F0A1FA15F095FA43280F
:1091300028D22B20FFF7C0FF102823D22F2015F0B4
:1091400095FA002015F0B2FA3220FFF7DBFF142861
:1091500018D1CF20FFF7B0FF040013D04C20FFF749
:109160009FFF00EB04214C2000F042F85020FFF755
:1091700097FF00EB0421502000F03AF80021702006
:1091800000F036F82F2015F071FA2C7806E015F86B
:10919000014F5C2C01D02F2C00D10024204615F06B
:1091A00085FA002CF3D1BDE870404FF4805101489E
:1091B00000F009BF0004024070B505462D2015F0EF
:1091C00055FA15F049FA0446260007D0287815F01C
:1091D0006DFA641E6D1C14F0FF04F7D14FF480513A
:1091E000024800F0F0FE304670BD0000000402406E
:1091F00070B505460C460D2015F038FA284615F0D6
:1092000055FAE0B215F052FAC4F3072015F04EFA01
:10921000C4F3074015F04AFA200E15F047FABDE8EE
:1092200070404FF48051014800F0CDBE0004024070
:1092300070B5094DFF22134605F5807605E010F85C
:10924000014B54402A5D5A40335D491E89B2F6D223
:1092500042EA032070BD000015F0010870B500223D
:109260001346154605E010F8014BA2186B41491E44
:1092700089B20029F7D1100C40EA034092B280185D
:1092800045EB13414FEA014242EA104108186FEAE8
:10929000000080B270BD0AF0E3BE0AF081BE0AF0A1
:1092A0004FBE0AF0ADBE0BF0CFBF10F00DBA0000FC
:1092B000074A904201D2074801E005481038064AA3
:1092C0008B0001EA020101D5C160704781607047DF
:1092D00010640240006002407D0F7D0F002901688C
:1092E00002D041F0010101E021F00101016070476D
:1092F0002DE9F043016821F00101016000210160C6
:1093000041608160C1600161212141613C493C4A69
:109310003D251039904202D18D60BDE8F083384A76
:109320004FF474661832904201D18E60F5E7344AEA
:109330004FF474173032904201D18F60EDE7304A1C
:109340004FF0746C4832904202D1C1F808C0E4E793
:109350002B4B2C4A6033984201D1CA60DDE7284C80
:10936000294B7834A04201D1CB60D6E7DFF890805A
:10937000264C08F19008404501D1CC60CDE7DFF8DC
:1093800080804FF03D5908F1A808404502D1C1F84E
:109390000C90C2E71E49DFF878800839404501D1BA
:1093A0000D60BAE71A4D1835A84201D10E60B4E736
:1093B000174D3035A84201D10F60AEE7144D483546
:1093C000A84202D1C1F800C0A7E7114D104960358D
:1093D000091FA84201D10A609FE70D4A78329042E6
:1093E00001D10B6099E70A4A9032904201D10C609A
:1093F00093E7074AA83290428FD1C1F800908CE7DA
:10940000106002403D000020400F002000003D2081
:10941000106402400B0607D5436912B143F0800384
:1094200001E023F080034361802908D0002A02680C
:1094300001F01E0101D00A4300E08A430260704738
:1094400030B50368124ACC6813400A682243D1E958
:1094500005452C432243CC6922430C6A22434C6AC3
:1094600022438C6A22434C6B22438C6B22431A4367
:109470000260426922F00703D1E90B2422431A4318
:1094800042610A6942604A6882608968C16030BD91
:109490003F801CF02DE9FC410121202010F0AAFCA6
:1094A00001268DF8046000258DF8065003208DF804
:1094B00005001B4C302700978DF807506946204661
:1094C00000F02CFD3021204600F07DFD154C84F885
:1094D000785684F87A5684F8796684F87B664FF477
:1094E000FA70C4F8800600F01FF894F8EA038028A8
:1094F00014D1A4F580508565232084F8EF0305205E
:1095000084F8EE0384F8ED73142084F8EC03202033
:1095100084F8EB0384F8EA5300F042F8BDE8FC81DC
:1095200000140240A42200207CB514F073FFD02068
:1095300014F040FF14F0A2FF002014F03BFF14F0E1
:109540009DFF14F067FFD12014F034FF14F096FF54
:1095500000246D4601E0062C01D2012000E000202D
:1095600014F0F8FE2855641CE4B2072CF3D314F071
:109570006BFF0A489DF8061041719DF805100171B6
:109580009DF80410C1709DF8021081709DF80110C3
:1095900041709DF8001001707CBD00008E260020F7
:1095A0007CB51848002401788DF8001041788DF8BA
:1095B000011081788DF8021001218DF80310C17817
:1095C0008DF8041001798DF8051040798DF80600AA
:1095D00014F020FFD02014F0EDFE14F04FFF002017
:1095E00014F0E8FE14F04AFF6D46285D14F0E2FE28
:1095F00014F044FF641CE4B2072CF6D314F024FFEB
:109600007CBD00008E26002070B5094D0022134657
:1096100005F5807605E010F8014B54402A5D5A406C
:10962000335D491E89B2F6D242EA032070BD0000C4
:1096300015F00108072A00D9072240EA002021B1CD
:10964000012901D1D040C0B270479040C0F307203B
:1096500070477047072A00D9072240EA002029B145
:10966000012902D19040C0F307207047D040C0B21A
:109670007047000070B5ADF5327D00260D46ADF89F
:10968000BC62ADF8C06200EB4001324800EBC1049F
:10969000608AA8425CD9ADF8C06255E0012264211D
:1096A0002D4800F0BFF92C4800788DF800003828CC
:1096B00042D1228AE06802FB0501274800F0B2F996
:1096C000ADF8BC626A46208A0BE0BDF8BC32616826
:1096D000C95CBDF8BC32D154BDF8BC12491CADF810
:1096E000BC12BDF8BC128842EFD8401E81B21046B1
:1096F00000F05AFA228A0DF1FF31515C81421BD1F0
:10970000ADF8BC620EE0BDF8BC226168895CA2685D
:1097100000FB0520BDF8BC221154BDF8BC02401C62
:10972000ADF8BC02208ABDF8BC12401E8842EADCBB
:1097300001200DF5327D70BD642014F097FDBDF859
:10974000C002401CADF8C002BDF8C0020628A5D377
:109750000020EEE770EB010844570020F0B50E46FC
:10976000074600EB47012648ADF5317D002500EBAB
:10977000C1048DF8BC52608AB0423DD90021084630
:10978000FFF778FF012837D1694609E0A268401E3B
:1097900000FB06206268285C505548556D1CADB230
:1097A000208AA842F2D80025208AE16800FB061131
:1097B000401E82B2134800F0B3F9208A401E81B2E5
:1097C000684600F0F1F98DF8BC02208AE1680122B8
:1097D00001447043401E0144AFA800F0A1F9314696
:1097E0003846FFF747FF012807D0642014F03EFDFC
:1097F0006D1CADB2062DD7D300200DF5317DF0BD27
:1098000070EB0108445700202DE9F041ADF5307DA3
:10981000354D4FF000088DF8BC82344EA5F800801D
:1098200000243FE000206F4607E056F832204968E8
:10983000125C0A543A54401C80B2298801EB410260
:1098400006EBC2010B8A5B1E8342EEDC288800EB2C
:10985000400006EBC000008A401E81B2384600F08E
:10986000A3F98DF8BC02288800EB400006EBC0008D
:10987000C168008A00FB0411401E82B21C4800F03F
:109880004FF92888012200EB400006EBC000C168B8
:10989000008A01446043401E0144AFA800F040F933
:1098A000641CA4B2288800EB400006EBC000408A8C
:1098B000A042B7D82888401C80B228800B28AFD39C
:1098C0000C48017821F001010170017841F0060196
:1098D0000170A0F8028000210120FFF73FFF0DF585
:1098E000307DBDE8F08100001000002070EB010821
:1098F00044570020802400207CB50121084610F048
:1099000079FA01208DF8040002258DF80550002415
:109910008DF806408DF807001820154E0090694616
:10992000304600F0FBFA05221146304600F032FBCB
:1099300005220621304600F02DFB05220721304686
:1099400000F028FBA02000908DF8045003208DF833
:1099500005008DF806408DF807406946304600F056
:10996000DDFA402000906946304600F0D7FA7CBD11
:1099700000000240F8B5002634460096FFF7BCFF11
:1099800000F0A0F82248641C8442FCD3214C08213A
:10999000204600F016FB1021204600F014FB0620A4
:1099A00000F076F80821204600F00DFB0821204643
:1099B00000F007FB1021204600F005FB012000F01D
:1099C00067F8002000F064F80821204600F0FBFA58
:1099D0001148D0F81C0208B9FFF716FF0F4D2E8072
:1099E0000F4E002405E0C0B22146FFF743FE641C81
:1099F000A4B2288800EB400106EBC101498AA142CC
:109A0000F1D880B2401C80B228800B28E9D3F8BD81
:109A1000FFFF0F0000000240000043421000002042
:109A200070EB01082DE9F0410546002416460F466B
:109A3000012080F31088DFF854800821404600F0B0
:109A4000C0FA1021404600F0BEFA032000F020F8D2
:109A5000C7F3074000F01CF8C7F3072000F018F820
:109A6000F8B200F015F806E0002000F011F8641CD0
:109A700005F8010BA4B2B442F6D30821404600F029
:109A8000A2FA002080F31088BDE8F08100000240B7
:109A900070B50B4C05460221204610F075FB0028DE
:109AA000F9D02946204610F078FB0121204610F01D
:109AB0006BFB0028F9D0204610F06DFBC0B270BDE2
:109AC0000030014010B5012186B0080310F0CEF936
:109AD000124C204610F02EFB0021ADF80810601546
:109AE000ADF80A003820ADF80C000720ADF80010E2
:109AF000ADF81000ADF804104FF48270ADF8061008
:109B0000ADF80E10ADF802006946204610F047FB94
:109B10000121204610F004FB06B010BD00300140CA
:109B20002DE9F0410546002416460F46012080F33A
:109B30001088DFF870800821404600F042FA1021BA
:109B4000404600F040FA0620FFF7A2FF08214046F9
:109B500000F039FA0821404600F033FA102140465F
:109B600000F031FA0220FFF793FFC7F30740FFF739
:109B70008FFFC7F30720FFF78BFFF8B2FFF788FFCF
:109B800005E02878FFF784FF641CA4B26D1CB44282
:109B9000F7D30821404600F016FA002080F3108821
:109BA000BDE8F08100000240027803E010F8013BBC
:109BB0001A44D2B2491E89B2F8D21046704700004A
:109BC00070B51E4A907B012825D1002595731C494C
:109BD0001C480F244E780123F6B14D70D0F828525E
:109BE000D0F8346245EAC605D0F83062D0F82C02CD
:109BF000B60046EA40000543AC43CC708878CC7888
:109C0000A04208D108710C78A04204D050720870AC
:109C1000002800D0137270BD4B70D0F82852D0F8D5
:109C2000346245EAC605D0F83062D0F82C02B6009E
:109C300046EA40000543AC438C70DFE7A4120020E5
:109C4000C90A0020000042422DE9F041ADF57C7DBB
:109C500000273D46ADF8E873FFF7AAF9142808D0AD
:109C6000664880F8E95314F03DFC0DF57C7DBDE8B5
:109C7000F0816348FFF7B4F9614C103C1428207060
:109C800006D0422879D00120FFF79DF92570ECE736
:109C9000FFF7B8F9C4E90205A046BDF8E803FFF7ED
:109CA00003F9FAAA4FF4FA716846FFF71BF955A1B8
:109CB000684614F07BFCA080544C6E46F0B1E1196C
:109CC00001F5805181F847577F1CBFB2282FF6D38A
:109CD000474630444EA114F069FC78800021001FF3
:109CE0000AE0BA880A443244D378621802F58052F6
:109CF00082F84737491C89B28142F2DB45A16846A8
:109D000014F054FC4746A8F80400F0B10021621892
:109D100002F5805282F86F57491C89B22829F6D380
:109D200030443BA114F042FC7880002109380AE05D
:109D3000BA880A443244137A621802F5805282F8D3
:109D40006F37491C89B28142F2DB35A1684614F0B5
:109D50002DFCB880F8B10021621802F5805282F81B
:109D60009757491C89B21429F6D3304428A114F01E
:109D70001DFC788000210D380BE03AE0BA880A44D7
:109D80003244137B621802F5805282F89737491CDF
:109D900089B28142F2DB26A1684614F007FCB88044
:109DA000F0B10021621802F5805282F80157491C77
:109DB00089B23229F6D3304415A114F0F7FB78802C
:109DC0000021C01F0AE0BA880A443244937962181D
:109DD00002F5805282F80137491C89B28142F2DBD8
:109DE00000210320FFF7BAFC0120FFF7ECF8012067
:109DF0003BE70348FFF7EBF837E70000A422002019
:109E0000380A002041504E3D00000000A4120020FE
:109E10003B000000574946494E414D453D0000007A
:109E20005749464950415353574F52443D00000053
:109E30005345525645523D002F4910B5884206D130
:109E4000012108460FF0E2FF002101204FE02B49DD
:109E5000884206D1012102200FF0D8FF0021022004
:109E600045E02749884206D1012104200FF0CEFFAA
:109E7000002104203BE02349884206D1012108202B
:109E80000FF0C4FF0021082031E01F49884206D1AD
:109E9000012110200FF0BAFF0021102027E01B49FC
:109EA000884206D1012120200FF0B0FF00212020A0
:109EB0001DE01749884206D1012140200FF0A6FF7E
:109EC0000021402013E01349884206D1012180205F
:109ED0000FF09CFF0021802009E00F4988420AD141
:109EE0008415012120460FF091FF00212046BDE896
:109EF00010400FF08BBF10BD000002400004024074
:109F000000080240000C0240001002400014024011
:109F100000180240001C024000200240F0B5002260
:109F200001274FF0030C0B6807FA02F52B40AB42F8
:109F30002CD1066853000CFA03F4A64306600E7990
:109F4000D0F800E09E4046EA0E0606600E79012E2B
:109F500001D0022E12D18668A64386604E79D0F8D1
:109F600008E09E4046EA0E0686604668AE434660BC
:109F700045688E799640B6B235434560C568A543BD
:109F8000C560CC799C40C3681C43C460521C102A35
:109F9000C9D3F0BD4B07DB0E9A40C90810B500EBE2
:109FA0008100016A0F249C40A1430162016A1143B0
:109FB000016210BD0246002012690A4200D0012051
:109FC0007047418370470183704700000249487A17
:109FD00000224A7270470000A41200200248006864
:109FE000C00700D000BEFEE7F0ED00E002494AF6EF
:109FF000AA200860704700000030004010B514F03F
:10A0000071FABDE81040642014F030B92DE9F04F2A
:10A0100083466BA0ADF2DC7D002500689A460F46B2
:10A02000A946CDF8D407ADF8D057042A25D8654CF9
:10A0300094F8EE03302101EB101302EBC20000EBA9
:10A04000021261481618337194F8EE0300F00F0005
:10A050003030707194F8ED0301EB1010B07194F88A
:10A06000ED0300F00F003030F071FEF7A1FF14286F
:10A0700007D084F8E99314F035FA0DF2DC7DBDE8E1
:10A08000F08FDFF84481A8F1240898F80000142824
:10A090000ED03046FEF7A4FF88F80000142807D041
:10A0A00042287CD00120FEF78EFF88F80090E4E77C
:10A0B0004FF47A70874200D90746FEF7A3FFC8E93C
:10A0C00002094E46FEF7F0FE94F8ED13302000EB47
:10A0D00011118DF8001094F8ED1301F00F013031DB
:10A0E0008DF8011094F8EC1300EB11118DF80210AB
:10A0F00094F8EC1301F00F0130318DF8031094F84F
:10A10000EB1300EB11118DF8041094F8EB1301F030
:10A110000F0130318DF8051094F8EA1300EB11109F
:10A120008DF8060094F8EA0300F00F0030308DF847
:10A130000700BAF1000F03D0BAF1010F02D004E01A
:10A14000542000E052208DF808003A208DF80900D4
:10A150000A236C4617E00BEB550108780009B0FBA9
:10A16000F3F2C2EBC20210446219303090720878E8
:10A1700000F00F00B0FBF3F1C1EBC1010844303037
:10A18000AD1CD072ADB2B5EB470FE4D303EB470083
:10A1900081B20DF5FA622046FEF7D6FE00E00BE034
:10A1A0000DF5FA620221101DFEF7CEFE0120FEF72A
:10A1B0000AFF88F8006060E73046FEF708FF5CE7BA
:10A1C0000D0A0000A42200204C0A00202DE9F04FC7
:10A1D0004FF0000B2DED028B9FB08DF820B08DF865
:10A1E00000B08DF810B0CDE910BBCDE900BB8DF803
:10A1F00008B08DF80CB08DF81CB08DF814B0ADF827
:10A2000018B0DA46ADF800B09FEDFE0AFE4CCDF86E
:10A2100004B08DED0B0A04F129000C9004F59C505C
:10A220000A9004F5804041F696554FF0010904F577
:10A2300080540990A1E094F83A0B30B384F83ABB0B
:10A240000998B0F84C04F14ED6F88C10C1F57A712B
:10A2500088421AD156F88C0F0999C0F57A70A1F886
:10A260004404EA4F002188373846FFF737F8E849B9
:10A270003846FFF71DF8E74981F800904FF47A70EF
:10A28000306001213846FFF729F894F8460B20B3D7
:10A2900084F846BB0998B0F84E04DC4E716CC1F5E9
:10A2A0007A71884219D1706C0999C0F57A70A1F859
:10A2B0004604D64F002140373846FFF70FF8D649FD
:10A2C0003846FEF7F5FFD34981F801904FF47A70D4
:10A2D000706401213846FFF701F894F8520B20B35F
:10A2E00084F852BB0998B0F85004C84E7169C1F5A2
:10A2F0007A71884219D170690999C0F57A70A1F80C
:10A300004804C24F002110373846FEF7E7FFC34923
:10A310003846FEF7CDFFBF4981F802904FF47A70BE
:10A32000706101213846FEF7D9FF94F85E0B20B327
:10A3300084F85EBB0998B0F85204B44EF16AC1F5D6
:10A340007A71884219D1F06A0999C0F57A70A1F83A
:10A350004A04AE4F002128373846FEF7BFFFB04908
:10A360003846FEF7A5FFAB4981F803904FF47A70A9
:10A37000F06201213846FEF7B1FF94F83A0B94F8E9
:10A38000461B084494F8521B94F85E2B1144C842B3
:10A390007FF451AF07F096BB017821B180F800B08F
:10A3A0008DF808B012E0417819B180F801B0484644
:10A3B0000AE0817819B180F802B0022004E0C17887
:10A3C00021B180F803B003208DF808009DF8080043
:10A3D00000EB400101EB00118B4800EB011000F590
:10A3E000805090F86A1D9DF8080000EB4002C2EB17
:10A3F000C0128C4810F83200C1280BD19DF808001B
:10A4000000EB4002C2EBC012864800EBC20080782D
:10A41000082827D07C4E9DF8080006EB400000F588
:10A42000805090F82C0B00069DF8080047F1A98198
:10A4300000EB400202EB001206EB021000F5805028
:10A44000B04690F8710D02287ED0082987F0078366
:10A45000DFE811F0442CE5010C10311C2227F02814
:10A460006F2C5F30099981F89C949DF8080030B1F9
:10A47000012807D002280FD0032808D10FE04FF49D
:10A48000804101E04FF400516748FFF79AFD6749AA
:10A49000C1F888B207F0E3BA4FF48051F4E74FF403
:10A4A0000061F1E79DF808005E4E00EB4002C2EB50
:10A4B000C01006EBC000C27C9DF8080000EB400312
:10A4C000C3EBC01006EBC000007C42EA00629DF8BE
:10A4D000080000EB4003C3EBC01006EBC000407C5B
:10A4E00003049DF8080000EB4007C7EBC01006EB23
:10A4F000C000807C43EA002002439DF80800A6F5D6
:10A50000176353F8207097427AD09DF8080043F8FB
:10A5100020209DF8080000EB4002C2EBC01006EBC3
:10A52000C000C27B9DF8080000EB4003C3EBC010E5
:10A5300006EBC000807B42EA00228DF80C209DF8DB
:10A54000080001EB400000E00DE100F58040B0F8AC
:10A5500044249DF80C000930824251D39DF8080034
:10A5600001EB400000F58040B0F844049DF80C2059
:10A57000801A9DF80820093808EB420101F5804156
:10A58000A1F844049DF8080000EB4001C1EBC010A5
:10A590009DF80C1006EBC000C01DFEF749FE824678
:10A5A0009DF8080000EB4001C1EBC0109DF80C10B5
:10A5B00006EBC0000844017A9DF8080000EB400259
:10A5C000C2EBC0109DF80C2006EBC0001044C0790F
:10A5D00041EA002151457DD194F8E90378B19DF815
:10A5E0000800012300EB4001C1EBC0109DF80C10E6
:10A5F00006EBC0000422C01D891CFFF707FD17E011
:10A6000004E1000000000000A412002000600240ED
:10A610000088002012000020008020102080001000
:10A6200000880010A0640020001802400000424290
:10A630009DF8080000EB4001C1EBC01006EBC00024
:10A64000407C00F0010000909DF8080000EB400104
:10A65000C1EBC01006EBC000C07CC0F342075846F7
:10A6600016E09DF820100844007D3A460099FEF758
:10A67000E1FF9DF8081001EB4102C2EBC1119DF80A
:10A68000202006EBC101114408759DF82000401CF4
:10A690008DF820009DF820109DF80C00C01F81420D
:10A6A0009DF8080000EB4001C1EBC01006EBC000B4
:10A6B000D7DB90F83200ADF818005946ADF800B07D
:10A6C000BDF81800122872D00BDCA0F10B0007288F
:10A6D00015D200E078E0DFE800F0476A6A6A6A2194
:10A6E0006A00A22863D006DC142860D015285ED04A
:10A6F000A1285CD003E0A32812D0A42857D09DF84D
:10A70000080000EB001202EB002208EBC20000F58B
:10A71000005080F829128DF8201044E0102124E028
:10A720009DF8080000EB4001C1EBC01006EBC00033
:10A7300090F833209DF8080000EB001101EB002099
:10A7400008EBC00000F5005080F82A229DF80800B0
:10A75000A32200EB001303EB002008EBC00000F580
:10A76000005080F8292222E00B219DF8080000EB20
:10A77000001202EB002208EBC20000F5005080F846
:10A78000291214E09DF8080000EB4002C2EBC01053
:10A790009DF8202006EBC000104441739DF8200076
:10A7A000401C8DF820009DF820000528EAD39DF874
:10A7B0000800414608EB400000F58040B0F8440432
:10A7C00000287FF46FAE65E659468DF820B010E0A2
:10A7D0009DF8080000EB4002C2EBC0109DF820205D
:10A7E00006EBC000104441739DF82000401C8DF81A
:10A7F00020009DF820000528EAD39DF8082008EBEA
:10A80000420000F58040A0F8441443E69DF808207B
:10A8100008EB420101F58041A1F844B43AE69DF805
:10A82000080000EB4001C1EBC011FE4800EBC10085
:10A8300040785E46002109F0B5FA8DF81C008DF8CD
:10A84000106047461BE09DF8080000EB400101EB5B
:10A8500000109DF8101007EB001000EB011000F540
:10A86000805090F8950D9DF81C1088429DF81000BE
:10A8700002D18DF81C0012E0401C8DF810009DF8EC
:10A88000080000EB400101EB001007EB001000F5A1
:10A89000805090F86B0D9DF810108842D3D89DF829
:10A8A0000800DFF8808300EB4001C1EBC01008EB2B
:10A8B000C00080780A21B1EB101F9DF8080000EB62
:10A8C0004001C1EBC01008EBC000807801D100F05E
:10A8D0000F008DF80C009DF80C0010B910208DF8B9
:10A8E0000C009DF8080000EB4001C1EBC0109DF882
:10A8F0000C1008EBC00008444078ADF818009DF833
:10A90000080000EB4001C1EBC0109DF80C1008EBF3
:10A91000C000491C09F027FE8DF800009DF80800D2
:10A9200000EB4001C1EBC0109DF80C1008EBC0001B
:10A93000084480789DF80010884247F090809DF888
:10A94000080000EB4001C1EBC01008EBC0004078EC
:10A95000002807F084809DF8080000EB4001C1EB5F
:10A96000C01008EBC0019DF80C000844C1789DF8A8
:10A97000080000EB001202EB002007EBC0029DF87C
:10A980001C0000EB001002EBC00000F5005080F846
:10A9900068129DF8080007EB00119DF81C000844A0
:10A9A00000F5805080F8986B387E012820D19DF802
:10A9B000080000EB400101EB00109DF81C1007EBB4
:10A9C000001000EB01102844017841F08001017073
:10A9D000BDF81800B62805D0C52803D0D52801D069
:10A9E000D92803D19DF80C00032801D2ADF81860D6
:10A9F000BDF81800C5287DD012DCB5287BD008DC56
:10AA0000112879D0122878D0132877D0B22894D181
:10AA1000FEE3B62873D0B928F0D0C3288DD1F8E36F
:10AA2000D9286DD006DCCA286BD0CE28FCD0D5281A
:10AA3000EDD106E0E128F7D0E5287DD0E728E6D182
:10AA4000E8E39DF8080000EB4001C1EBC01008EB03
:10AA5000C000C07884F8E2019DF80800B84600EB19
:10AA6000001101EB002007EBC0029DF81C0000EB79
:10AA7000001002EBC00000F5005090F82C229DF869
:10AA8000080000EB001303EB002007EBC00000F50B
:10AA9000005090F8280282429DF8080000EB400127
:10AAA00001EB00107ED29DF81C10474608EB001009
:10AAB00000EB011094F8E2212844A9EBD2120178AE
:10AAC00062F30001017094F8E201800647D49DF81A
:10AAD000080000EB400101EB00109DF81C1007EB93
:10AAE000001000EB011000F5805090F8960D8006E4
:10AAF00035D507E0FEE3FEE3FEE3FEE3FEE3FEE31F
:10AB0000FEE3FEE39DF8080000EB400101EB0011BD
:10AB100007EB01109DF81C1000EB01102844017890
:10AB200041F0020202709DF8080000EB001101EBF9
:10AB3000002007EBC00200E0FDE39DF81C0042F29C
:10AB4000442100EB001002EBC0000844017841F002
:10AB5000020202709DF808100220FEF7FFFD9DF82A
:10AB6000080000EB001101EB002007EBC00000F52E
:10AB7000005080F827629DF80800022100EB0012C7
:10AB800002EB002007EBC0029DF81C0000EB001058
:10AB900002EBC00000F5005080F82C12B6219DF8A1
:10ABA000080000E010E000EB001202EB002007EBD1
:10ABB000C0029DF81C0000EB001002EBC00000F585
:10ABC000005080F831124BE39DF81C20414608EB01
:10ABD000001000EB021094F8E2312844A9EBD313E3
:10ABE000027863F3000202709DF8080000EB400257
:10ABF00002EB00109DF81C2008EB001000EB021087
:10AC000094F8E22128445309027863F34102027068
:10AC10009DF8080000EB400202EB001001EB001071
:10AC200002E00000A06400209DF81C2000EB021050
:10AC300000F5805090F8960DC0F340029DF8080092
:10AC400000EB001303EB002008EBC0019DF81C0093
:10AC500000EB001001EBC00000F5005090F844023A
:10AC6000C0F34000824250D09DF8080000EB001174
:10AC700001EB002008EBC0029DF81C00414600EBF0
:10AC8000001002EBC00042F2442202449DF808008A
:10AC900000EB400303EB00109DF81C3008EB0010A4
:10ACA00000EB031000F5805090F8960D43081078E3
:10ACB00063F3410010709DF8080000EB400202EBC6
:10ACC00000109DF81C2001EB001000EB021000F5B5
:10ACD000805090F8960D800718D59DF80800D9226D
:10ACE00000EB001303EB002008EBC0019DF81C00F3
:10ACF00000EB001001EBC00000F5005080F831229D
:10AD00009DF808100220FEF729FD37E09DF80800A5
:10AD10004A4600EB001303EB002001EBC0039DF853
:10AD20001C0000EB001003EBC00000F5005080F8A1
:10AD300039929DF80800D92300EB001707EB00209B
:10AD400001EBC0079DF81C0000EB001007EBC000F2
:10AD500000F5005080F831329DF8080000EB001338
:10AD600003EB002008EBC0019DF81C0000EB001075
:10AD700001EBC00000F5005080F86A229DF8080041
:10AD80009DF81C2000EB400101EB001008EB0010C7
:10AD900000EB021000F5805090F8960D00F00102D3
:10ADA0009DF8080000EB001303EB002008EBC00146
:10ADB0009DF81C0000EB001001EBC00000F50050F6
:10ADC00090F8440200F00100824270D09DF8080023
:10ADD000474600EB001101EB002008EBC0019DF895
:10ADE0001C0000EB001001EBC00042F244210144C2
:10ADF0009DF8080000EB400202EB00109DF81C20BB
:10AE000008EB001000EB021000F5805090F8960D52
:10AE10000A7860F300020A709DF8080000EB400118
:10AE200001EB00109DF81C1007EB001000EB011067
:10AE300000F5805090F8960DC0079DF8080037D0B7
:10AE400000EB001101EB002007EBC0019DF81C0096
:10AE500000EB001001EBC00000F5005090F86A0212
:10AE6000F0B39DF8080000EB001101EB002007EBA8
:10AE7000C0019DF81C0000EB001001EBC00000F5C4
:10AE8000005080F869629DF8080000EB400101EB7A
:10AE9000001007EB00119DF81C0001EB0010284486
:10AEA000017821F00101017094F8AC07F0B362E180
:10AEB00000EB400101EB00109DF81C1007EB0010A7
:10AEC00000EB011000F5805090F8960D800676D5C5
:10AED0009DF8080000EB001101EB0020414600E066
:10AEE00080E008EBC0029DF81C0000EB001002EBB4
:10AEF000C00000F5005090F86A02E8BB9DF8080019
:10AF000000EB001202EB002001EBC0029DF81C00D8
:10AF100000EB001002EBC00000F5005090F8390281
:10AF200050BB9DF8080000EB400200E06DE002EB32
:10AF300000109DF81C2001EB001000EB021000F542
:10AF4000805090F8960D800739D49DF808004A4645
:10AF500000EB001303EB002001EBC0039DF81C0085
:10AF600000EB001003EBC00000F5005080F83992B0
:10AF7000D9239DF8080000E021E000EB001C0CEB59
:10AF8000002001EBC00C9DF81C0000EB00100CEB46
:10AF9000C00000F5005080F831329DF8080000EB49
:10AFA000001303EB002008EBC0019DF81C0000EB30
:10AFB000001001EBC00000F5005080F86A229DF8F7
:10AFC000080000EB001101EB002007EBC0019DF829
:10AFD0001C0000EB001001EBC00000F5005080F8F1
:10AFE0006962C8E09DF8080000EB001202EB002047
:10AFF00007EBC0029DF81C0000EB001002EBC00044
:10B0000000F5005080F869924EE7787E012868D1FB
:10B01000B86D798B884264D29DF8080000EB00116E
:10B0200001EB002007EBC0019DF81C0000EB0010B5
:10B0300001EBC00000F5005090F86902012850D1E2
:10B040009DF8080000EB001101EB002007EBC001A8
:10B050009DF81C0000EB001001EBC00000F5005053
:10B0600090F8A302E8BB9DF8080000EB400101EB5B
:10B07000001007EB00119DF81C0001EB001000F51B
:10B08000805090F8941D9DF8080000EB001202EB30
:10B09000002007EBC00000F5005080F825129DF855
:10B0A0000800C32100EB001202EB002007EBC002F6
:10B0B0009DF81C0000EB001002EBC00000F50050F2
:10B0C00080F831129DF8080000EB400101EB001000
:10B0D00007EB00119DF81C0001EB001000F58050FB
:10B0E00000E048E0C0F8986D9DF808100220FEF7D7
:10B0F00035FB8DF8206019E09DF8080000EB001189
:10B1000001EB002007EBC0019DF81C0000EB0010D4
:10B1100001EBC0009DF82010084400F5005080F8B5
:10B120006B629DF82000401C8DF820009DF82000E7
:10B130001428E1D38DF8206019E09DF8080000EB99
:10B14000001101EB002007EBC0019DF81C0000EB93
:10B15000001001EBC0009DF82010084400F50050DD
:10B1600080F887629DF82000401C8DF820009DF833
:10B1700020000A28E1D39DF8080000EB400101EB14
:10B18000001008EB00129DF81C00414602EB001075
:10B1900000F5805090F8960D800712D59DF80800B4
:10B1A000D92200EB001303EB002001EBC0039DF854
:10B1B0001C0000EB001003EBC00000F5005080F80D
:10B1C00031229DF8080000EB001202EB002001EB99
:10B1D000C0029DF81C0000EB001002EBC00000F55F
:10B1E000005090F82E02B2283AD19DF8080000EBEA
:10B1F000400202EB001001EB00129DF81C0002EB74
:10B20000001000F5805090F8960D800728D402E0D9
:10B21000DCE3F5E2FEE39DF8080000EB400202EB00
:10B22000001001EB00129DF81C0002EB001000F56D
:10B23000805090F8960D800612D49DF80800E52203
:10B2400000EB001303EB002008EBC0019DF81C008D
:10B2500000EB001001EBC00000F5005080F8312237
:10B260009DF8080000EB400101EB001008EB001214
:10B270009DF81C00414602EB001000F5805090F84C
:10B28000960D000646F1EB839DF8080000EB4002A6
:10B2900002EB00109DF81C2001EB001000EB0210E7
:10B2A00000F5805090F8960DC00746F0D8839DF8C1
:10B2B000080000EB001202EB002001EBC0029DF839
:10B2C0001C0000EB001002EBC00000F5005090F8ED
:10B2D0006A020028E9D19DF8080000EB400202EB69
:10B2E00000109DF81C2001EB001000EB021000F58F
:10B2F000805007E095E3ACE2FEE3FEE3FEE3B6E256
:10B30000C5E0D3E290F8960D000706F1A8839DF8FA
:10B31000080000EB400202EB00109DF81C2001EB3E
:10B32000001000EB021000F5805090F89D0DC00752
:10B3300006F0958300E0FDE39DF8080000EB0012A5
:10B3400002EB002001EBC0029DF81C0000EB001096
:10B3500002EBC00000F5005090F8B202C007A4D183
:10B360009DF8080000EB001202EB002001EBC00288
:10B370009DF81C0000EB001002EBC00000F500502F
:10B3800090F8A4020028D3D08DF820602AE09DF820
:10B39000080000EB001202EB002001EBC0029DF858
:10B3A0001C0000EB001002EBC0009DF820201044B0
:10B3B00000F5005090F8A5229DF8080000EB40032E
:10B3C00003EB001001EB00139DF82000184400F57A
:10B3D000805090F8720D824208D19DF82000401CE8
:10B3E0008DF820009DF820000628D0D39DF820007D
:10B3F00006282AD006F033BB9DF8080000EB0012A7
:10B4000002EB002001EBC0029DF81C0000EB0010D5
:10B4100002EBC0009DF82020104400F5005090F889
:10B42000A5229DF8080000EB400303EB00109DF8F7
:10B43000203001EB0010184400F5805090F8720D98
:10B44000824208D19DF82000401C8DF820009DF814
:10B4500020000A28D0D39DF820000A28CAD09DF8E1
:10B46000080000EB001202EB002001EBC0029DF887
:10B470001C0000EB001002EBC00042F2B2221044AC
:10B48000027842F001020270122205F02DBD9DF8F3
:10B49000080000EB400101EB001007EB001000F585
:10B4A000805090F8700D00289DF80C0002D00A28FA
:10B4B000A0D182E008289DD18DF8206024E09DF87D
:10B4C000080000EB4001C1EBC0109DF8201008EB14
:10B4D000C0000844C07800F00F00092818D89DF873
:10B4E000080000EB4001C1EBC0109DF8201008EBF4
:10B4F000C0000844C07800F0F000902808D89DF8FB
:10B500002000401C8DF820009DF820000628D6D38E
:10B510009DF820000628C6F0A2829DF8080000EBE6
:10B520004001C1EBC01008EBC000C07801049DF8D9
:10B53000080000EB4002C2EBC01008EBC00000792D
:10B5400041EA00219DF8080000EB4002C2EBC01068
:10B5500008EBC000407901439DF8080000EB0012A1
:10B5600002EB002007EBC0029DF81C0000EB00106E
:10B5700002EBC00000F50050C0F845129DF808002D
:10B5800000EB4001C1EBC01008EBC0008079010462
:10B590009DF8080000EB4002C2EBC01008EBC000B1
:10B5A000C07941EA00219DF8080000EB4002C2EB9F
:10B5B000C01008EBC000007A95E08DF8206024E010
:10B5C0009DF8080000EB4001C1EBC0109DF8201071
:10B5D00008EBC0000844C07800F00F00092818D814
:10B5E0009DF8080000EB4001C1EBC0109DF8201051
:10B5F00008EBC0000844C07800F0F000902808D89C
:10B600009DF82000401C8DF820009DF8200008289F
:10B61000D6D39DF820000828C6F021829DF80800A6
:10B6200000EB4001C1EBC01008EBC00081799DF830
:10B63000080000EB4002C2EBC01008EBC000C0786D
:10B6400041EA00619DF8080000EB4002C2EBC01027
:10B6500008EBC000007902049DF8080000EB4003ED
:10B66000C3EBC01008EBC000407942EA0020014360
:10B670009DF8080000EB001202EB002007EBC0026F
:10B680009DF81C0000EB001002EBC00000F500501C
:10B69000C0F845129DF8080000EB4001C1EBC01056
:10B6A00008EBC000817A9DF8080000EB4002C2EB75
:10B6B000C01008EBC000C07941EA00619DF80800A5
:10B6C00000EB4002C2EBC01008EBC000007A02049D
:10B6D0009DF8080000EB4003C3EBC01008EBC0006E
:10B6E000407A42EA002001439DF8080000EB001276
:10B6F00002EB002007EBC0029DF81C0000EB0010DD
:10B7000002EBC00000F50050C0F849129DF8080097
:10B7100000EB001101EB002007EBC0019DF81C00BD
:10B7200000EB001001EBC00000F5005090F82C1267
:10B730009DF8080000EB001202EB002007EBC000B0
:10B7400000F5005090F8280281429DF808001ED2B2
:10B7500000EB001101EB002007EBC00000F50050EA
:10B7600080F827629DF80800042100EB001202EB2C
:10B77000002007EBC0029DF81C0000EB001002EB5C
:10B78000C00000F5005080F82C12C521FDE300EB4D
:10B79000400101EB00109DF81C1007EB001000EBBE
:10B7A000011000F5805090F8960D80077ED49DF82A
:10B7B000080000EB001101EB002007EBC0019DF831
:10B7C0001C0000EB001001EBC00000F5005090F8E9
:10B7D0003A02012846F043819DF8080000EB001171
:10B7E00001EB002007EBC0019DF81C0000EB0010EE
:10B7F00001EBC00000F5005080F83A62B621C6E0C7
:10B800009DF80800D52100EB001202EB002007EBA9
:10B81000C0029DF81C0000EB001002EBC00000F518
:10B82000005080F831129DF8080000EB001202EB86
:10B83000002007EBC00000F5005080F827929DF82B
:10B84000080000EB400101EB001007EB001005F0D1
:10B85000A7BB9DF8080000EB001101EB002007EBEF
:10B86000C00000F5005080F82762C3218DE39DF8E9
:10B87000080000EB400101EB001007EB001000F5A1
:10B88000805090F8700D00289DF8080000EB4001F2
:10B89000C1EBC01008EBC0006BD0C07801049DF86C
:10B8A000080000EB4002C2EBC01000E0F3E308EB3D
:10B8B000C000007941EA00219DF8080000EB400239
:10B8C000C2EBC01008EBC000407901439DF80800AE
:10B8D00000EB001202EB002007EBC0029DF81C00F9
:10B8E00000EB001002EBC00000F50050C0F8601241
:10B8F0009DF8080000EB001101EB002007EBC001F0
:10B900009DF81C0000EB001001EBC00000F500509A
:10B9100090F82C129DF8080000EB001202EB0020BA
:10B9200007EBC00000F5005090F8280281422DD2AC
:10B930009DF8080000EB001101EB002007EBC000B0
:10B9400000F5005080F827629DF80800032100EB05
:10B95000001202EB002007EBC0029DF81C0000EB78
:10B96000001002EBC00000F5005080F82C12D92125
:10B97000D6E301799DF8080000EB4002C2EBC0104D
:10B9800008EBC000C07841EA00219FE7C5219DF87F
:10B99000080000EB001202EB002007EBC0029DF84C
:10B9A0001C0000EB001002EBC00000F5005080F816
:10B9B00031129DF8080000EB001101EB002007EBAD
:10B9C000C00000F5005080F8276213E59DF80800DC
:10B9D00000EB001202EB002007EBC00000F5005066
:10B9E00080F827929DF80800D52100EB001202EBA9
:10B9F000002007EBC0029DF81C0000EB001002EBDA
:10BA0000C00000F5005080F831129DF8080000EBEE
:10BA1000400100E0D3E301EB001007EB001005F05C
:10BA200011BB9DF80800BE4600EB400101EB001180
:10BA300007EB011000F5805090F8700D00289DF87C
:10BA40000C0002D00E28C0D1A5E00C28BDD18DF885
:10BA5000206024E09DF8081001EB4100C0EBC1100C
:10BA60009DF8201008EBC0000844C07800F00F00DB
:10BA7000092818D89DF8081001EB4100C0EBC1104F
:10BA80009DF8201008EBC0000844C07800F0F000DA
:10BA9000902808D89DF82010491C8DF820109DF89A
:10BAA00020000A28D6D39DF820000A288DD3002034
:10BAB000CDE9000030468DF8206023E0DDE900127A
:10BAC000120242EA11620902CDE900129DF8081043
:10BAD00001EB4102C2EBC1119DF8202008EBC1012E
:10BAE0001144CA78DDE900130A4340EA0301CDE9B5
:10BAF00000219DF8201002E064E3A3E3FEE3491C6B
:10BB00008DF820109DF820100529D7D3DDE90023FA
:10BB10009DF8081001EB011707EB01210EEBC10C9A
:10BB20009DF81C10774601EB01110CEBC10101F5EA
:10BB3000005C00E0B2E2CCF84D226146C1F851321F
:10BB40000023CDE900331A468DF820001EE000994D
:10BB5000120242EA11620902CDE900129DF80810B2
:10BB600001EB4102C2EBC1119DF8202008EBC1019D
:10BB70001144097ADDE90023114340EA0302CDE9CB
:10BB800000129DF82010491C8DF820109DF82010FF
:10BB90000529DCD39DE08DF8206024E09DF8081095
:10BBA00001EB4100C0EBC1109DF8201008EBC00074
:10BBB0000844C07800F00F00092818D89DF8081034
:10BBC00001EB4100C0EBC1109DF8201008EBC00054
:10BBD0000844C07800F0F000902808D89DF82010A4
:10BBE000491C8DF820109DF820000C28D6D39DF814
:10BBF00020000C28C5F033870020CDE90000304636
:10BC00008DF820601FE0DDE90012120242EA1162A5
:10BC10000902CDE900129DF8081001EB4102C2EBC8
:10BC2000C1119DF8202008EBC1011144C978DDE95C
:10BC30000023114340EA0302CDE900129DF82010D1
:10BC4000491C8DF820109DF820100629DBD3DDE972
:10BC500000239DF8081001EB011707EB01210EEB03
:10BC6000C10C9DF81C10774601EB01110CEBC101D2
:10BC700001F5005CCCF84D226146C1F85132002339
:10BC8000CDE900331A468DF820001EE0009912021B
:10BC900042EA11620902CDE900129DF8081001EB99
:10BCA0004102C2EBC1119DF8202008EBC1011144F3
:10BCB000497ADDE90023114340EA0302CDE900128D
:10BCC0009DF82010491C8DF820109DF820100629A1
:10BCD000DCD3DDE900129DF8080000EB001303EB54
:10BCE000002007EBC0039DF81C0000EB001003EBE5
:10BCF000C00000F50053C3F855121846C0F8592289
:10BD00009DF80800F04600EB001101EB00200EEB5F
:10BD1000C0029DF81C0000EB001002EBC00000F513
:10BD2000005090F82C229DF8080000EB001303EB64
:10BD300000200EEBC00000F5005090F8280282426F
:10BD40007DD194F8AC0780B19DF8080000EB40016C
:10BD500001EB001108EB01109DF81C1000EB011025
:10BD60002844017841F0080194E04746C8F839605A
:10BD70009DF8080000EB001101EB002008EBC0016A
:10BD80009DF81C00102200EB001001EBC00142F2F4
:10BD90004D2001440C98FCF758FA9DF8080000EB80
:10BDA000001101EB002007EBC0019DF81C0000EB27
:10BDB000001001EBC00000F2452000F500500168C2
:10BDC000C7F81D104068C7F821009DF8080000EB77
:10BDD000400101EB001007EB00119DF81C0001EB86
:10BDE000001000F5805090F8940D38770A9850F8BC
:10BDF0006A1FC7F83D108088A7F841009DF8080029
:10BE000000EB001101EB002007EBC0019DF81C00C6
:10BE100000EB001001EBC00000F50050D0F860020C
:10BE2000C7F825009DF8080000EB400101EB001069
:10BE300007EB00119DF81C0001EB001000E0DAE0B8
:10BE400000F58050D0F8980DC7F84300B86D81B266
:10BE50000220FCF779FE00210620FDF77FFCB86D7B
:10BE6000798B884202D2B86D401CB865002105204C
:10BE7000FDF774FC9DF8080000EB400101EB001099
:10BE80009DF81C1007EB001000EB0110284401780E
:10BE900021F0080101709DF80800474600EB4001C1
:10BEA00001EB00109DF81C1008EB001000EB0110D6
:10BEB0002844017821F0200101709DF8081002202B
:10BEC000FDF74CFC9DF81C009DF8081000EB0110DC
:10BED000C117CDE9000100EB8001C1EB80103844AF
:10BEE000C0F87D609DF8081001EB011202EB012102
:10BEF00007EBC1029DF81C106D3001EB011102EB44
:10BF0000C10242F24D2111441022FCF79EF99DF826
:10BF1000080000EB001101EB002007EBC0019DF8C9
:10BF20001C0000EB001001EBC001009801F245215C
:10BF300000EB800201F50051C2EB80100A68384422
:10BF400040F8612F496841609DF8081001EB4102FB
:10BF500002EB01119DF81C2007EB011101EB02110E
:10BF600001F5805191F8941D00F8011C0A9951F8CF
:10BF70006A2F0262898881849DF8081001EB011202
:10BF800002EB012107EBC10200E0C9E09DF81C10A3
:10BF900001EB011102EBC10101F50051D1F8601272
:10BFA00081609DF8081001EB410202EB01119DF840
:10BFB0001C2007EB011101EB021101F58051D1F8B2
:10BFC000981DC0F82610009881B20820FDF7C6FB26
:10BFD0009DF8080000EB001101EB002007EBC00109
:10BFE0009DF81C0000EB001001EBC00000F50050B4
:10BFF00080F86A624CE09DF808009DF81C2000EB78
:10C00000400101EB0010414608EB001000EB02106C
:10C010002844027842F0040202709DF8080000EB08
:10C02000400202EB00109DF81C2008EB001000EB12
:10C0300002102844027842F0800202709DF8080045
:10C0400000EB001303EB002001EBC00000F50050F3
:10C0500080F827929DF8080000EB001202EB002008
:10C0600001EBC00000F5005090F828229DF8080070
:10C0700000EB001303EB002008EBC0019DF81C004F
:10C0800000EB001001EBC00000F5005080F82C22FE
:10C09000D52104F08FBFFFE7D52141E0494684F860
:10C0A000E8969DF8080000EB001202EB002007EB79
:10C0B000C0029DF81C0000EB001002EBC00000F570
:10C0C000005090F82C229DF8080000EB001303EBC1
:10C0D000002007EBC00000F5005090F828028242D3
:10C0E0009DF8080026D200EB001202EB002007EBBF
:10C0F000C00000F5005080F827629DF8080000EBB2
:10C10000001202EB002007EBC0029DF81C0000EBC0
:10C11000001002EBC00000F5005080F82C12112135
:10C120009DF8080000EB001202EB002007EBC002B4
:10C1300004F048BF00EB001101EB002007EBC00149
:10C140009DF81C0000EB001001EBC00000F5005052
:10C1500090F82E02B22845F082849DF8080000EB8A
:10C16000001101EB002007EBC00000F5005080F843
:10C1700027629DF80800B22100EB001202EB0020BC
:10C1800007EBC0029DF81C0000EB001002EBC000A2
:10C1900000F5005080F831129DF8080000EB001106
:10C1A00001EB002007EBC0019DF81C0000EB001024
:10C1B00001EBC00000F5005080F82E6205E484F821
:10C1C000E86669E79DF8080000EB001202EB00202A
:10C1D00007EBC0029DF81C0000EB001002EBC00052
:10C1E00000F5005080F8A4928DF8206025E09DF8BD
:10C1F000080000EB4001C1EBC01008EBC0019DF846
:10C2000020000844C1789DF8080000EB001202EB02
:10C21000002007EBC0029DF81C0000EB001002EBB1
:10C22000C0009DF82020104400F5005080F8A512B1
:10C230009DF82000401C8DF820009DF820000A2861
:10C24000D5D3BBE79DF8080000EB4001C1EBC0105F
:10C2500008EBC000C07801049DF8080000EB400224
:10C26000C2EBC01008EBC000007941EA00229DF843
:10C27000080000EB4001C1EBC01008EBC0004079A2
:10C280004FF4E13102438A4298D19DF8080000EB57
:10C29000400202EB00109DF81C2007EB001000EBA1
:10C2A00002102844027822F0040202709DF808006F
:10C2B00000EB001202EB002007EBC0029DF81C000F
:10C2C00000EB001002EBC00000F50050A0F8B062D7
:10C2D0009DF80800132200EB001303EB002007EB8E
:10C2E000C0069DF81C0000EB001006EBC00000F536
:10C2F000005080F831229DF8080000E023E000EBB8
:10C30000400202EB001007EB001000F5805090F89F
:10C31000692D9DF8080008F035F99DF8080000EB3C
:10C32000001101EB002007EBC0019DF81C0000EBA1
:10C33000001001EBC00042F2B2210844017841F044
:10C34000080105F03ABB9DF8080000EB4001C1EB85
:10C35000C01008EBC00001799DF8080000EB400216
:10C36000C2EBC01008EBC000C07841EA00219DF884
:10C37000080000EB001202EB002007EBC0029DF862
:10C380001C0000EB001002EBC00000F50050A0F80C
:10C39000B0129DF8080000EB001101EB002007EB44
:10C3A000C0019DF81C0000EB001001EBC00000F57F
:10C3B0000050B0F8B0129DF8080000EB400202EB0C
:10C3C000001007EB001000F58050B0F87E0D8142A0
:10C3D000C5F045839DF80800E52200EB001101EB54
:10C3E000002007EBC0039DF81C0000EB001003EBDE
:10C3F000C00000F5005080F831229DF8080000EBE5
:10C40000001101EB002007EBC0029DF81C0000EBBF
:10C41000001002EBC00000F5005080F82C629DF87F
:10C42000080000EB400101EB00109DF81C1007EB29
:10C43000001000EB01102844017821F08002027006
:10C440009DF8080000EB001101EB002007EBC00293
:10C450009DF81C0042F2B22100EB001002EBC0007C
:10C460000844017821F001020270A7E69DF8080057
:10C4700000EB4001C1EBC010FE4911F83000042868
:10C4800009D09DF8080000EB4002C2EBC01011F883
:10C490003000152801D1ADF818009DF80800F549C5
:10C4A00000EB4002C2EBC01001EBC00042789DF8E7
:10C4B000080000EB4003C3EBC01011F8300042EA63
:10C4C0000020A0F58051303922D09DF8080000EB03
:10C4D0004001C1EBC010E74901EBC00042789DF874
:10C4E000080000EB4003C3EBC01011F8300042EA33
:10C4F0000020A0F58052313A0CD09DF8080000EBE6
:10C500004002C2EBC01011F83000022804D019E03C
:10C51000A62015E0A72013E09DF8080000EB4002DC
:10C52000C2EBC01001EBC00002799DF8080000EBDF
:10C530004003C3EBC01001EBC000C07842EA00200A
:10C54000ADF818009DF8080000EB001101EB002188
:10C5500008EBC10101F5005191F826128DF81C106D
:10C560009DF808105F469DF81C2008EB011111444E
:10C5700001F5805181F898BB98F81800012810D176
:10C580009DF8080000EB400101EB001108EB0110E1
:10C590009DF81C1000EB01102844017841F0800147
:10C5A0000170BDF8180043F23002811A904274D035
:10C5B00009DC042872D0152871D0A6280DD0A72830
:10C5C00045F04D82F9E0B1F5C06F69D0A1F5C061C9
:10C5D00001397CD00429F3D1F3E39DF8080000EB86
:10C5E000001101EB002008EBC00000F500504146AF
:10C5F00080F827729DF8080000EB001202EB002083
:10C6000008EBC0029DF81C0000EB001002EBC0001C
:10C6100000F5005090F82C02032815D89DF808006A
:10C62000042200EB001303EB002001EBC0039DF894
:10C630001C0000EB001003EBC00000F5005080F878
:10C640002C22A82204F050BC9DF8080000EB001238
:10C6500002EB002001EBC0029DF81C0000EB001073
:10C6600002EBC00000F5005090F82C02082818D802
:10C670009DF80800092200EB001303EB002001EBFA
:10C68000C0039DF81C0000EB001003EBC00000F598
:10C69000005080F82C22A922D4E727E174E191E32D
:10C6A000B6E39DF8080000EB001202EB002001EB5E
:10C6B000C0029DF81C0000EB001002EBC00000F56A
:10C6C000005090F82C020D2816D80E2200E0DDE371
:10C6D0009DF8080000EB001303EB002001EBC00302
:10C6E0009DF81C0000EB001003EBC00000F50050AB
:10C6F00080F82C22A222A5E79DF8080000EB00128A
:10C7000002EB002001EBC0029DF81C0000EB0010C2
:10C7100002EBC00000F5005090F83102A52810D1BE
:10C720009DF8080000EB400202EB00109DF81C2071
:10C7300001EB001000EB02102844027842F00402E2
:10C7400002709DF8080000EB001202EB002001EBE4
:10C75000C0029DF81C0000EB001002EBC00000F5C9
:10C76000005090F82E02A12805F079819DF808006C
:10C7700000EB001202EB002001EBC0029DF81C0050
:10C7800000EB001002EBC00000F5005090F82E22E4
:10C790009DF8080000EB001303EB002001EBC00341
:10C7A0009DF81C0000EB001003EBC00000F50050EA
:10C7B00080F83122A12202F065BE9DF808004646AD
:10C7C00000EB001101EB002008EBC00000F5005069
:10C7D00080F827729DF8080000EB001101EB0020A3
:10C7E00008EBC0019DF81C0000EB001001EBC0003D
:10C7F00000F5005090F82C0205289DF8080000EB89
:10C80000001101EB002007D806EBC00000F5005036
:10C8100080F8277206210EE006EBC0019DF81C008F
:10C8200000EB001001EBC00000F5005090F82C0266
:10C83000092812D80A219DF8080000EB001202EB2B
:10C84000002006EBC0029DF81C0000EB001002EB7C
:10C85000C00000F5005080F82C129DF8080000EB95
:10C86000001101EB002006EBC0019DF81C0000EB5D
:10C87000001001E0A064002001EBC00000F50050B2
:10C8800090F83102A42827D19DF8080000EB400160
:10C8900001EB001006EB00119DF81C0001EB0010ED
:10C8A0002844017841F0200101709DF8080000EB58
:10C8B000001101EB002006EBC0019DF81C0000EB0D
:10C8C000001001EBC00000F5005080F869729DF87F
:10C8D00008100220FCF742FF9DF80800A12100EBA0
:10C8E000001202EB002006EBC00221E48DF820705C
:10C8F00012AAFE4913E09DF8080000EB4003C3EBC9
:10C90000C0109DF8203001EBC0001844C0789DF89D
:10C910002030D0549DF82000401C8DF820009DF858
:10C9200020000628E7D30621104611F0B5FCCDE91A
:10C930001007109B000AC01847EB07014FF48072E4
:10C940000023FBF73FFC9DF8080000EB001101EB12
:10C95000002008EBC0039DF81C00414600EB0010CE
:10C9600003EBC00000F5005080F830229DF808006D
:10C9700000EB001202EB002008EBC00000F50050B5
:10C9800080F827724A4665E29DF8080000EB001126
:10C9900001EB002008EBC0029DF81C00414600EBB3
:10C9A000001002EBC00000F5005090F82C020628A1
:10C9B00031D89DF8080000EB001202EB002001EBDB
:10C9C000C00000F5005080F827729DF8080007228B
:10C9D00000EB001303EB002001EBC0039DF81C00EB
:10C9E00000EB001003EBC00000F5005080F82C2293
:10C9F0009DF80800A72200EB001303EB002001EBD9
:10CA0000C0039DF81C0000EB001003EBC00000F514
:10CA1000005080F831229DF8080000EB001202EB74
:10CA2000002001EBC0029DF81C0000EB001002EB9F
:10CA3000C00000F5005090F82C0201289DF8080075
:10CA400000EB001202EB002007D801EBC00000F55C
:10CA5000005080F8277202221AE001EBC0029DF814
:10CA60001C0000EB001002EBC00000F5005090F835
:10CA70002C0207289DF8080000EB001202EB0020B2
:10CA80001AD801EBC00000F5005080F82772082288
:10CA90009DF8080000EB001303EB002001EBC0033E
:10CAA0009DF81C0000EB001003EBC00000F50050E7
:10CAB00080F82C22A322C5E501EBC0029DF81C00E2
:10CAC00000EB001002EBC00000F5005090F82C02C3
:10CAD0000B289DF8080000EB001202EB00201AD88A
:10CAE00001EBC00000F5005080F827729DF80800A7
:10CAF0000C2200EB001303EB002001EBC0039DF8B8
:10CB00001C0000EB001003EBC00000F5005080F8A3
:10CB10002C22A12296E501EBC0029DF81C0000EB3F
:10CB2000001002EBC00000F5005090F82C020C2819
:10CB30009DF8080000EB001202EB002007D801EB83
:10CB4000C00000F5005080F827720D22A0E701EB2D
:10CB5000C0029DF81C0000EB001002EBC00000F5C5
:10CB6000005090F82C020E287ED89DF808000F2265
:10CB700000EB001303EB002001EBC0069DF81C0046
:10CB800000EB001006EBC00000F5005080F82C22EE
:10CB90009DF80800A12200EB001303EB002001EB3D
:10CBA000C0069DF81C0000EB001006EBC00000F56D
:10CBB000005080F831229DF8080000EB001303EBD1
:10CBC000002001EBC0069DF81C0000EB001006EBF6
:10CBD000C00000F5005080F82E229DF8080000EB00
:10CBE000400202EB00109DF81C2001EB001000EB4E
:10CBF00002102844027842F0800202709DF808007A
:10CC000000EB400202EB00109DF81C2001EB00102D
:10CC100000EB02102844027842F0040202709DF8F2
:10CC2000080000EB400202EB00109DF81C2001EB15
:10CC3000001000EB021000F5805090F8960D800671
:10CC400044F10D879DF8080000EB400202EB001054
:10CC50009DF81C2001EB001000EB02102844027824
:10CC600022F02003037000E023E09DF8080000EBB1
:10CC7000400202EB001001EB00139DF81C0003EBD7
:10CC8000001000F5805090F8960D800710D49DF8A4
:10CC900008009DF81C1000EB400202EB001008EBAE
:10CCA000001000EB01102844017841F008010170E8
:10CCB000FDE39DF8080000EB001202EB002001EB01
:10CCC000C0029DF81C0000EB001002EBC00000F554
:10CCD000005090F82C229DF8080000EB001303EBA5
:10CCE000002001EBC00000F5005001E0A06400202E
:10CCF00090F82802824244F0B2869DF8080000EBCA
:10CD0000001202EB002001EBC0029DF81C0000EBBA
:10CD1000001002EBC00000F5005090F82E02A12890
:10CD20002ED09DF80800A32200EB001303EB002097
:10CD300001EBC0039DF81C0000EB001003EBC000EA
:10CD400000F5005080F831229DF8080000EB001239
:10CD500002EB002001EBC0029DF81C0000EB00106C
:10CD600002EBC00000F5005090F82E02A22804F05B
:10CD700076869DF8080000EB001202EB0020FCE331
:10CD80009DF80800A12200EB001303EB002001EB4B
:10CD9000C0039DF81C0000EB001003EBC00000F581
:10CDA000005080F831229DF8080000EB001303EBDF
:10CDB000002008EBC00000F5005080F8279204F036
:10CDC0004EBEFCE39DF80800A12200EB001101EB30
:10CDD000002008EBC0039DF81C0000EB001003EBE3
:10CDE000C00000F5005080F82E229DF8080000EBEE
:10CDF000001303EB002008EBC0039DF81C0000EBC0
:10CE0000001003EBC00000F5005080F83122B0E7BD
:10CE10009DF8080000EB001101EB002008EBC002B8
:10CE20009DF81C00414600EB001002EBC00000F52D
:10CE3000005090F82C020628C1D89DF8080000EB9D
:10CE4000001202EB002001EBC00000F5005080F85A
:10CE5000277207229DF8080000EB001303EB002067
:10CE600001EBC0039DF81C0000EB001003EBC000B9
:10CE700000F5005080F82C22A7220DE49DF81C003C
:10CE800000EB001001EBC00004F038B89DF808007A
:10CE900000EB001101EB002008EBC00000F5005092
:10CEA00080F827729DF80800A72200EB001303EB1F
:10CEB000002008EBC0019DF81C0000EB001001EB06
:10CEC000C00000F5005080F831229DF8080000EB0A
:10CED0004001C1EBC011FE4800EBC1004079302891
:10CEE0007DD19DF80800464600EB001101EB0020C3
:10CEF00008EBC0019DF81C0000EB001001EBC00026
:10CF000000F5005090F82C129DF8080000EB00127C
:10CF100002EB002008EBC00000F5005090F828025A
:10CF2000814275D19DF8080000EB400101EB001033
:10CF30009DF81C1006EB001000EB0110284401784E
:10CF400021F0010101709DF8080000EB400101EBA8
:10CF500000109DF81C1006EB001000EB0110284497
:10CF6000017821F0020101709DF8080000EB00112A
:10CF700001EB002006EBC0019DF81C0000EB001047
:10CF800001EBC00000F5005090F82F02312829D1A4
:10CF90009DF8080000EB400101EB00109DF81C100B
:10CFA00006EB001000EB01102844017821F020016D
:10CFB00001709DF8080000EB001101EB002006EB6A
:10CFC000C0019DF81C0000EB001001EBC00000F553
:10CFD000005080F869729DF80810022000E017E008
:10CFE000FCF7BCFB9DF8080000EB001101EB0020F2
:10CFF00006EBC0019DF81C0000EB001001EBC00027
:10D0000000F5005090F86A0201287DD1A921C4E101
:10D010009DF80800AE4A00EB4001C1EBC01002EBE6
:10D02000C0004079312870D19DF8080000EB001154
:10D0300001EB002008EBC0039DF81C00414600EB0B
:10D04000001003EBC00000F5005090F82C329DF862
:10D05000080000EB001606EB002008EBC00000F50E
:10D06000005090F8280283424FD19DF8080000EB51
:10D07000001202EB002001EBC0029DF81C0000EB47
:10D08000001002EBC00000F5005090F86A0210BBDF
:10D090009DF8080000EB001303EB002001EBC00338
:10D0A0009DF81C0000EB001003EBC00000F50050E1
:10D0B00080F869929DF8080000EB400202EB001036
:10D0C0009DF81C2001EB001000EB021028440278B0
:10D0D00042F0010202709DF8080000EB400202EBF2
:10D0E00000109DF81C2001EB001000EB02102844FA
:10D0F000027822F00202027094F8AC0720B9487E50
:10D10000012801D1886D01E067E0B4E04A8B9042CC
:10D1100063D29DF8080000EB001202EB002001EB47
:10D12000C0029DF81C0000EB001002EBC00000F5EF
:10D13000005090F8690201284FD19DF8080000EBDB
:10D14000001202EB002001EBC0029DF81C0000EB76
:10D15000001002EBC00000F5005090F8A302E0BB05
:10D160009DF808004FF0104200EB001303EB002085
:10D1700001EBC0039DF81C0000EB001003EBC000A6
:10D1800000F50050C0F834229DF8080000EB400282
:10D1900002EB001001EB00129DF81C0002EB0010E6
:10D1A00000F5805090F8942D9DF8080000EB0013D6
:10D1B00003EB002001EBC00000F5005080F82522B1
:10D1C0009DF8080000EB001202EB002001EBC0020A
:10D1D0009DF81C0000EB001000E04BE002EBC000EB
:10D1E00000F5005090F82C229DF8080000EB001389
:10D1F00003EB002001EBC00000F5005090F828027E
:10D20000824237D19DF8080000EB001202EB0020AB
:10D2100001EBC0029DF81C0000EB001002EBC00007
:10D2200000F5005080F832729DF80800A42200EB4F
:10D23000001303EB002001EBC0039DF81C0000EB82
:10D24000001003EBC00000F5005080F82E229DF87E
:10D250000800A32200EB001303EB002008EBC00141
:10D260009DF81C0000EB001001EBC00000F5005021
:10D2700080F831221FE19DF8080000EB4001C1EB6E
:10D28000C01002EBC000407933289DF8080000EB85
:10D29000400107D0C1EBC01002EBC0004079342838
:10D2A0007ED008E101EB00109DF81C10464608EB0B
:10D2B000001000EB01102844017841F001020270D7
:10D2C0009DF8080000EB400101EB001002E00000B7
:10D2D000A06400209DF81C1008EB001000EB01106A
:10D2E0002844017821F0200202709DF8080000EB2C
:10D2F000400101EB00109DF81C1006EB001000EB44
:10D3000001102844017841F0020202709DF80800E3
:10D3100000EB001101EB002006EBC00000F500500F
:10D3200090F828229DF8080000EB001101EB002086
:10D3300006EBC0039DF81C0000EB001003EBC000DF
:10D3400000F5005080F82C229DF8080000EB400109
:10D3500001EB00109DF81C1006EB001000EB011013
:10D360002844017841F0800202709DF8080000EB2B
:10D37000400101EB00109DF81C1006EB001000EBC3
:10D38000011000F5805090F8960D800704D49DF8A8
:10D3900008100220FCF7E2F9A2219DF8080000E045
:10D3A00010E000EB001202EB002006EBC0029DF83B
:10D3B0001C0000EB001002EBC00000F5005080F8EC
:10D3C0002E1278E09DF808009DF81C2000EB40012B
:10D3D00001EB0011404608EB011101EB0211294459
:10D3E0000A7822F020030B709DF8081001EB41022F
:10D3F00002EB01119DF81C2008EB011101EB021159
:10D4000029440A7822F002030B709DF8081001EB02
:10D41000011202EB012100EBC1069DF81C1001EB8B
:10D42000011106EBC10101F5005181F86A929DF8E6
:10D430000810A92301EB011202EB012100EBC10648
:10D440009DF81C1001EB011106EBC10101F5005123
:10D4500081F82E329DF8081001EB011202EB012138
:10D4600000EBC10101F5005191F828329DF8081038
:10D4700001EB011202EB012100EBC1069DF81C102B
:10D4800001EB011106EBC10101F5005181F82C32CD
:10D490009DF8081001EB410202EB011108EB0110AD
:10D4A0009DF81C1000EB01102844017800E0C5E154
:10D4B00041F0800101700020CDE900008DF820705E
:10D4C000FB4920E0DDE90002120142EA107200018E
:10D4D000CDE900029DF8080000EB4002C2EBC0104D
:10D4E0009DF8202001EBC00010448079DDE9003672
:10D4F0003038C21718433243CDE900029DF82000AE
:10D50000401C8DF820009DF820000628DAD39DF8F5
:10D510000800009A00EB001303EB002008EBC00C9E
:10D520009DF81C00464600EB00100CEBC00000F517
:10D530000050C0F845220020CDE900008DF8207091
:10D5400023E0DDE90002120142EA10720001CDE998
:10D5500000029DF8080000EB4002C2EBC0109DF8ED
:10D56000202001EBC0001044407BDDE9003C303856
:10D57000C217184342EA0C0200E0EEE3CDE90002D4
:10D580009DF82000401C8DF820009DF82000042804
:10D59000D7D39DF80800009A00EB001303EB00209E
:10D5A00006EBC00C9DF81C0000EB00100CEBC0005B
:10D5B00000F50050C0F860220020024600E042E181
:10D5C000CDE900008DF8207020E00098120142EAB9
:10D5D00010720001CDE900029DF8080000EB400246
:10D5E000C2EBC0109DF8202001EBC0001044407C2D
:10D5F000DDE9003C3038C217184342EA0C02CDE99D
:10D6000000029DF82000401C8DF820009DF82000AD
:10D610000628DAD39DF80800009A00EB001303EB0C
:10D62000002006EBC0039DF81C0000EB001003EB8C
:10D63000C00000F50050C0F849229DF8080000EB3A
:10D640004002C2EBC01001EBC00041799DF8080018
:10D6500000EB001202EB002006EBC0029DF81C005C
:10D6600000EB001002EBC00000F5005080F82F1214
:10D670009DF8080000EB400101EB001006EB0011E3
:10D680009DF81C0001EB001000F5805090F8961DED
:10D690009DF8080000EB001202EB002006EBC00230
:10D6A0009DF81C0000EB001002EBC00000F50050DC
:10D6B00080F844129DF8080000EB001101EB0020F7
:10D6C00006EBC0019DF81C0000EB001001EBC00050
:10D6D00000F5005090F82C129DF8080000EB0012A5
:10D6E00002EB002006EBC00000F5005090F8280285
:10D6F000814284F0B4819DF8080000EB001101EB39
:10D70000002006EBC00000F5005080F827729DF85D
:10D710000800A72100EB001202EB002006EBC0027C
:10D720009DF81C0000EB001002EBC00000F500505B
:10D7300080F831129DF8080000EB001202EB002087
:10D7400006EBC00000F5005080F827929DF8080015
:10D7500000EB001101EB002006EBC00000F50050CB
:10D7600090F828129DF8080000EB001202EB002050
:10D7700006EBC0029DF81C0000EB001002EBC0009D
:10D7800000F5005080F82C129DF80800A12100EB54
:10D79000001202EB002006EBC0029DF81C0000EB1B
:10D7A000001002EBC00000F5005080F831129DF827
:10D7B000080000EB400101EB001006EB00119DF8A2
:10D7C0001C0001EB00102844017841F08001017039
:10D7D0009DF8080000EB400101EB00109DF81C10C3
:10D7E00006EB001000EB01102844017841F0040121
:10D7F00001709DF8080000EB400101EB00109DF85E
:10D800001C1006EB001000EB011000F5805090F8A2
:10D81000960D800644F123819DF8080000EB40013D
:10D8200001EB00109DF81C1006EB001000EB01103E
:10D830002844017821F020020270FCE39DF80810D2
:10D84000022003F041BE9DF80800464600EB00129E
:10D8500002EB002008EBC00000F5005080F82772B2
:10D860009DF8080000EB001101EB002008EBC0015F
:10D870009DF81C0000EB001001EBC00000F500500B
:10D8800090F82C020A2815D89DF808000B2100EB0F
:10D89000001202EB002006EBC0029DF81C0000EB1A
:10D8A000001002EBC00000F5005080F82C1253E18C
:10D8B000A06400209DF8080000EB001101EB00209F
:10D8C00006EBC0019DF81C0000EB001001EBC0004E
:10D8D00000F5005090F82C129DF8080000EB0012A3
:10D8E00002EB002006EBC00000F5005090F8280283
:10D8F00081427DD194F8AC0780B19DF8080000EB1F
:10D90000400101EB00109DF81C1006EB001000EB2D
:10D9100001102844017841F0080181E0C6F839700F
:10D920009DF8080000EB001101EB002006EBC001A0
:10D930009DF81C00102200EB001001EBC00142F228
:10D940004D2001440C98FAF780FC9DF8080000EB8C
:10D95000001101EB002006EBC0019DF81C0000EB5C
:10D96000001001EBC00000F2452000F500500168F6
:10D97000C6F81D104068C6F821009DF8080000EBAD
:10D98000400101EB001006EB00119DF81C0001EBBB
:10D99000001000F5805090F8940D30779DF8080045
:10D9A00000EB001101EB002006EBC0019DF81C000C
:10D9B00000EB001001EBC00000F50050D0F8600251
:10D9C000C6F825000A9850F86A1FC6F83D108088EE
:10D9D000A6F84100B06D81B20220FBF7B5F8002136
:10D9E0000620FBF7BBFEB06D718B884204D200E0CD
:10D9F000B2E0B06D401CB06500210520FBF7AEFE23
:10DA00009DF8080000EB400101EB00109DF81C1090
:10DA100006EB001000EB01102844017821F008010A
:10DA200001709DF8080000EB001101EB002006EBEF
:10DA3000C0019DF81C0000EB001001EBC00000F5D8
:10DA4000005080F86A729DF808100220FBF786FEED
:10DA50009DF81C009DF8081000EB0110C117CDE9DE
:10DA6000000100EB8001C1EB80103044C0F87D70F4
:10DA70009DF8081001EB011202EB012106EBC10237
:10DA80009DF81C106D3001EB011102EBC10242F256
:10DA90004D2111441022FAF7D8FB9DF8080000EB45
:10DAA000001101EB002006EBC0019DF81C0000EB0B
:10DAB000001001EBC001009801F2452100EB80024B
:10DAC00001F50051C2EB80100A68304440F8612F24
:10DAD000496841609DF8081001EB410202EB011119
:10DAE0009DF81C2006EB011101EB021101F580519C
:10DAF00091F8941D00F8011C0A9951F86A2F0262EE
:10DB0000898881849DF8081001EB011202EB012144
:10DB100006EBC1029DF81C1001EB011102EBC101E3
:10DB200001F50051D1F8601281609DF8081001EBF9
:10DB3000410202EB01119DF81C2006EB011101EBE3
:10DB4000021101F58051D1F8981DC0F826100098F7
:10DB500081B20820FBF702FE9DF80800A72100EB28
:10DB6000001202EB002006EBC0029DF81C0000EB47
:10DB7000001002EBC00000F5005080F831129DF853
:10DB80000800A22100EB001202EB002006EBC0020D
:10DB90009DF81C0000EB001002EBC00000F50050E7
:10DBA00080F82E120020CDE900003A468DF8207052
:10DBB000FE4921E0DDE900031B0143EA1073000187
:10DBC000CDE900039DF8080000EB4003C3EBC01053
:10DBD0009DF8203001EBC0001844C07ADDE9007CDC
:10DBE0003038C317384343EA0C03CDE900039DF8EE
:10DBF0002000401C8DF820009DF820000A28D9D371
:10DC0000DDE900379DF8080000EB001C0CEB00205C
:10DC100006EBC0089DF81C0000EB001008EBC000EC
:10DC200000F5005CCCF84D326046C0F8517200201F
:10DC3000CDE900008DF8202020E0DDE9000212018E
:10DC400042EA10720001CDE900029DF8080000EBE5
:10DC50004002C2EBC0109DF8202001EBC000104430
:10DC6000407DDDE900373038C21718433A43CDE92B
:10DC700000029DF82000401C8DF820009DF8200037
:10DC80000A28DAD3DDE900129DF8080000EB001342
:10DC900003EB002006EBC0039DF81C0000EB001016
:10DCA00003EBC00000F50053C3F855121846C0F846
:10DCB000592203F0D4BE9DF8080000EB4001C1EBEF
:10DCC000C010BA4911F83000042809D09DF80800A6
:10DCD00000EB4002C2EBC01011F83000152801D152
:10DCE000ADF818009DF80800B04900EB4002C2EB07
:10DCF000C01001EBC00043789DF8080000EB400223
:10DD0000C2EBC01011F8300043EA0021A1F58050A9
:10DD1000303823D09DF8080000EB4001C1EBC01063
:10DD2000A24901EBC00043789DF8080000EB4002D7
:10DD3000C2EBC01011F8300043EA0020A0F5805279
:10DD4000313A0DD09DF8080000EB4002C2EBC01044
:10DD500011F83000022805D01AE084E2A62015E070
:10DD6000A72013E09DF8080000EB4002C2EBC010B2
:10DD700001EBC00002799DF8080000EB4003C3EB03
:10DD8000C01001EBC000C07842EA0020ADF81800D6
:10DD90009DF80800464600EB001101EB002008EB5F
:10DDA000C00000F5005090F826028DF81C009DF888
:10DDB00008005F469DF81C1008EB0010084400F5B1
:10DDC000805080F898BB98F81800012810D19DF871
:10DDD000080000EB400101EB00109DF81C1006EB61
:10DDE000001000EB01102844017841F0800101701F
:10DDF000BDF81800A7287BD007DC042879D01528A7
:10DE000078D0A62843F02B863DE000F51D60B0F5E4
:10DE1000804004D011286ED01228F3D1FDE39DF884
:10DE2000080000EB001101EB002006EBC0019DF89B
:10DE30001C0000EB001001EBC00000F5005090F852
:10DE40002C020028DED19DF8080000EB001101EB48
:10DE5000002006EBC00000F5005080F827729DF806
:10DE6000080000EB001202EB002006EBC0029DF858
:10DE70001C0000EB001002EBC00000F5005080F821
:10DE80002C92A72182E19DF8080000EB001101EB24
:10DE9000002006EBC00000F5005080F827729DF8C6
:10DEA000080000EB001101EB002006EBC0019DF81B
:10DEB0001C0000EB001001EBC00000F5005090F8D2
:10DEC0002C02022818D89DF80800032100EB00124C
:10DED00002EB002006EBC0029DF81C0000EB0010D6
:10DEE00002EBC00000F5005080F82C12A9214DE192
:10DEF000A2E0EBE0DEE103E29DF8080000EB001198
:10DF000001EB002006EBC0019DF81C0000EB0010A7
:10DF100001EBC00000F5005090F82C02052814D841
:10DF20009DF80800062100EB001202EB002006EB32
:10DF3000C0029DF81C0000EB001002EBC00000F5D1
:10DF4000005080F82C12A22120E19DF8080000EB7F
:10DF5000001101EB002006EBC0019DF81C0000EB56
:10DF6000001001EBC00000F5005090F83102A52828
:10DF700010D19DF8080000EB400101EB00109DF866
:10DF80001C1006EB001000EB01102844017841F052
:10DF9000040101709DF8080000EB001101EB002066
:10DFA00006EBC0019DF81C0002E00000A064002008
:10DFB00000EB001001EBC00000F5005090F82E02BD
:10DFC000A12803F04C859DF8080000EB001101EB3F
:10DFD000002006EBC0019DF81C0000EB001001EBD7
:10DFE000C00000F5005090F82E129DF8080000EBDC
:10DFF000001202EB002006EBC0029DF81C0000EBB3
:10E00000001002EBC00000F5005080F831129DF8BE
:10E010000800A12100EB001202EB002008EBC00277
:10E020009DF81C0000EB001002EBC00000F5005052
:10E0300080F82E123DE6F0E39DF8080000EB001199
:10E0400001EB002006EBC0019DF81C0000EB001066
:10E0500001EBC00000F5005090F83102A42827D150
:10E060009DF8080000EB400101EB00109DF81C102A
:10E0700006EB001000EB01102844017841F020016C
:10E0800001709DF8080000EB001101EB002006EB89
:10E09000C0019DF81C0000EB001001EBC00000F572
:10E0A000005080F869729DF808100220FBF756FBBB
:10E0B0009DF8080000EB001101EB002006EBC0000A
:10E0C00000F5005080F82772FEF706BC9DF80800A6
:10E0D00000EB001101EB002006EBC0019DF81C00D5
:10E0E00000EB001001EBC00000F5005090F82C028E
:10E0F00001289DF8080000EB001101EB002007D873
:10E1000006EBC00000F5005080F8277202211AE0EB
:10E1100006EBC0019DF81C0000EB001001EBC000F5
:10E1200000F5005090F82C0204289DF8080000EB40
:10E13000001101EB00201AD806EBC00000F50050DA
:10E1400080F8277205219DF8080000EB001202EB11
:10E15000002006EBC0029DF81C0000EB001002EB53
:10E16000C00000F5005080F82C12A3210EE006EB51
:10E17000C0019DF81C0000EB001001EBC00000F591
:10E18000005090F82C0206280AD8A1219DF808001A
:10E1900000EB001202EB002008EBC00202F012BFFD
:10E1A0009DF8080000EB001101EB002006EBC00118
:10E1B0009DF81C0000EB001001EBC00000F50050C2
:10E1C00090F82C129DF8080000EB001202EB0020E2
:10E1D00006EBC00000F5005090F82802814243F0A1
:10E1E0003E849DF8080000EB001101EB002006EBD7
:10E1F000C0019DF81C0000EB001001EBC00000F511
:10E20000005090F82E02A12834D09DF80800A321D8
:10E2100000EB001202EB002006EBC0029DF81C0090
:10E2200000EB001002EBC00000F5005080F8311246
:10E230009DF8080000EB001101EB002006EBC00187
:10E240009DF81C0000EB001001EBC00000F5005031
:10E2500090F82E02A22803F002849DF8080000EB3B
:10E26000001101EB002008EBC00000F5005080F821
:10E2700027721EE59DF80800A12100EB001202EBB9
:10E28000002006EBC0029DF81C0000EB001002EB22
:10E29000C00000F5005080F831129DF8080000EB36
:10E2A000001202EB002008EBC00000F5005080F8DF
:10E2B0002792FEE49DF80800A12100EB001202EB7A
:10E2C000002006EBC0029DF81C0000EB001002EBE2
:10E2D000C00000F5005080F831129DF8080000EBF6
:10E2E000001202EB002006EBC0029DF81C0000EBC0
:10E2F000001002EBC00000F5005080F82E12ACE7D1
:10E300009DF8080000EB001101EB002006EBC000B7
:10E3100000F5005080F827729DF80800A72200EB56
:10E32000001303EB002008EBC0019DF81C0000EB7C
:10E33000001001EBC00000F5005080F831229DF87C
:10E34000080000EB4001C1EBC011FE4800EBC1002A
:10E35000407930287DD19DF80800464600EB001139
:10E3600001EB002008EBC0019DF81C0000EB001041
:10E3700001EBC00000F5005090F82C129DF8080049
:10E3800000EB001202EB002008EBC00000F500508B
:10E3900090F82802814275D19DF8080000EB4001F9
:10E3A00001EB00109DF81C1006EB001000EB0110B3
:10E3B0002844017821F0010101709DF8080000EB6C
:10E3C000400101EB00109DF81C1006EB001000EB63
:10E3D00001102844017821F0020101709DF8080025
:10E3E00000EB001101EB002006EBC0019DF81C00C2
:10E3F00000EB001001EBC00000F5005090F82F0278
:10E40000312829D19DF8080000EB400101EB0010F4
:10E410009DF81C1006EB001000EB01102844017859
:10E4200021F0200101709DF8080000EB001101EBC4
:10E43000002006EBC0019DF81C0000EB001001EB72
:10E44000C00000F5005080F869729DF808100220A5
:10E4500000E017E0FBF782F99DF8080000EB0011DF
:10E4600001EB002006EBC0019DF81C0000EB001042
:10E4700001EBC00000F5005090F86A0201287DD140
:10E48000A921C6E19DF80800AE4A00EB4001C1EBAE
:10E49000C01002EBC0004079312870D19DF808000F
:10E4A00000EB001101EB002008EBC0039DF81C00FD
:10E4B000414600EB001003EBC00000F5005090F85F
:10E4C0002C329DF8080000EB001606EB002008EB4C
:10E4D000C00000F5005090F8280283424FD19DF80B
:10E4E000080000EB001202EB002001EBC0029DF8D7
:10E4F0001C0000EB001002EBC00000F5005090F88B
:10E500006A0210BB9DF8080000EB001303EB00202B
:10E5100001EBC0039DF81C0000EB001003EBC000F2
:10E5200000F5005080F869929DF8080000EB400269
:10E5300002EB001001EB00129DF81C0002EB001032
:10E540002844027842F0010202709DF8080000EBB6
:10E55000400202EB001001EB00129DF81C0002EBE0
:10E5600000102844027822F00202027094F8AC07EE
:10E5700020B9487E012801D1886D01E067E0B6E04E
:10E580004A8B904263D29DF8080000EB001202EB28
:10E59000002001EBC0029DF81C0000EB001002EB14
:10E5A000C00000F5005090F8690201284FD19DF895
:10E5B000080000EB001202EB002001EBC0029DF806
:10E5C0001C0000EB001002EBC00000F5005090F8BA
:10E5D000A302E0BB9DF808004FF0104200EB0013CF
:10E5E00003EB002001EBC0039DF81C0000EB0010C2
:10E5F00003EBC00000F50050C0F834229DF808007D
:10E6000000EB400202EB001001EB00129DF81C0031
:10E6100002EB001000F5805000E0F3E390F8942D39
:10E620009DF8080000EB001303EB002001EBC00095
:10E6300000F5005080F825229DF8080000EB00123C
:10E6400002EB002001EBC0029DF81C0000E04DE051
:10E6500000EB001002EBC00000F5005090F82C22F7
:10E660009DF8080000EB001303EB002001EBC00055
:10E6700000F5005090F82802824237D19DF808003A
:10E6800000EB001202EB002001EBC0029DF81C0021
:10E6900000EB001002EBC00000F5005080F8327271
:10E6A0009DF80800A42200EB001303EB002001EB0F
:10E6B000C0039DF81C0000EB001003EBC00000F548
:10E6C000005080F82E229DF80800A32200EB0013D2
:10E6D00003EB002008EBC0019DF81C0000EB0010CC
:10E6E00001EBC00000F5005080F831221EE19DF8DA
:10E6F000080000EB4001C1EBC01002EBC000407904
:10E7000033289DF8080000EB400107D0C1EBC01092
:10E7100002EBC000407934287ED007E101EB001005
:10E720009DF81C10464608EB001000EB0110284431
:10E73000017841F0010101709DF8080000EB4001F3
:10E7400002E00000A064002001EB00109DF81C1006
:10E7500008EB001000EB01102844017821F02001A3
:10E7600001709DF8080000EB400101EB00109DF8DE
:10E770001C1006EB001000EB01102844017841F05A
:10E78000020101709DF8080000EB001101EB002070
:10E7900006EBC00000F5005090F828129DF8080024
:10E7A00000EB001202EB002006EBC0029DF81C00FB
:10E7B00000EB001002EBC00000F5005080F82C12B6
:10E7C0009DF8080000EB400101EB00109DF81C10C3
:10E7D00006EB001000EB01102844017841F08001A5
:10E7E00001709DF8080000EB400101EB00109DF85E
:10E7F0001C1006EB001000EB011000F5805090F8A3
:10E80000960D800704D49DF808100220FAF7A6FFA1
:10E81000A2219DF8080001E011E045E200EB0012A2
:10E8200002EB002006EBC0029DF81C0000EB00107C
:10E8300002EBC00000F5005080F82E1276E09DF843
:10E8400008009DF81C2000EB400101EB0011404640
:10E8500008EB011101EB021129440A7822F0200390
:10E860000B709DF8081001EB410202EB01119DF8BD
:10E870001C2008EB011101EB021129440A7822F057
:10E8800002030B709DF8081001EB011202EB01214D
:10E8900000EBC1069DF81C1001EB011106EBC10154
:10E8A00001F5005181F86A929DF80810A92301EB47
:10E8B000011202EB012100EBC1069DF81C1001EBD7
:10E8C000011106EBC10101F5005181F82E329DF8CE
:10E8D000081001EB011202EB012100EBC10101F56F
:10E8E000005191F828329DF8081001EB011202EB5B
:10E8F000012100EBC1069DF81C1001EB011106EB94
:10E90000C10101F5005181F82C329DF8081001EB8E
:10E91000410202EB011108EB01109DF81C1000EB05
:10E9200001102844017841F0800101700020CDE9F8
:10E9300000008DF82070FE4920E0DDE900021201A0
:10E9400042EA10720001CDE900029DF8080000EBD8
:10E950004002C2EBC0109DF8202001EBC000104423
:10E960008079DDE900363038C21718433243CDE9EB
:10E9700000029DF82000401C8DF820009DF820002A
:10E980000828DAD39DF80800009A00EB001303EB87
:10E99000002008EBC00C9DF81C00464600EB001060
:10E9A0000CEBC00000F50050C0F845220020CDE976
:10E9B000000002468DF8207020E00098120142EA23
:10E9C00010720001CDE900029DF8080000EB400242
:10E9D000C2EBC0109DF8202001EBC0001044C07BAA
:10E9E000DDE9003C3038C217184342EA0C02CDE999
:10E9F00000029DF82000401C8DF820009DF82000AA
:10EA00000628DAD39DF80800009A00EB001303EB08
:10EA1000002006EBC00C9DF81C0000EB00100CEB76
:10EA2000C00000F50050C0F860220020CDE90000D1
:10EA30008DF8207021E0DDE90002120142EA107237
:10EA40000001CDE900029DF8080000EB4002C2EB96
:10EA5000C0109DF8202001EBC0001044407DDDE98E
:10EA6000003C3038C217184342EA0C02CDE90002DC
:10EA70009DF82000401C8DF820009DF820000828FB
:10EA8000D9D39DF80800009A00EB001303EB002097
:10EA900006EBC0039DF81C0000EB001003EBC00068
:10EAA00000F50050C0F849229DF8080000EB400234
:10EAB000C2EBC01001EBC00041799DF8080000EBEB
:10EAC000001202EB002006EBC0029DF81C0000EBD8
:10EAD000001002EBC00000F5005080F82F129DF8E6
:10EAE000080000EB400101EB001006EB00119DF85F
:10EAF0001C0001EB001000F5805090F8961D9DF869
:10EB0000080000EB001202EB002006EBC0029DF8AB
:10EB10001C0000EB001002EBC00000F5005080F874
:10EB200044129DF8080000EB001101EB002006EBF9
:10EB3000C0019DF81C0000EB001001EBC00000F5C7
:10EB4000005090F82C129DF8080000EB001202EB28
:10EB5000002006EBC00000F5005090F8280281422A
:10EB600082F07D879DF8080000EB001101EB00208A
:10EB700006EBC00000F5005080F827729DF80800F1
:10EB8000A72100EB001202EB002006EBC0029DF86B
:10EB90001C0000EB001002EBC00000F5005080F8F4
:10EBA00031129DF8080000EB001202EB002006EB8A
:10EBB000C00000F5005080F827929DF8080000EB97
:10EBC000001101EB002006EBC00000F5005090F8AA
:10EBD00028129DF8080000EB001202EB002006EB63
:10EBE000C0029DF81C0000EB001002EBC00000F515
:10EBF000005080F82C129DF80800A12100EB0012B3
:10EC000002EB002006EBC0029DF81C0000EB001098
:10EC100002EBC00000F5005080F831129DF80800AA
:10EC200000EB400101EB001006EB00119DF81C0009
:10EC300001EB00102844017841F0800101709DF83B
:10EC4000080000EB400101EB00109DF81C1006EBE2
:10EC5000001000EB01102844017841F0040101701C
:10EC60009DF8080000EB400101EB00109DF81C101E
:10EC700006EB001000EB011000F5805090F8960DA7
:10EC8000800642F1EC869DF8080000EB400101EBA4
:10EC900000109DF81C1006EB001000EB011028443A
:10ECA000017821F0200101709DF8080000EB40017F
:10ECB00001EB00109DF81C1006EB001000EB01109A
:10ECC00000F5805090F8960D80073EF5B7AD9DF8A1
:10ECD000080000EB400101EB00109DF81C1006EB52
:10ECE000001000EB01102844017841F00801017088
:10ECF0009DF81C009DF8081000EB0110C117CDE92C
:10ED0000000100EB8001C1EB80103044C0F87D7041
:10ED10009DF8081001EB011202EB012106EBC10284
:10ED20009DF81C1001EB011102EBC10202E0000092
:10ED3000A064002042F24D21114410226D30F9F7F9
:10ED400084FA9DF8080000EB001101EB002006EBAF
:10ED5000C0019DF81C0000EB001001EBC001009801
:10ED600001F2452100EB800201F50051C2EB801059
:10ED70000A68304440F8612F496841609DF80810E6
:10ED800001EB410202EB01119DF81C2006EB011181
:10ED900001EB021101F5805191F8941D00F8011C5E
:10EDA0000A9951F86A2F0262898881849DF80810B7
:10EDB00001EB011202EB012106EBC1029DF81C10D0
:10EDC00001EB011102EBC10101F50051D1F8601214
:10EDD00081609DF8081001EB410202EB01119DF8E2
:10EDE0001C2006EB011101EB021101F58051D1F855
:10EDF000981DC0F82610009881B20820FAF7AEFCE2
:10EE0000FEF71CBDFFE79DF8080000EB001101EBC9
:10EE1000002006EBC00000F5005080F827729DF836
:10EE2000080000EB001202EB002008EBC0019DF887
:10EE30001C0000EB001001EBC00000F5005090F842
:10EE40002C02032813D89DF80800042100EB0012BF
:10EE500002EB00229DF81C0008EBC20200EB001040
:10EE600002EBC00000F5005080F82C1252E19DF832
:10EE70000800464600EB001101EB002008EBC00142
:10EE80009DF81C0000EB001001EBC00000F50050E5
:10EE900090F82C129DF8080000EB001202EB002005
:10EEA00008EBC00000F5005090F8280281427DD1A7
:10EEB00094F8AC0780B19DF8080000EB400101EB2D
:10EEC00000109DF81C1006EB001000EB0110284408
:10EED000017841F0080181E0C6F839709DF808001A
:10EEE00000EB001101EB002006EBC0019DF81C00B7
:10EEF000102200EB001001EBC00142F24D20014452
:10EF00000C98F9F7A2F99DF8080000EB001101EB4D
:10EF1000002006EBC0019DF81C0000EB001001EB87
:10EF2000C00000F2452000F500500168C6F81D1031
:10EF30004068C6F821009DF8080000EB400101EB95
:10EF4000001006EB00119DF81C0001EB001000F50D
:10EF5000805090F8940D30779DF8080000EB001178
:10EF600001EB002006EBC0019DF81C0000EB001037
:10EF700001EBC00000F50050D0F86002C6F8250093
:10EF80000A9850F86A1FC6F83D108088A6F841001C
:10EF9000B06D81B20220F9F7D7FD00210620FAF703
:10EFA000DDFBB06D718B884204D200E0B2E0B06D41
:10EFB000401CB06500210520FAF7D0FB9DF8080041
:10EFC00000EB400101EB00109DF81C1006EB001057
:10EFD00000EB01102844017821F0080101709DF830
:10EFE000080000EB001101EB002006EBC0019DF8CA
:10EFF0001C0000EB001001EBC00000F5005080F891
:10F000006A729DF808100220FAF7A8FB9DF81C0010
:10F010009DF8081000EB0110C117CDE9000100EBCD
:10F020008001C1EB80103044C0F87D709DF808105D
:10F0300001EB011202EB012106EBC1029DF81C104D
:10F040006D3001EB011102EBC10242F24D2111447E
:10F050001022F9F7FAF89DF8080000EB001101EB17
:10F06000002006EBC0019DF81C0000EB001001EB36
:10F07000C001009801F2452100EB800201F500512A
:10F08000C2EB80100A68304440F8612F4968416043
:10F090009DF8081001EB410202EB01119DF81C20C4
:10F0A00006EB011101EB021101F5805191F8941D5D
:10F0B00000F8011C0A9951F86A2F0262898881843C
:10F0C0009DF8081001EB011202EB012106EBC102D1
:10F0D0009DF81C1001EB011102EBC10101F500517B
:10F0E000D1F8601281609DF8081001EB410202EB3B
:10F0F00001119DF81C2006EB011101EB021101F535
:10F100008051D1F8981DC0F82610009881B20820CF
:10F11000FAF724FB9DF808003B4600EB001101EBD9
:10F12000002008EBC0019DF81C00424600EB0010D7
:10F1300001EBC00000F5005080F86A729DF80800ED
:10F14000A72100EB001606EB002008EBC0079DF896
:10F150001C0000EB001007EBC00000F5005080F829
:10F1600031129DF80800A22100EB001606EB0020EA
:10F1700002EBC0079DF81C0000EB001007EBC0007D
:10F1800000F5005080F82E120020CDE900008DF827
:10F190002030FE4921E0DDE90006360146EA10761E
:10F1A0000001CDE900069DF8080000EB4006C6EB23
:10F1B000C0109DF8206001EBC0003044C07ADDE94A
:10F1C000007C3038C617384346EA0C06CDE9000605
:10F1D0009DF82000401C8DF820009DF820000C2890
:10F1E000D9D3DDE900679DF8080000EB001C0CEBAB
:10F1F000002002EBC0089DF81C0000EB001008EB9B
:10F20000C00000F5005CCCF84D626046C0F8517259
:10F210000020CDE900008DF8203020E0DDE900037A
:10F220001B0143EA10730001CDE900039DF80800BB
:10F2300000EB4003C3EBC0109DF8203001EBC00091
:10F240001844C07DDDE900673038C31730433B43C5
:10F25000CDE900039DF82000401C8DF820009DF8AA
:10F2600020000C28DAD3DDE900139DF8080000EB3C
:10F27000001606EB002002EBC0029DF81C0000EB1C
:10F28000001002EBC00000F50052C2F85512104603
:10F29000C0F8593202F0E3BB9DF808005A464146D7
:10F2A0009DF81C3008EB0010184400F5805080F8E1
:10F2B00098BB9DF8080000EB4003C3EBC010B34BB4
:10F2C00003EBC000407870280AD19DF8080000EBDD
:10F2D0004006C6EBC01003EBC0008078FA2858D077
:10F2E0009DF8080000EB4006C6EBC01003EBC00021
:10F2F00040780C26B6EB101F0AD19DF8080000EBF1
:10F300004006C6EBC01003EBC0008078FA2842D05C
:10F310009DF8080000EB4006C6EBC01013F8300063
:10F320000526B6EB101F17D19DF8080000EB40062C
:10F33000C6EBC01003EBC00046780320B0EB161FED
:10F340000AD19DF8080000EB4006C6EBC01003EBA5
:10F35000C0008078ADF818009DF8080000EB00169A
:10F3600006EB002001EBC00000F5005090F826628B
:10F370008DF81C609DF8080001EB00169DF81C003C
:10F38000304400F5805080F8982B087E012804D086
:10F3900014E0B120DEE7B620DCE79DF8080000EBC2
:10F3A000400606EB00109DF81C6001EB001000EB1E
:10F3B00006102844067846F080060670BDF818004E
:10F3C000652872D002F34B83012803D0032842F052
:10F3D00046836BE09DF8080000EB4006C6EBC010CA
:10F3E00003EBC0000079012802F039830228FBD02A
:10F3F0000328F9D00528EAD19DF8080000EB001396
:10F4000003EB002001EBC0039DF81C0000EB001093
:10F4100003EBC00000F5005090F82C020028D6D174
:10F420009DF8080000EB001303EB002001EBC00087
:10F4300000F5005080F827229DF8080000EB00132B
:10F4400003EB002001EBC0039DF81C0000EB001053
:10F4500003EBC00000F5005080F82C929DF80800E6
:10F46000B62200EB001303EB002001EBC0039DF874
:10F470001C0000EB001003EBC00000F5005080F80A
:10F480003122B2229DF8080000EB001303EB0020AC
:10F4900008EBC0019DF81C0000EB001001EBC00060
:10F4A00000F5005080F82E22F4E61FE09DF80800D9
:10F4B00000EB4002C2EBC01003EBC000C07984F83F
:10F4C000E4019DF808009DF81C1000EB400202EBDF
:10F4D000001008EB001000EB011094F8E411284430
:10F4E000CA08017862F3000102F067BA9DF80800CB
:10F4F00000EB4006C6EBC01003EBC000007900092A
:10F5000012D0B920ADF818009DF8080000EB4006B5
:10F51000C6EBC01003EBC000007900F00F008DF8BF
:10F5200014008DF8202021E0B820EBE79DF80800BA
:10F5300000EB400606EB00109DF8206001EB001088
:10F5400000EB061000F5805090F8956D9DF80800CE
:10F5500000EB4007C7EBC01013F83000503886426C
:10F5600017D09DF82000401C8DF820009DF8080061
:10F5700000EB400606EB001001EB001000F5805098
:10F5800090F86B0D9DF82060B04201E0A06400206F
:10F59000CCD89DF820009DF8143018448DF81C003C
:10F5A0009DF8080000EB001303EB002001EBC00303
:10F5B0009DF81C0000EB001003EBC00000F50050AC
:10F5C00090F82C02012814D09DF8080000EB0013DD
:10F5D00003EB002001EBC0039DF81C0000EB0010C2
:10F5E00003EBC00000F5005090F82C02012842F017
:10F5F00036829DF8080000EB001303EB002001EBBE
:10F60000C00000F5005080F827229DF80800022273
:10F6100000EB001303EB002001EBC0039DF81C007E
:10F6200000EB001003EBC00000F5005080F82C2226
:10F63000B922EFE39DF8080000EB400101EB001157
:10F64000FE4800EB011000F5805090F8700D20B1DD
:10F6500001287CD00228CAD194E2F84E9DF8080017
:10F6600006EB400000F58040B0F84404801F81B2F2
:10F670009DF80800DFF8C88300EB4002C2EBC0121F
:10F6800008EBC200401CF9F7E9FDCDE9100B9DF82D
:10F6900008005F4606EB400000F58040B0F84414D7
:10F6A0009DF80800414400EB4002C2EBC0126FF02D
:10F6B000040000EBC200084404210AF07FFEC117D9
:10F6C000CDE90001DDE910235040594008438ED1B7
:10F6D0009DF8080006EB001000F5805080F8987B3C
:10F6E0009DF8080000EB4001C1EBC01108EBC10020
:10F6F0000079ADF81800BDF818003128ABD19DF89D
:10F70000080006EB400000F58040B0F844044121B9
:10F71000183890FBF1F0C117CDE9000184F88C0591
:10F720008DF82070BB46C7E09DF80800474600EB07
:10F730004001C1EBC01008EBC0019DF8200000EBB8
:10F7400080100844017D9DF82000304400E0BDE0B9
:10F7500000F5805080F88D159DF8080000EB400101
:10F76000C1EBC01008EBC0019DF8200000EB801039
:10F77000084408211A300AF0EDFD8DED0B0A10EE59
:10F78000100A9DF8201006EB011101F58051C1F817
:10F790009D059DF8080000EB4001C1EBC01007EB90
:10F7A000C0019DF8200000EB801008440821323091
:10F7B0000AF0D0FD8DED0B0A10EE100A9DF8201016
:10F7C00006EB011101F58051C1F899059DF808007B
:10F7D00000EB4001C1EBC01007EBC0019DF8200019
:10F7E00000EB8010084408213A300AF0B3FD8DED9B
:10F7F0000B0A10EE100A9DF8201006EB011101F51E
:10F800008051C1F8A1059DF8080000EB4001C1EB53
:10F81000C01007EBC0019DF8200000EB80100844E9
:10F82000082142300AF096FD8DED0B0A10EE100A09
:10F830009DF8201006EB011101F58051C1F8A505D6
:10F840009DF8080000EB400101EB00109DF820102E
:10F8500006EB001000EB01102844017841F0800114
:10F8600001709DF8080006EB400000F58040B0F8FC
:10F870004404C1199DF8080000EB4002C2EBC0101F
:10F880004FF0FF3202EBC000095C9DF8080000EB6E
:10F89000001202EB002006EBC0039DF81C0000EBF9
:10F8A000001003EBC00000F5005080F868129DF8CE
:10F8B0002000401C8DF820009DF82010DDE9002379
:10F8C000891A7BEB0300FFF62FAFE3E49DF80800F5
:10F8D0005B4E00EB4001C1EBC01006EBC000417D68
:10F8E0009DF8080000EB4002C2EBC01006EBC00020
:10F8F000807D41EA0020C117CDE900019DF8080094
:10F9000000EB4001C1EBC01006EBC0001521F9F778
:10F910008FFCCDE9100BDDE90001109F5A467840BD
:10F9200051400843D1D19DF8080000EB4001C1EBE4
:10F93000C01016F83000401E8DF81C003F4F9DF897
:10F94000080039469DF81C3007EB0010184400F5FC
:10F95000805080F8982B9DF81C00384400F58050AA
:10F9600080F88D259DF81C0007EB001000F58050F5
:10F97000C0F89D259DF8080000EB4002C2EBC010C6
:10F9800006EBC00082799DF8080000EB4003C3EB52
:10F99000C01006EBC000407942EA002000EE100AD9
:10F9A0009DF80800F8EE400A9FED260A80EE801AC6
:10F9B00000EB4002C2EBC01006EBC00002799DF8DC
:10F9C000080000EB4003C3EBC01006EBC000C0789A
:10F9D00042EA002000EE900A9DF81C00F8EE600A52
:10F9E00071EE200A10EE902A01EB001000F5805015
:10F9F000C0F899259DF8080000EB4002C2EBC0104A
:10FA000006EBC000827A9DF8080000EB4003C3EBD0
:10FA1000C01006EBC000407A42EA002000EE900AD7
:10FA20009DF80800B8EE601AC1EE000A00EB400233
:10FA3000C2EBC01006EBC000027A05E0A412002061
:10FA4000A064002000FF7F479DF8080000EB400302
:10FA5000C3EBC01006EBC000C07942EA002000EE04
:10FA6000100A9DF81C20B8EE400A30EE800A10EE15
:10FA7000100A01EB021101F58051C1F8A1059DF8B2
:10FA8000080000EB4001C1EBC01006EBC000C07ADB
:10FA900000069DF8080000EB4001C1EBC01006EB2A
:10FAA000C0001AD4017B9DF8080000EB4002C2EBB5
:10FAB000C01006EBC000C07A41EA002000EE100A38
:10FAC000B8EE400ADFEDF70A9DF81C2020EE200A70
:10FAD00010EE100A07EB02111BE0027B9DF80800F4
:10FAE00000EB4001C1EBC01006EBC000C07A42EA57
:10FAF0000020404280B2F8F775FD9FEDEB1B53EC00
:10FB0000112BF8F77DFCF8F7D2FD9DF81C1007EBE0
:10FB1000011101F58051C1F8A5059DF808009DF877
:10FB20001C2000EB400101EB001007EB001000EB84
:10FB300002102844027842F0800202709DF808000A
:10FB400000EB4002C2EBC01006EBC000C27D9DF886
:10FB5000080000EB001303EB002007EBC0039DF847
:10FB60001C0000EB001003EBC00000F5005080F813
:10FB700068229DF8080000EB400202EB001007EB42
:10FB80000010CFE09DF80800DFF8248300EB40016F
:10FB9000C1EBC01008EBC000C3799DF8080000EB72
:10FBA0004002C2EBC01008EBC000007A43EA00201C
:10FBB000C317CDE900039DF80800072100EB4002C0
:10FBC000C2EBC01008EBC000F9F732FBCDE9100B17
:10FBD000DDE90001109B5E465840714008437DD12D
:10FBE0009DF8080000EB4001C1EBC01118F831008E
:10FBF000401E8DF81C00AF4F9DF8081007EB011058
:10FC000000F5805080F8986B9DF81C10781800F56E
:10FC1000805080F88D659DF8080000EB4001C1EB35
:10FC2000C01108EBC1008079F8F7DCFC41EC110B46
:10FC30009FEDA10B0DF0D4F99DF80800B0EE408ABD
:10FC4000F0EE608A00EB4001C1EBC01108EBC1008F
:10FC500002799DF8080000EB4001C1EBC01108EBF0
:10FC6000C100C07842EA0020F8F7BCFC53EC182B26
:10FC7000F8F738FCF8F71BFD9DF81C1007EB011195
:10FC800001F58051C1F89D059DF81C1007EB01108E
:10FC900000F58050C0F899659DF81C1007EB011025
:10FCA00000F58050C0F8A1659DF81C1007EB01100D
:10FCB00000F58050C0F8A5659DF8080000EB4001F4
:10FCC00001EB001107EB01109DF81C1000EB011077
:10FCD0002844017841F08002027000E093E29DF830
:10FCE000080000EB4001C1EBC01108EBC100427AF3
:10FCF0009DF8080000EB001101EB00219DF81C00AD
:10FD000007EBC10300EB001003EBC00000F500504F
:10FD100080F868229DF8080000EB400101EB00111B
:10FD200007EB011000F5805090F86B0D84F88C05FE
:10FD3000CBE59DF808005E4E00EB4001C1EBC01022
:10FD400006EBC000C1789DF8080000EB4002C2EB52
:10FD5000C01006EBC000807841EA00208DF80C004E
:10FD60009DF8080000EB4001C1EBC0109DF80C109D
:10FD700006EBC000084441789DF8080000EB400203
:10FD8000C2EBC0109DF80C2006EBC000805C41EA7D
:10FD90000020C117CDE900019DF8080000EB4001EB
:10FDA000C1EBC01006EBC0009DF80C10F9F740FA4B
:10FDB000CDE9100BDDE90001109F5A467840514013
:10FDC0000843B5D19DF8080000EB4001C1EBC0101D
:10FDD00006EBC00040788DF81C008DF820204146CD
:10FDE0001CE09DF8080000EB400303EB00109DF8B9
:10FDF000203001EB001000EB031000F5805090F86C
:10FE0000950D9DF81C3098429DF8200003D18DF887
:10FE10001C0013E094E2401C8DF820009DF80800BF
:10FE200000EB400303EB001001EB001000F58050E5
:10FE300090F86B0D9DF820309842D2D89DF80800BC
:10FE400000EB400303EB001001EB00139DF81C00D6
:10FE500003EB00104319187840F080071F709DF8DD
:10FE6000080000EB4003C3EBC01006EBC0000379B1
:10FE7000ADF818309DF8080001EB00139DF81C0048
:10FE8000184400F5805080F8982BBDF81800F3282E
:10FE900006D015DC052878D0F12816D0F22890D1AC
:10FEA0004DE200000000803D000000000000B0BFF7
:10FEB000A0640020A41200200000000000002440E4
:10FEC000F42879D0F628EAD13BE29DF8080000EB4F
:10FED000001303EB002001EBC0039DF81C0000EBB6
:10FEE000001003EBC00000F5005090F82C0230B376
:10FEF0009DF8080000EB400303EB00109DF81C3058
:10FF000001EB001000EB031000F5805090F89D0D00
:10FF1000C00713D09DF8080000EB001303EB00238B
:10FF20009DF81C0001EBC30300EB001003EBC000C5
:10FF300000F5005090F8B202C00727D0B9E09DF854
:10FF4000080000EB001707EB002001EBC0079DF84D
:10FF50001C0000EB001007EBC00000F5005080F81B
:10FF60002C929DF80800F42300EB001707EB00200B
:10FF700001EBC0079DF81C0000EB001007EBC00070
:10FF800000F5005080F8313293E054E29DF808000B
:10FF900000EB001303EB002001EBC0039DF81C00F5
:10FFA00000EB001003EBC00000F5005090F8A40235
:10FFB000B0B38DF820202BE0D7E19DF8080000EBCE
:10FFC000001303EB002001EBC0039DF81C0000EBC5
:10FFD000001003EBC0039DF82000184400F500500A
:10FFE00090F8A5329DF8080000EB400707EB0010E1
:10FFF00001EB00179DF82000384400F5805090F880
:020000040801F1
:10000000720D834208D19DF82000401C8DF820001D
:100010009DF820000428D0D39DF82000042829D082
:1000200047E09DF8080000EB001303EB002001EB14
:10003000C0039DF81C0000EB001003EBC0039DF80B
:100040002000184400F5005090F8A5329DF80800F3
:1000500000EB400707EB001001EB00179DF82000B4
:10006000384400F5805090F8720D834208D19DF815
:100070002000401C8DF820009DF820000A28D0D3D5
:100080009DF820000A2814D09DF8080000EB00130A
:1000900003EB002001EBC0079DF81C0042F2B223E5
:1000A00000EB001007EBC0001844037843F0010791
:1000B00007709DF80C00112845D09DF80C001428FD
:1000C0009DF8080000EB400303EB00109DF81C3086
:1000D00001EB001000EB03102844037874D023F0E8
:1000E000040606709DF8080000EB001303EB0020E7
:1000F00001EBC0069DF81C0000EB001006EBC000F1
:1001000000F5005090F8B202C0077CD09DF80800BE
:1001100000EB001303EB002001EBC0039DF81C0073
:1001200000EB001003EBC00000F50050A0F8B02277
:100130009DF80800052200EB001303EB002001EB03
:10014000C001FCF79BBE9DF8080000EB400303EBE9
:1001500000109DF81C3001EB001000EB0310284448
:10016000037843F0040303708DF8202025E09DF808
:10017000080000EB4003C3EBC0109DF8203006EBF5
:10018000C000184443799DF8080000EB001707EB06
:10019000002001EBC0079DF81C0000EB001007EBEE
:1001A000C0009DF82070384400F5005080F86B3294
:1001B0009DF82000401C8DF820009DF820000A28A2
:1001C000D5D38DF8202028E02CE09DF8080000EB26
:1001D0004002C2EBC01006EBC0029DF820001044A4
:1001E000C27B9DF8080000EB001303EB002001EB3D
:1001F000C0039DF81C0000EB001003EBC0009DF84D
:100200002030184400E077E200F5005080F88422A6
:100210009DF82000401C8DF820009DF82000022849
:10022000D3D385E543F0040707708DF8202025E03F
:100230009DF8080000EB4003C3EBC0109DF8203090
:1002400006EBC000184443799DF8080000EB001746
:1002500007EB002001EBC0079DF81C0000EB00102D
:1002600007EBC0009DF82070384400F5005080F87E
:100270006B329DF82000401C8DF820009DF8200076
:100280000A28D5D38DF820201AE0C27B9DF80800FB
:1002900000EB001303EB002001EBC0039DF81C00F2
:1002A00000EB001003EBC0009DF82030184400F56F
:1002B000005080F884229DF82000401C8DF820001A
:1002C0009DF8200002289DF8080000EB4002C2EBD8
:1002D000C0109DF8202006EBC0001044D5D3407C10
:1002E00002049DF8080000EB4003C3EBC0109DF82A
:1002F000203006EBC0001844807C42EA00229DF8C2
:10030000080000EB4003C3EBC0109DF8203006EB63
:10031000C0001844C07C02439DF8080000EB0013A5
:1003200003EB002001EBC0019DF81C0000EB001066
:1003300001EBC00000F50050C0F89822F8E4F1226B
:10034000FDE39DF80800032200EB001303EB0020FF
:1003500001EBC0039DF81C0000EB001003EBC00094
:1003600000F5005080F82C22E9E79DF808000223F0
:1003700000EB001707EB002001EBC0079DF81C0005
:1003800000EB001007EBC00000F5005080F82C32A5
:100390009DF80800F62300EB001707EB002001EBA7
:1003A000C0079DF81C0000EB001007EBC00000F533
:1003B000005080F831329DF8080000EB001707EB81
:1003C000002001EBC0079DF81C0000EB001007EBBC
:1003D000C00000F5005080F8A4928DF8202025E0A0
:1003E0009DF8080000EB4002C2EBC0109DF82020F1
:1003F00006EBC000104442799DF8080000EB0013A2
:1004000003EB002001EBC0039DF81C0000EB001083
:1004100003EBC0009DF82030184400F5005080F830
:10042000A5229DF82000401C8DF820009DF820009A
:100430000A28D5D37CE49DF8080000EB4002C2EB0B
:10044000C01006EBC00082799DF8080000EB400365
:10045000C3EBC01006EBC000407942EA00229DF8D1
:10046000080000EB001303EB002001EBC0039DF834
:100470001C0000EB001003EBC00000F50050A0F8DA
:10048000B0229DF8080000EB001202EB002001EB07
:10049000C0029DF81C0000EB001002EBC00000F54C
:1004A0000050B0F8B0229DF8080000EB400303EBC9
:1004B000001001EB001000F58050B0F87E0D824274
:1004C000B8D39DF80800F12200EB001303EB0020E5
:1004D00001EBC0039DF81C0000EB001003EBC00013
:1004E00000F5005080F831229DF8080000EB001262
:1004F00002EB002008EBC0019DF81C0000EB00108F
:1005000001EBC00042F2B2210844017821F0010160
:10051000FEE39DF8080000EB4001C1EBC010FE4F68
:1005200007EBC00000798DF81C008DF810B046462E
:100530001BE09DF8080000EB400101EB001006EB0A
:1005400000119DF8100001EB001000F5805090F8AC
:10055000950D9DF81C1088429DF8100002D18DF871
:100560001C0012E0401C8DF810009DF8080000EB04
:10057000400101EB001006EB001000F5805090F8F0
:100580006B0D9DF810108842D3D89DF8080000EB41
:100590004001C1EBC01007EBC000C078ADF81800F7
:1005A000BDF8180017280FD2DFE800F00E6C6C0EB3
:1005B0007070706A6C0E0E0E0E0E0E6E70700E0E57
:1005C000727274008DF80C009DF80C00001FC1B20F
:1005D0009DF8080000EB4002C2EBC01007EBC00022
:1005E000C01CF8F753FC8DF800009DF8080000EBE4
:1005F0004001C1EBC0109DF80C1007EBC00008448F
:1006000010F8010C9DF80010884275D19DF8080083
:1006100000EB4001C1EBC01007EBC00040780028A0
:100620006AD09DF8080000EB4001C1EBC011BA4848
:1006300000EBC1009DF80C10425C9DF80800B0462C
:1006400000EB001101EB0020314606EBC0069DF8DF
:100650001C0000EB001006EBC00000F5005080F815
:1006600068229DF808209DF81C3001EB02121A4404
:1006700002F5805282F898BB087E01280CD01CE05D
:1006800012209FE707209DE709209BE7062099E7B6
:100690000B2097E72A2095E79DF8080000EB400122
:1006A00001EB001108EB01109DF81C1000EB01108C
:1006B0002844017841F080010170BDF81800072836
:1006C0007ED007DC072817D2DFE800F016FDFC1605
:1006D000FBFAF90010380728F5D2DFE800F0F2F253
:1006E0000D0D0404F500BDF81800142805D0BDF860
:1006F0001800152865D01DE1C1E39DF8080000EB46
:100700004001C1EBC010844901EBC000027A9DF8A2
:10071000080000EB4003C3EBC01001EBC0004079C0
:1007200042EA00629DF8080000EB4003C3EBC010F2
:1007300001EBC000807903049DF8080000EB40063F
:10074000C6EBC01001EBC000C07943EA00200243B1
:100750009DF8080000EB001101EB00219DF81C0042
:1007600008EBC10100EB001001EBC00000F50050E8
:10077000C0F845229DF8080000EB001101EB0021B4
:100780009DF81C0008EBC10100EB001001EBC0005C
:1007900000F50050D0F84502002103F003FBCDE93D
:1007A00000019DF8080000EB400101EB001108EB8F
:1007B000011000F5805090F8800D00F0030101E079
:1007C000F7E36BE09DF8080000EB400202EB00123B
:1007D00008EB021000F5805090F8800DC0F3011076
:1007E00001449DF8080000EB400202EB001208EB08
:1007F000021000F5805090F8800DC0F38100081AB7
:10080000F7F7DFFE41EC110B9FED440B0CF0E8FB1A
:1008100051EC100BF7F726FFCDE910019DF8080009
:1008200000EB001101EB00219DF81C0008EBC10159
:1008300000EB001001EBC00000F50050D0F86002A2
:10084000002103F0AFFADDE90023A0FB026701FB02
:10085000027100FB0317DDE9100102220023F7F704
:10086000B1FCDDE9102330187941F7F7ABFCCDE995
:10087000000103F047FF9DF8081001EB011202EBA5
:1008800001229DF81C1008EBC20201EB011102EBE2
:10089000C10101F50051C1F849024BE09DF8080083
:1008A00000EB4001C1EBC0101B4901EBC000027A14
:1008B0009DF8080000EB4003C3EBC01005E0FDE32A
:1008C00047E3FCE397E388E3C5E301EBC00040792D
:1008D00042EA00629DF8080000EB4003C3EBC01041
:1008E00001EBC000807903049DF8080000EB40068E
:1008F000C6EBC01001EBC000C07943EA0020024300
:100900009DF8080000EB001101EB002108EBC1018C
:100910009DF81C0006E00000A0640020000000001C
:100920000000244000EB001001EBC00000F5005077
:10093000C0F849229DF8080000EB4001C1EBC0114E
:10094000FE4800EBC100407A84F8E3019DF80800FE
:10095000464600EB400101EB00109DF81C1008EB2F
:10096000001000EB011094F8E3112844CA09017843
:1009700062F30001017094F8E30100F00300012824
:100980007ED094F8E301C043800779D09DF8080039
:1009900000EB400101EB00109DF81C1006EB00106D
:1009A00000EB01102844017821F0020101709DF84C
:1009B000080000EB400101EB00109DF81C1006EB55
:1009C000001000EB011000F5805090F8960DC0F378
:1009D00040019DF8080000EB001202EB002006EB3E
:1009E000C0029DF81C0000EB001002EBC00000F5F7
:1009F000005090F84402C0F34000814261D09DF85D
:100A0000080000EB001101EB002006EBC0019DF88F
:100A10001C0000EB001001EBC00042F24421014435
:100A20009DF8080000EB400202EB00109DF81C202E
:100A300006EB001000EB021000F5805090F8960DC8
:100A40004208087862F3410008709DF8080000EB46
:100A5000400101EB00109DF81C1006EB001000EBAC
:100A6000011000F5805090F8960D800724D49DF871
:100A7000080000EB400101EB001008EB001000E063
:100A8000BCE09DF81C2000EB02102844027822F004
:100A9000200202709DF8080000EB001303EB002019
:100AA00006EBC0019DF81C0000EB001001EBC0003C
:100AB00000F5005080F86A929DF808100220F8F7BF
:100AC0004DFE9DF808009DF81C2000EB400101EB55
:100AD0000010B04606EB001000EB021000F580504D
:100AE00090F8960D00F001029DF8080000EB00134D
:100AF00003EB002006EBC0019DF81C0000EB00108A
:100B000001EBC00000F5005090F8440200F0010035
:100B1000824272D09DF80800464600EB001101EBBE
:100B2000002008EBC0019DF81C0000EB001001EB59
:100B3000C00042F2442101449DF8080000E0D3E1E6
:100B400000EB400202EB00109DF81C2008EB0010A7
:100B500000EB021000F5805090F8960D0A7860F3D3
:100B600000020A709DF8080000EB400101EB001044
:100B70009DF81C1006EB001000EB011000F58050F2
:100B800090F8960DC0079DF808005CD000EB0011AE
:100B900001EB002006EBC0019DF81C0000EB0010EB
:100BA00001EBC00000F5005090F86A02F0B39DF828
:100BB000080000EB001202EB002006EBC0029DF8DB
:100BC0001C0000EB001002EBC00000F5005080F8A4
:100BD00069B29DF8080000EB400101EB001006EB44
:100BE00000119DF81C0001EB00102844017821F051
:100BF0000101017094F8AC07E8B318E19DF8080012
:100C000000EB400101EB00109DF81C1006EB0010FA
:100C100000EB01102844017841F0020202709DF8B7
:100C2000080000EB400101EB001000E02FE09DF810
:100C30001C1006EB001000EB01102844017821F095
:100C400020020270B3E600EB400101EB00109DF8BA
:100C50001C1006EB001000EB01102844017821F075
:100C6000200101709DF8080000EB001202EB00204B
:100C700008EBC00200E01DE09DF81C0000EB001036
:100C800002EBC00000F5005080F869B2CFE09DF89B
:100C9000080000EB001202EB002006EBC0029DF8FA
:100CA0001C0000EB001002EBC00000F5005080F8C3
:100CB00069929FE7707E012869D1B06D718B88427F
:100CC00065D29DF8080000EB001101EB002006EB57
:100CD000C0019DF81C0000EB001001EBC00000F506
:100CE000005090F86902012851D19DF8080000EBEE
:100CF000001101EB002006EBC0019DF81C0000EB89
:100D0000001001EBC00000F5005090F8A30200E0D5
:100D1000FEE3E0BB9DF8080000EB400101EB001092
:100D200006EB00119DF81C0001EB001000F580504F
:100D300090F8941D9DF8080002E00000A0640020D7
:100D400000EB001202EB002006EBC00000F50050A3
:100D500080F825129DF80800052100EB001202EB37
:100D6000002006EBC0029DF81C0000EB001002EB17
:100D7000C00000F5005080F831129DF808005F4671
:100D800000EB400101EB001006EB001100E04EE02B
:100D90009DF81C0001EB001000F58050C0F898BDD4
:100DA0009DF808100220F8F7D9FC8DF8207019E0A2
:100DB0009DF8080000EB001101EB002006EBC001DC
:100DC0009DF81C0000EB001001EBC0009DF8201006
:100DD000084400F5005080F86B729DF82000401C1C
:100DE0008DF820009DF820001428E1D38DF82070A4
:100DF00019E09DF8080000EB001101EB002006EB64
:100E0000C0019DF81C0000EB001001EBC0009DF834
:100E10002010084400F5005080F887729DF82000EB
:100E2000401C8DF820009DF820000A28E1D39DF891
:100E3000080000EB001101EB002008EBC0029DF858
:100E40001C00414600EB001002EBC00000F5005012
:100E500090F82C02012813D89DF80800022200EB1C
:100E6000001303EB002008EBC0019DF81C0000EB11
:100E7000001001EBC00000F5005080F82C2225E3A3
:100E80009DF8080000EB001202EB002001EBC0020D
:100E90009DF81C0000EB001002EBC00000F50050B4
:100EA00090F82C0202282ED89DF8080000EB0013C1
:100EB00003EB002001EBC00000F5005080F827B2E2
:100EC0009DF80800032200EB001303EB002001EB68
:100ED000C0039DF81C0000EB001003EBC00000F500
:100EE000005080F82C2207229DF8080000EB001328
:100EF00003EB002008EBC001FBF7C0BF00F500507A
:100F000080F83122E2E29DF8080000EB001202EBCB
:100F1000002001EBC0029DF81C0000EB001002EB6A
:100F2000C00000F5005090F82C229DF8080000EB5E
:100F3000001303EB002001EBC00000F5005090F817
:100F4000280282429BD194F8E301800697D51622AD
:100F5000CAE79DF80800142200EB001101EB002005
:100F600008EBC0039DF81C0000EB001003EBC00071
:100F700000F5005080F831229DF8080000EB0013C6
:100F800003EB002008EBC00000F5005080F827922A
:100F90009DF8080000EB400202EB001008EB001087
:100FA0009DF81C1000EB01102844017841F020014D
:100FB000AEE215E19DF8080000EB001202EB002202
:100FC00008EBC2029DF81C0000EB001002EBC00011
:100FD00000F5005080F8311278E29DF8080000EB2F
:100FE000001101EB002008EBC00000F5005080F874
:100FF00027B2052278E79DF8080000EB001101EB0D
:10100000002008EBC00000F5005080F827929DF802
:101010000800142200EB001303EB002008EBC003D0
:101020009DF81C0000EB001003EBC00000F5005021
:1010300080F831229DF8080000EB400202EB00101E
:1010400008EB00109DF81C1000EB011028440178FB
:1010500041F004015CE20020CDE900005E468DF81D
:1010600020B01EE0090241EA10610002CDE9000152
:101070009DF8080000EB4001C1EBC011FE4800EBF9
:10108000C1009DF8201008444079DDE900120843B2
:1010900046EA0201CDE900019DF82000401C8DF8D0
:1010A00020009DF820000328DDE90001DAD303F0D9
:1010B00029FB9DF8081001EB011201E019E35EE342
:1010C00002EB012108EBC1029DF81C10474601EB21
:1010D000011102EBC10101F50051C1F849020020E4
:1010E000CDE900008DF82060DFF88C831DE0090257
:1010F00041EA10610002CDE900019DF8080000EB13
:101100004001C1EBC01108EBC1009DF8201008445C
:10111000017ADDE90023114346EA0300CDE900101E
:101120009DF82000401C8DF820009DF82000032829
:10113000DDE90001DBD303F0E5FA9DF8081001EBCF
:10114000011202EB012107EBC1029DF81C1001EB1B
:10115000011102EBC10101F50051C1F84502002067
:10116000CDE9000002468DF8206041461EE000985F
:10117000120242EA10620002CDE900029DF8080066
:1011800000EB4002C2EBC0109DF8202001EBC00034
:101190001044C07CDDE90023104346EA0302CDE998
:1011A00000029DF82000401C8DF820009DF82000D2
:1011B0000328DCD39DF80800009900EB001202EB35
:1011C000002007EBC0029DF81C0000EB001002EBB2
:1011D000C00000F50050C0F860120721FAF7A0BF68
:1011E0000021CDE900115F468DF820B01EE0090214
:1011F00041EA10610002CDE900019DF8080000EB12
:101200004001C1EBC0119C4800EBC1009DF82010CB
:1012100008444179DDE90002014347EA0200CDE9D3
:1012200000109DF82000401C8DF820009DF8200043
:10123000042808460199DAD303F064FA9DF80820DF
:10124000464602EB021303EB022208EBC2039DF8B1
:101250001C2002EB021203EBC20202F50053C3F89A
:1012600055021A46C2F859120020CDE90000014685
:101270008DF82070B846804A1DE0090241EA1061ED
:101280000002CDE900019DF8080000EB4001C1EB30
:10129000C0109DF8201002EBC0000844407ADDE940
:1012A0000037184348EA0701CDE900019DF8200006
:1012B000401C8DF820009DF8200004280098DCD305
:1012C00003F020FA9DF8082002EB021303EB022240
:1012D00006EBC2039DF81C2002EB021203EBC202D4
:1012E00002F50053C3F84D021A46C2F851129DF898
:1012F000080000EB001101EB002006EBC0019DF897
:101300001C0000EB001001EBC00000F5005090F84D
:101310002C129DF8080000EB001202EB002006EBF7
:10132000C00000F5005090F8280281427ED194F868
:10133000E301800601D5172100E014219DF8080083
:1013400000EB001202EB002006EBC0029DF81C002F
:1013500000EB001002EBC00000F5005080F83112E5
:1013600094F8AC07F0B39DF8080000EB400101EBE6
:1013700000109DF81C1006EB001000EB0110284433
:10138000017841F0080101709DF8080000EB00129F
:1013900002EB002006EBC0029DF81C0000EB0010E1
:1013A00002EBC00000F5005080F86A829DF808103A
:1013B0000220F8F7D3F99DF81C009DF8081000EB07
:1013C0000110C117CDE9000100EB8002C2EB8010D3
:1013D0003044C0F87D809DF8081001EB011202EB4B
:1013E000012100E073E006EBC1029DF81C106D3096
:1013F00001EB011102EBC10242F24D211144102216
:10140000F6F723FF9DF8080000EB001101EB002028
:1014100006EBC0019DF81C0000EB001001EBC001C1
:10142000009800EB8002C2EB801000E0E5E001F2E2
:10143000452101F5005130440A6840F8612F4968A0
:1014400041609DF8081001EB410202EB01119DF88B
:101450001C2006EB011101EB021101F5805191F8FE
:10146000941D00F8011C0A9951F86A2F02628988BC
:1014700081849DF8081001E0A064002001EB0112B6
:1014800002EB012106EBC1029DF81C1001EB0111DA
:1014900002EBC10101F50051D1F8601281609DF8A5
:1014A000081001EB410202EB01119DF81C2006EB34
:1014B000011101EB021101F58051D1F8981DC0F81E
:1014C0002610009881B20820F8F748F9C7E29DF885
:1014D000080000EB001202EB002006EBC0029DF8B2
:1014E0001C0000EB001002EBC00000F5005080F87B
:1014F0006A82C6F839809DF8080000EB001101EB04
:10150000002006EBC0019DF81C0000EB001000E07D
:1015100053E201EBC00142F24D20014410220C982D
:10152000F6F793FE9DF8080000EB001101EB002098
:1015300006EBC0019DF81C0000EB001001EBC000A1
:1015400000F2452000F500500168C6F81D10406803
:10155000C6F821009DF8080000EB400101EB0010E7
:1015600006EB00119DF81C0001EB001000F5805007
:1015700090F8940D30779DF8080000EB001101EB16
:10158000002006EBC0019DF81C0000EB001001EBF1
:10159000C00000F50050D0F86002C6F825000A9897
:1015A00050F86A1FC6F83D108088A6F84100B06D5B
:1015B00081B20220F7F7C8FA00210620F8F7CEF82A
:1015C000B06D718B884202D2B16D491CB1650021AA
:1015D0000520F8F7C3F89DF8080000EB400101EB87
:1015E000001106EB01109DF81C1000EB01102844BF
:1015F000017821F008010170D8E69DF8080000EBA1
:10160000001101EB002006EBC0019DF81C0000EB6F
:10161000001001EBC00000F5005090F82C129DF86E
:10162000080000EB001202EB002006EBC00000F502
:10163000005090F8280281427ED29DF8080000EB0D
:10164000400101EB00109DF81C1006EB001000EBB0
:1016500001102844017841F0040202709DF808004E
:1016600000EB400101EB00109DF81C1006EB001090
:1016700000EB01102844017841F0800202709DF8CF
:10168000080000EB001101EB002006EBC00000F5A4
:10169000005080F827929DF8080000EB001101EB44
:1016A000002006EBC00000F5005090F828229DF8BD
:1016B000080000EB001101EB002006EBC0039DF8D1
:1016C0001C0000EB001003EBC00000F5005080F898
:1016D0002C229DF80800142200EB001101EB0020E1
:1016E00006EBC0039DF81C0000EB001003EBC000EC
:1016F00004E44A4684F8E8969DF8080000EB0011DF
:1017000001EB002008EBC0039DF81C00414600EBF4
:10171000001003EBC00000F5005090F82C329DF84B
:10172000080000EB001606EB002008EBC00000F5F7
:10173000005090F8280200E07FE083427DD29DF8BF
:10174000080000EB001606EB002001EBC00000F5DE
:10175000005080F827B29DF8080000EB001303EB5F
:10176000002001EBC0039DF81C0000EB001003EB10
:10177000C00000F5005080F82C2214223AE4142115
:1017800018E406EB400000F5805090F82C0B0006A2
:1017900053D49DF8080006EB400000F5805090F807
:1017A0002C0BC0F3C300062847D2DFE800F0036328
:1017B00087F2F1329DF8080000EB4001C1EBC01147
:1017C000C84800EBC100C8A10CF0F0FE5FEA000AB7
:1017D00033D09DF8080000EB400006EB800000F5D8
:1017E0008050C0F86CBB9DF8080000EB400006EB91
:1017F000800000F5805080F86A9B9DF8080006EB99
:10180000400141F62C300844017821F0780128315C
:10181000D3E09DF8080000EB4001C1EBC011B148D6
:1018200000EBC100B0A10CF0C1FE5FEA000A04D0D9
:101830009DF8080000EB400000E0A8E006EB800007
:1018400000F58050C0F86CBB9DF8080000EB40002C
:1018500006EB800000F5805080F86A9B9DF8080038
:1018600006EB400141F62C300844017821F0780164
:101870002031A2E09DF8080000EB4001C1EBC0114F
:10188000984800EBC10098A10CF090FE5FEA000AB6
:101890007DD09DF8080000EB400006EB800000F5CD
:1018A0008050C0F86CBB9DF8080000EB400006EBD0
:1018B000800000F5805080F86A9B73E09DF8080076
:1018C00000EB400006EB800000F58050C0F86CBBD8
:1018D0009DF8080000EB400006EB800000F580500A
:1018E00080F86A9B9DF808007E4F00EB4001C1EB39
:1018F000C01007EBC00101EB0A0081799DF80800D8
:1019000000EB4002C2EBC01007EBC00303EB0A0080
:1019100040793039303841EA0010C11702F042FAFC
:1019200084F8B2079DF8080000EB4001C1EBC0103D
:1019300007EBC0006DA10CF039FE5FEA000A31D060
:101940009DF8080000EB4001C1EBC01007EBC0019F
:1019500001EB0A00407830289DF8080000EB4001B8
:10196000C1EBC01007EBC00114D301EB0A004178B2
:101970009DF8080000EB4002C2EBC01007EBC0026C
:1019800012F80A003038303941EA001005E03FE033
:101990003FE014E011F80A003038C11702F002FAF3
:1019A00084F8B3079DF8080006EB400141F62C309F
:1019B0000844017821F07801183101704FE09DF85A
:1019C000080000EB4001C1EBC011464800EBC1002C
:1019D00045A10CF0EBFD5FEA000A40D04449C1F894
:1019E00088B29DF8080006EB400141F62C3008440F
:1019F000017841F0800101709DF808004FF47A7180
:101A000000EB400006EB800000F58050C0F8701B32
:101A100025E09DF8080000EB4001C1EBC011314802
:101A200000EBC10030A10CF0C1FD5FEA000A16D046
:101A300094F8EA0620F0800084F8EA069DF8080091
:101A400006EB400141F62C300844017821F0780182
:101A500008310170099981F886B4C1F888B494F806
:101A6000E903B0B123489DF8081000EB410000F5F0
:101A70008040B0F844149DF80800012300EB4002B8
:101A8000C2EBC012174800EBC2009DF80820F8F71F
:101A9000BDFA59468DF820B0124A0FE09DF80800B3
:101AA00000EB4003C3EBC0109DF8203002EBC000F8
:101AB000C1549DF82000401C8DF820009DF82000A6
:101AC0001428EBD30C4801784278114482781144F1
:101AD000C278D14278F460AC1FB0BDEC028BBDE897
:101AE000F08F0000A06400204F4B00002C0000008D
:101AF00000004242A4120020120000202DE9F74FFE
:101B000096B000209246ADF80800ADF81400ADF88C
:101B10000000ADF800008DF820008DF810008DF861
:101B20002800CDE91000CDE90000ADF80C00FEA1C1
:101B3000D1E90031CDE90631FDA1D1E90031CDE98E
:101B40000B31FD490871169800EB400101EB0010C4
:101B5000FA4901EB0010139000F58050814690F88F
:101B60006A0D8DF820001698179A01EB0010159059
:101B7000104400F58050009090F8983B1698052B83
:101B800000EB001202EB00200A4602EBC00E179A8F
:101B9000139802EB02120EEBC20B179A0BF50057CB
:101BA00000EB021000F58050059038D9009806230C
:101BB00080F8983B002087F82C02059890F8960D45
:101BC00020F08002059880F8962D97F8B20220F058
:101BD000080087F8B202169800EB00100EEBC00068
:101BE00000F5005090F8B22222F0010280F8B222F3
:101BF00099F86A2DA120082A11D2DFE802F010041A
:101C00000B0B06080A0EE52004E0B12002E03120AB
:101C100000E0F12087F8310201E087F831321698B0
:101C200001EB400000F58050019090F82C0BC44E61
:101C300002061698DFF80C83C0EB001000EB80045E
:101C400041F14D8799F8711D1698022900EB001299
:101C500002EB0020B94A02EBC00505F5005517D08C
:101C60001046007E012801F032879DF820300221C5
:101C70004122AAF1A100082B81F0CE86DFE813F003
:101C8000F8033D036506ED075E09530AC90A670CB0
:101C900008F05AF9C8F8F803D8F8F803C0F3004080
:101CA0000090D8F8F803C0F342005FEA000BEFD0D1
:101CB000552006F8340006EBC404FD206070AA200D
:101CC000A0700021E170217161206071A171FA2082
:101CD000E07198F8EF03207298F8EE03607298F8BC
:101CE000ED03A07298F8EC03E07298F8EB03207310
:101CF00098F8EA036073ADF8081010E0D8F8F8031C
:101D0000BDF80820C2F10302D200D040BDF808207F
:101D100022441074BDF80800401CADF80800BDF85E
:101D200008000428EAD384F814A01520ADF80C00AC
:101D30000020824F85F82902BAF100007ED01228D7
:101D400014D009DCAAF10B00072815D2DFE800F057
:101D5000FE0E0E0E0E0E0E00A228F1D007DC142887
:101D6000EED01528ECD0BAF1A10F05D122E2A328BC
:101D700010D0BAF1A40FF9D00021ADF80C10ADF8D5
:101D80000810169800EB4002C2EBC0106E4A02EB3E
:101D9000C0020BE295F82A021699C0EB001000EB86
:101DA0008000BDF80C2006EBC000491C8154BDF832
:101DB0000C00401CADF80C0095F82A0200EB400125
:101DC00001EB001007EB001000F58050D0F8640D17
:101DD0000026314602F096FCCDE91001ADF808600E
:101DE00013E0BDF80800C0F10200C200DDE91001F7
:101DF000F6F719FABDF80C10BDF80820114460542C
:101E0000BDF80800401CADF80800BDF80800032824
:101E1000E7D3BDF80C00C01CADF80C0095F82A0201
:101E200000EB400101EB001007EB001000F58050C3
:101E300090F8680D002105F22A2500E0DAE202F0B0
:101E400061FCBDF80C106054BDF80C00401CADF8EE
:101E50000C00287800EB400101EB001007EB0010AC
:101E600000F5805090F8690D002102F04BFCBDF8A0
:101E70000C106054BDF80C00401CADF80C00287824
:101E800000EB400101EB001007EB001000F5805063
:101E900090F86A0D002102F035FCBDF80C1060547A
:101EA000BDF80C00401CADF80C00287800EB400198
:101EB00001EB001007EB001000F5805090F86B0D5F
:101EC000002102F01FFCBDF80C106054BDF80C009E
:101ED000401CADF80C00287800EB400101EB00102D
:101EE00007EB001000F58050D0F86C0D002102F0D7
:101EF00009FCBDF80C106054BDF80C00401CADF896
:101F00000C00287800EB400101EB001007EB0010FB
:101F100000F5805090F8700D0021A5F22A2502F0FE
:101F2000F1FBBDF80C1012E00169323031303000A5
:101F3000016932304530300012000020A412002028
:101F4000405B0020A4220020A06400200AE160542D
:101F5000BDF80C00401CADF80C0099F86A0DADF806
:101F60000860062868D03E46B2E0BDF808104FF081
:101F7000030AB1FBFAF195F82A0200EB400202EBEA
:101F8000001007EB001000EB011000F5805090F8F6
:101F9000940D314602F0B6FBBDF80C10BDF80820D8
:101FA00011446054BDF80C00401CADF80C00BDF8A5
:101FB000081095F82A02B1FBFAF100EB400202EB9F
:101FC000001007EB001000EB011000F5805090F8B6
:101FD000950D314602F096FBBDF80C20BDF80810B7
:101FE00011446054BDF80C00401CADF80C00BDF865
:101FF000081095F82A02B1FBFAF100EB400202EB5F
:10200000001007EB001000EB011000F5805090F875
:102010009C0D314602F076FBBDF80C20BDF808108F
:1020200011446054BDF80C00401CADF80C00BDF824
:102030000800C01CADF8080099F86B0DBDF8081039
:1020400000EB4000884290D849E095F82A0200EB66
:10205000400101EB0010BDF8081006EB0010490824
:1020600000EB011000F5805090F8940D002102F073
:1020700049FBBDF80C20BDF8081011446054BDF8B0
:102080000C00401CADF80C0095F82A0200EB400152
:1020900001EB0010BDF8081006EB0010490800EB3A
:1020A000011000F5805090F8950D002102F02AFBF8
:1020B000BDF80C20BDF8081011446054BDF80C00A8
:1020C000401CADF80C00BDF80800801CADF80800FD
:1020D00099F86B0DBDF80810B1EB400FB5D395F82A
:1020E0002A0200EB400202EB001007EB001000F5A3
:1020F000805090F8800DBDF80C2000F00300A05433
:10210000BDF80C00401CADF80C0095F82A0200EB5D
:10211000400202EB001007EB001000F5805090F831
:10212000800DBDF80C20C0F38100A054BDF80C0058
:10213000401CADF80C0095F82A0200EB400202EBBF
:10214000001007EB001000F5805090F8800DBDF8EE
:102150000C10C0F301106054BDF80C00401CADF829
:102160000C0027E098F8EF03607598F8EE03A0756F
:1021700098F8ED03E07598F8EC03207698F8EB03F7
:10218000607698F8EA03A076BDF80C00801DADF8E3
:102190000C00002085F829020CE0BDF8080010446E
:1021A0004173BDF80800401CADF80800BDF80800F8
:1021B0000528F2D3BDF80C00C01F000AA073BDF8BB
:1021C0000C00C01FE07300200EE0BDF808002044A2
:1021D000007D5A460099F7F73DFABDF808102144F2
:1021E0000875BDF80800401CADF80800BDF80810DF
:1021F000BDF80C00C01F8142E7DBBDF80C00C01F1A
:1022000081B2E01DF7F714F8BDF80C20010AA154C3
:10221000BDF80C10491CADF80C10BDF80C10605442
:10222000BDF80C00401CADF80C00BDF80C00401FC0
:10223000000AE070BDF80C00401F2071BDF80C00D2
:10224000401F81B2601D07F0C6FFBDF80C1060543E
:10225000BDF80C00401CADF80C00169830B10128F8
:1022600014D0022821D0032841D12FE0BDF80C0062
:10227000E8B38021FA48F7F7A4FEBDF80C10F9483E
:10228000C0F8A410F7480121A0302EE0BDF80C00E2
:1022900068B30821F248F7F794FEBDF80C10F14836
:1022A0004167F048012170301FE0BDF80C00F0B12B
:1022B0004FF48071EC48F7F784FEBDF80C10E94844
:1022C000C0F8BC10E7480121B8300EE0BDF80C00A2
:1022D00068B14FF48061E248F7F773FEBDF80C1067
:1022E000E048C165DF4801215830F6F7F7FF98F85C
:1022F000E90300287ED02046FEE3059890F8950D6E
:10230000002102F0FFF98DF8100097F82C0295F8E3
:102310002812884202D1012085F82702009890F8FF
:10232000980B0099401C81F8980B97F8B2020007AF
:102330000ED5179800EB400101EB0011CB4800EBE4
:10234000011000F5805090F8692D4FF4E13103E061
:1023500099F8692DD9F8641D169802F013F95046C2
:10236000A222A6234FF0D50AC5287DD014DC4FF059
:10237000A501B5283FD008DC112876D0122875D0E9
:10238000132874D0B22873D114E1B62871D0B928BB
:1023900070D0C328F7D1ECE0D92819D006DCCA28C0
:1023A00069D0CE2868D0D528EDD106E0E12871D0DB
:1023B000E52870D0E728E6D12FE2F52006F83400B2
:1023C0009DF8100006EBC4056870AA70504609E03D
:1023D000F52006F834009DF8100006EBC40568707F
:1023E000AA70D920E8702846032102F0BCF82871B1
:1023F0000520D9E3FEE3F52006F834009DF810002F
:1024000006EBC405687099F8700D4FF0B509002807
:10241000D7F8340205D0B0F1104F33D34FF010404D
:1024200032E0B0F5100F02D34FF4100001E0D7F8FE
:1024300034020022CDE90002A97010460FE0BDF879
:102440000800C0F10200C200DDE90001F5F7EBFE73
:10245000BDF808102944C870BDF80800401CADF84C
:102460000800BDF8080008E020E1E1E1F8E108E239
:10247000FBE294E027E087E023E10328DFD35EE07E
:10248000A871DBE0D7F834020021CDE90001AB7080
:10249000084611E0D9E0B5E1BDF80800C0F103003D
:1024A000C200DDE90001F5F7BEFEBDF808102944C1
:1024B000C870BDF80800401CADF80800BDF8080061
:1024C0000428E9D353E0F52006F834009DF8100005
:1024D00006EBC405687099F8700D4FF0B909002833
:1024E000D7F834020AD0B0F1104F01D0D7F8340237
:1024F0000021CDE90001AB70084632E0B0F5100FC5
:1025000001D0D7F834020022CDE90002A9701046AC
:102510000FE0BDF80800C0F10200C200DDE90001D3
:10252000F5F781FEBDF808102944C870BDF8080011
:10253000401CADF80800BDF808000328E9D3484660
:102540009EE7BDF80800C0F10300C200DDE900010C
:10255000F5F769FEBDF808102944C870BDF80800F9
:10256000401CADF80800BDF808000428E9D348462F
:1025700094E0F52006F834009DF8100006EBC40541
:102580006870AA70C3202DE7F52006F834009DF886
:10259000100006EBC4056870AA70CA2022E7F52077
:1025A00006F834009DF8100006EBC4056870AA70A8
:1025B000B62017E7F52006F834009DF8100006EB6A
:1025C000C405687099F8700DB22210B1A97000208E
:1025D0002DE0A420A87000200EE0D7F86002BDF81E
:1025E0000810C1F10101C900C840BDF80810294414
:1025F000C870BDF80800401CADF80800BDF8080020
:102600000228EAD36A712846052101F0ACFF2BE2CB
:10261000D7F86002BDF80810C1F10201C900C84036
:10262000BDF808102944C870BDF80800401CADF87A
:102630000800BDF808000328EAD3AA71284606213D
:1026400001F091FFE8710820D3E6F52006F8340088
:102650009DF8100006EBC4056870AB70002016E012
:10266000000C02400060024000000240A412002062
:10267000D7F86402BDF80810C1F10301C900C840D1
:10268000BDF808102944C870BDF80800401CADF81A
:102690000800BDF808000428EAD3E120E8712846C4
:1026A000072101F060FF28720920A2E6F52006F854
:1026B00034009DF8100006EBC4056870AA70C520B0
:1026C00090E6F52006F834009DF8100006EBC405EE
:1026D000687099F8700D4FF0CE0928B1AE20A8703F
:1026E0000027ADF8087061E0AC20A8700027ADF8B5
:1026F000087017E00BF50051D1F84D320846D0F8BC
:102700005112BDF80800C0F10400C2001846F5F7E8
:102710008AFDBDF808102944C870BDF80800401CA7
:10272000ADF80800BDF808000528E3D3ADF808703F
:1027300017E00BF50051D1F855320846D0F8591280
:10274000BDF80800C0F10400C2001846F5F76BFDA3
:10275000BDF8081029440872BDF80800401CADF807
:102760000800BDF808000528E3D385F80D90284639
:102770000D2101F0F8FEA8730F203AE60BF5005189
:10278000D1F84D320846D0F85112BDF80800C0F11A
:102790000500C2001846F5F746FDBDF808102944AB
:1027A000C870BDF80800401CADF80800BDF808006E
:1027B0000628E3D3ADF8087017E00BF50051D1F807
:1027C00055320846D0F85912BDF80800C0F105008E
:1027D000C2001846F5F727FDBDF8081029444872D5
:1027E000BDF80800401CADF80800BDF80800062838
:1027F000E3D385F80F9028460F2101F0B4FE28742A
:102800001120F6E5F52006F834009DF8100006EBDF
:10281000C4056870AA70E520E4E5F52006F83400E8
:102820009DF8100006EBC4056870AA70E720D9E592
:10283000F52006F834009DF8100006EBC40568701A
:10284000AA701120E8702846032101F08CFE28713F
:102850000520ADF80C00012087F82C025046FDE35E
:10286000F52006F834009DF8100006EBC4056870EA
:10287000A9700120E870C220287100206871122020
:10288000FEE5F52006F834009DF8100006EBC405BF
:102890006870FF20A8704FF0000AADF808A0FE494C
:1028A00010E0BDF808201398104400F5805090F80F
:1028B000720DBDF808202A44D070BDF80800401CF5
:1028C000ADF80800BDF808000A28EAD3B9F87E0D73
:1028D0008B46000A6873B9F87E0DA873B7F8B0028A
:1028E000000AE873B7F8B0022874B7F8B012169867
:1028F00001EB802081B20320F6F7BAF8ADF808A00A
:102900004FF4007259460FE0BDF80800084400F586
:10291000805090F8E801BDF808302B445874BDF899
:102920000800401CADF80800BDF808009042EBD349
:10293000132085F81102284640F2112101F013FE00
:1029400085F8120240F2132053E5059B93F8953D5C
:102950008DF8103097F82C3295F828C2634502D1D3
:10296000012385F82732009B93F8983BDDF800C0DF
:102970005B1C8CF8983B9DF8103023B19DF810300B
:102980005B1E8DF810300A286FD2DFE800F0FE4B96
:102990006FA5FDFCFB055A8506F834109DF8101054
:1029A00006EBC40040318146417082703021C17015
:1029B000017197F830120909417140790A28484697
:1029C00004D24079303089F8050002E0417937318E
:1029D000417197F8300200F00F0189F8061099F85C
:1029E00006000A2899F80600494601D2303000E076
:1029F000373088710320C87109F101000721F6F70B
:102A000045FA89F808000920ADF80C0097F82C0267
:102A1000042802D1052087F82C02002085F827021F
:102A2000062036E006F834109DF8100006EBC405C9
:102A300040306870AA703120E87035200DE0072022
:102A4000D7E406F834109DF8100006EBC4054030BA
:102A50006870AA703220E8703020287103206871F5
:102A6000681C0521F6F712FAEEE314E0042306F8D9
:102A700034309DF8101006EBC40040314170827074
:102A80000521C170ADF80C3097F82C02022802D154
:102A9000032087F82C021CE106F834109DF8100082
:102AA00006EBC40540306870AA703120E87032200F
:102AB000287103206871681C0521F6F7E7F9A871F1
:102AC0000720ADF80C00059890F8960D20F0200135
:102AD000059880F8961DDEE706F834109DF8100082
:102AE00006EBC40540306870AA703121E9703020CF
:102AF0002871D7F8342200E0F5E3B2F5100F00D2C8
:102B00003220687197F83202012803D097F8320218
:102B100010B103E0A97101E03220A8710021ADF8E5
:102B2000081013E0D7F83402BDF80820C2F10502FE
:102B30009200D040BDF8082000F00F002A44303049
:102B4000D071BDF80800401CADF80800BDF80800C1
:102B50000628E7D332206873ADF8081018E0D7F8DC
:102B60006002BDF80810C1F103018900C840BDF83A
:102B7000081000F00F00294430308873BDF80800B9
:102B8000401C03E05FE059E00FE093E0ADF808007F
:102B9000BDF808000428E2D30320A874681C1221A1
:102BA000F6F774F9E8741420BCE206F834109DF8C6
:102BB000100006EBC40540306870AA703220E8703F
:102BC000312129716871A8710021ADF8081015E054
:102BD000D7F86002BDF80820C2F103029200D0408D
:102BE000BDF8082000F00F002A443030D071BDF845
:102BF000080000E0FBE3401CADF80800BDF8080049
:102C00000428E5D3ADF80810302008E0BDF808101E
:102C10002944C872BDF80810491CADF80810BDF869
:102C200008101929F2D3032085F82400681C2421F8
:102C3000F6F72CF985F82500262073E2102006F817
:102C40003400302003E0102006F83400312006EB79
:102C5000C4025070ADF80C103BE0059B93F8953D15
:102C60008DF8103097F82C3295F828C2634502D1C0
:102C7000012385F82732009B93F8983B009D5B1C4D
:102C800085F8983B9DF8103023B19DF810305B1EFD
:102C90008DF810300A2801E0A4120020DCD2DFE811
:102CA00000F009081945FD0706180528C9E6CAE716
:102CB000C4E7B7E6042206F834209DF8101006EBAE
:102CC000C40040314170512181700521C170ADF8BF
:102CD0000C200CE2042306F834309DF8101006EBAB
:102CE000C4004031417082700521C170ADF80C30D4
:102CF000FDE106F834109DF8100006EBC4054030E5
:102D00006870AA703120E870322028710320687141
:102D1000681C0521F6F7BAF8A871059890F8960D89
:102D200020F02001059880F8961D88E606F83410FA
:102D30009DF8100006EBC40540306870AA70312081
:102D4000E8702A71D7F83412B1F1104F09D032214E
:102D5000697197F83212012905D097F8320238B11B
:102D600002E03021F4E7A8710021ADF8081015E069
:102D70003220F8E7D7F83402BDF80820C2F1070284
:102D80009200D040BDF8082000F00F002A443030F7
:102D9000D071BDF80800401CADF80800BDF808006F
:102DA0000828E7D33220E873ADF8081013E0D7F80D
:102DB0006002BDF80820C2F105029200D040BDF8C3
:102DC000082000F00F002A4430301074BDF80800CD
:102DD000401CADF80800BDF808000628E7D33020F5
:102DE000A875ADF8081008E0BDF808202A44D07591
:102DF000BDF80820521CADF80820BDF80820062AAE
:102E0000F2D36877ADF8081008E0BDF808202A442E
:102E10009077BDF80820521CADF80820BDF80820B6
:102E2000062AF2D385F82400ADF8081009E0BDF8B1
:102E300008202A4482F82500BDF80820521CADF86D
:102E40000820BDF80820062AF1D385F82B00ADF83C
:102E5000081009E0BDF808202A4482F82C00BDF8CB
:102E60000820521CADF80820BDF80820062AF1D32E
:102E700085F8320007E0BDF80810294481F83300D6
:102E8000BDF80810491CADF80810BDF80810062957
:102E9000F1D3032085F83900681C00E006E03921F1
:102EA000F5F7F4FF85F83A003B203BE106F83410D3
:102EB0009DF8100006EBC40540306870AA703220FF
:102EC000E8703121297133216971A8710021ADF8B1
:102ED000081013E0D7F86002BDF80820C2F105021F
:102EE0009200D040BDF8082000F00F002A44303096
:102EF000D071BDF80800401CADF80800BDF808000E
:102F00000628E7D3ADF80810302108E0BDF8080026
:102F100028444173BDF80800401CADF80800BDF816
:102F200008001928F2D3032085F82600681C262102
:102F3000F5F7ACFF85F827002820F3E0059890F816
:102F4000950D8DF81000BDF8080000EB00100EEB99
:102F5000C00000F5005090F82C0295F82812884225
:102F600002D1012085F82702009890F8980B00996B
:102F7000401C81F8980B4FF0000B58460FE0BDF84D
:102F80000810139800EB011000F5805090F8950D93
:102F90009DF8101088420AD0BDF80800401CADF81A
:102FA000080099F86B0DBDF808108842E7D8BDF805
:102FB0000810139800EB011000F5805090F8941D54
:102FC0001798401A401C8DF828009DF8100020B179
:102FD0009DF81000401E8DF8100097F82D020F2864
:102FE00003D297F82D02401C00E0584687F82D02C6
:102FF000AAF1B1016520092979D2DFE801F0050CB9
:1030000058787879783244009DF81000503006F8EE
:103010003400202180E09DF81000503006F8340084
:1030200097F82D0206EBC40540F0300068700120CF
:10303000A870E87085F804B028460521F6F7E4FA90
:10304000CDE9000B68710098000AA8710320E871AF
:10305000FA2028720920ADF80C0000E0D2E2B1207D
:10306000D0E29DF81010503106F8341097F82D1268
:1030700006EBC40541F030016970A8700120E870CA
:103080009DF8280023E09DF81010503106F8341008
:1030900097F82D1206EBC40541F030016970A87055
:1030A0000120E8709DF8280040F010000FE09DF826
:1030B0001000503006F8340097F82D0206EBC405D6
:1030C00040F0300068700120A870E8700520287179
:1030D00028460521F6F798FACDE9000B68710098AB
:1030E000000AA8710320E871FA20FFF7DCBAAAE011
:1030F00097F82E02B12806D097F82E0287F83102F1
:10310000B12087F82E029DF81000503006F83400E8
:1031100097F82D0240F0C00106EBC4004170FA217F
:103120008170032058E2BDF808201598104441F63C
:10313000983210440278521C027099F8700D38B120
:10314000179A521CD2B2012837D002287BD145E011
:10315000BAF1310F03D0BAF1450FF7D116E00020D4
:10316000ADF8080006A90CE0BDF80800BDF808306D
:1031700006EBC402085CD054BDF80800401CADF852
:103180000800BDF808000728EED358E40020ADF889
:1031900008000BA90CE0BDF80800BDF8083006EBEC
:1031A000C402085CD054BDF80800401CADF808000B
:1031B000BDF808000728EED341E48DF810209DF8F3
:1031C000100006F8340006EBC405032068700027E1
:1031D000AF70E9702F71092068710EE08DF8102032
:1031E0009DF8100006F8340006EBC4050320687053
:1031F0000027AF70EF702F71697128460621F6F72E
:1032000017F8CDE90007000AE8710098A871FFF7E8
:103210001ABA0098FD4990F8980B009A401C82F861
:10322000980B059890F8950D8DF810005046BAF15E
:10323000F30F71D009DC05286FD0F1280BD0BAF15B
:10324000F20F8AD115E0DFE116E1F4287ED0BAF161
:10325000F60FF6D1E2E0F52006F834009DF81000F4
:1032600006EBC40568700027AF700520E870F120F8
:10327000F8E0F52006F834009DF8100006EBC405D0
:1032800068704FF0000985F80290F220287197F8D5
:10329000A202687197F8A20201281DD097F8A20235
:1032A000202870D00620ADF80C00BDF80C00E870A6
:1032B0002846BDF80C10F5F7BBFFCDE90009BDF8B5
:1032C0000C10000A6854BDF80C100098294448708E
:1032D000BDF80C00801C9DE32520ADF80C0049468C
:1032E000ADF8089011E0E9E3BDF808200BEB02000F
:1032F00000F5005090F87502BDF808202A4490713E
:10330000BDF80800401CADF80800BDF808000F2803
:10331000EAD3ADF8081012E050E0AFE0BDF80820A5
:103320000BEB020000F5005090F88702BDF8082072
:103330002A445075BDF80800401CADF80800BDF8DF
:1033400008000A28EAD397F89C0200E07DE0E877BD
:10335000ADF8081011E0BDF808100BEB010000F506
:10336000005090F89D02BDF80810294481F8200013
:10337000BDF80800401CADF80800BDF8080005289D
:10338000E9D392E7FFE70A20ADF80C0048460EE0CB
:10339000BDF808100BEB010000F5005090F89D02FD
:1033A000BDF8081029448871BDF80800401CADF82C
:1033B0000800BDF808000428EAD376E7F52006F8EF
:1033C00034009DF8100006EBC40568704FF000094A
:1033D000484685F80290F321297197F8A212697185
:1033E0000C21ADF80C1097F89C12A9710FE06BE35B
:1033F000BDF808100BEB010000F5005090F89D029D
:10340000BDF808102944C871BDF80800401CADF88B
:103410000800BDF808000528EAD346E70620ADF805
:103420000C00F52006F834009DF8100006EBC405EA
:1034300068700027AF70BDF80C00E870F6202871A6
:10344000059890F89C0D687179E0F52006F8340035
:103450009DF8100006EBC40568700027AF700520CA
:10346000E870F420287128460521F5F7E1FECDE942
:103470000007000A68710098A87156E440F2132012
:10348000ADF80C00F52006F834009DF8100006EBAE
:10349000C4056870BDF80C00000AA870BDF80C00E7
:1034A000E870052028714FF0000A50460EE0BDF884
:1034B00008201398104400F5805090F8720DBDF864
:1034C00008202A445071BDF80800401CADF80800DF
:1034D000BDF808000A28EAD3B9F87E0D8B46000A29
:1034E000E873B9F87E0D2874B7F8B002000A687462
:1034F000B7F8B002A874B7F8B012169801EB8020A4
:1035000081B20320F5F7B4FA5746ADF808A04FF49E
:10351000007259460FE0BDF80800084400F58050DD
:1035200090F8E801BDF808302B44D874BDF80800C5
:10353000401CADF80800BDF808009042EBD32846C7
:10354000BDF80C10F5F774FECDE90007B7E6059855
:1035500090F8950D4FF00009494601F0D3F88DF829
:10356000100097F82C0295F82812884202D1012009
:1035700085F82702009890F8980B0099401C81F874
:10358000980BBAF1070F15D00ADCDFF884B0BAF156
:10359000070F39D2DFE80AF0383EF2380E0EF1009C
:1035A000AAF1100008282FD2DFE800F004E92E2E3F
:1035B000042E0417FA2006F8340006EBC4056870E0
:1035C000A87085F803A09DF810002871E81C02215E
:1035D000F5F75CFC687106201CE2FA2006F834005E
:1035E00006EBC4056870A87085F803A09DF810006C
:1035F0002871E81C0221F5F749FC68710620ADF836
:103600000C00142087F8310206E20000A41200200A
:1036100000E1F505FA2006F8340006EBC4056870F1
:10362000A87085F803A09DF81000287197F8320261
:10363000012803D097F83202E8B333E1D7F8340217
:10364000B0F1104F05D34FF410000021CDE9000177
:1036500003E0D7F83402CDE9000948460FE0BDF891
:103660000800C0F10200C200DDE90001F4F7DBFD53
:10367000BDF8081029444871BDF80800401CADF899
:103680000800BDF808000328E9D30020CDE90000B8
:1036900048460FE0BDF80800C0F10300C200DDE9B4
:1036A0000001F4F7C0FDBDF8081029440872BDF808
:1036B0000800401C00E05BE0ADF80800BDF8080021
:1036C0000428E7D348460FE0BDF80800C0F1020027
:1036D000C200DDE90001F4F7A6FDBDF80810294499
:1036E0000873BDF80800401CADF80800BDF80800DC
:1036F0000328E9D3D7F86012CDE9001948460FE056
:10370000BDF80800C0F10200C200DDE90001F4F7D5
:103710008AFDBDF808102944C873BDF80800401C94
:10372000ADF80800BDF808000328E9D3D7F8601207
:103730004F46BBFBF1F0CDE90009ADF8089011E070
:10374000BDF80800C0F10300C200DDE90001F4F794
:103750006AFDBDF8081029448874BDF80800401CB3
:10376000ADF80800BDF808000428E9D3384698E011
:103770000020CDE90000484612E014E1B8E024E161
:10378000BDF80800C0F10200C200DDE90001F4F755
:103790004AFDBDF8081029444871BDF80800401CD6
:1037A000ADF80800BDF808000328E9D3D7F83402C3
:1037B000B0F1104F05D34FF410000021CDE9000106
:1037C00003E0D7F83402CDE9000948460FE0BDF820
:1037D0000800C0F10300C200DDE90001F4F723FD99
:1037E000BDF8081029440872BDF80800401CADF867
:1037F0000800BDF808000428E9D348460FE0BDF8EA
:103800000800C0F10200C200DDE90001F4F70BFD81
:10381000BDF8081029440873BDF80800401CADF835
:103820000800BDF808000328E9D3D7F86002CDE905
:103830000009ADF8089011E0BDF80800C0F10200E1
:10384000C200DDE90001F4F7EEFCBDF808102944E0
:10385000C873BDF80800401CADF80800BDF80800AA
:103860000328E9D3D7F860124846BBFBF1F1CDE954
:1038700000190FE0BDF80800C0F10300C200DDE947
:103880000001F4F7D0FCBDF8081029448874BDF895
:103890000800401CADF80800BDF808000428E9D372
:1038A0000120A8750598D0F8980DADF80890401C37
:1038B000CDE9000911E0BDF80800C0F10100C20027
:1038C000DDE90001F4F7AFFCBDF808102944C87524
:1038D000BDF80800401CADF80800BDF8080002283B
:1038E000E9D3E81C1621F5F7D1FA68761A2091E0A1
:1038F000FA2006F8340006EBC4056870A87085F855
:1039000003A09DF810002871D7F86002CDE90009E6
:10391000ADF8089011E0BDF80800C0F10200C20047
:10392000DDE90001F4F77FFCBDF808102944487177
:10393000BDF80800401CADF80800BDF808000328D9
:10394000E9D3D7F860024F46002100F02BFA024677
:103950000B4658460021F4F735FCCDE9000100F094
:10396000D1FECDE90001ADF8087011E0BDF8080006
:10397000C0F10300C200DDE90001F4F754FCBDF81A
:10398000081029440872BDF80800401CADF8080072
:10399000BDF808000428E9D3E81C0921F5F776FAF8
:1039A00028730D2036E0FA2006F8340006EBC40533
:1039B0006870A87085F803A09DF810002871552044
:1039C0006871E81C0321FFF74DB8FA2006F83400AF
:1039D00006EBC4056870A87085F803A09DF8100078
:1039E0002871AA2068714846ADF8089008E0BDF833
:1039F000081029448871BDF80810491CADF808105A
:103A0000BDF808100329F2D3E81C0621F5F73EFAA9
:103A100068720A20ADF80C00169830B1012814D055
:103A2000022821D0032843D12FE0BDF80C00E0B3D9
:103A30008021D648F6F7C5FABDF80C10D448C0F876
:103A4000A410D3480121A0302EE0BDF80C0060B3D3
:103A50000821CE48F6F7B5FABDF80C10CC484167FE
:103A6000CB48012170301FE0BDF80C00E8B14FF4E5
:103A70008071C848F6F7A5FABDF80C10C448C0F824
:103A8000BC10C3480121B8300EE0BDF80C0060B195
:103A90004FF48061BD48F6F794FABDF80C10BC48AD
:103AA000C165BB480121583000E001E0F5F716FC84
:103AB00098F8E903002807D006EBC4000023BDF8FE
:103AC0000C10169AF6F7A2FA19B0BDE8F08F00981C
:103AD00090F8980B0099401C81F8980BF4E7019836
:103AE00090F82C0B0006EFD4019890F82C0BAA4A02
:103AF000C0F3C301169842F2107700EB400902EBC5
:103B0000890505F58055062943D2DFE801F00368F1
:103B1000A5EC4323002088F8AF07ADF808009F4FBD
:103B20000AE0385CBDF8082006EBC4018854BDF8F3
:103B30000800401CADF808009848F4F7A4FBBDF855
:103B400008108842BDF80800EBD8ADF80C004FF41F
:103B50007A70A9E0002088F8AF07ADF808008F4D13
:103B60000B350AE0285CBDF8082006EBC401885438
:103B7000BDF80800401CADF8080088480B30F4F789
:103B800082FBBDF808108842BDF80800EAD8ADF8FD
:103B90000C008BE00020ADF80800DFF80082A8F1EF
:103BA00009080DE0BDF80810BDF8082018F801005C
:103BB00006EBC4018854BDF80800401CADF80800AD
:103BC00076480938F4F75FFBBDF808108842E9D859
:103BD000BDF80800ADF80C00C5F8707B66E0002069
:103BE00088F8AF07ADF80800DFF8B081A8F15108F8
:103BF0000DE0BDF80810BDF8082018F8010006EB2C
:103C0000C4018854BDF80800401CADF808006348A2
:103C10005138F4F738FBBDF808108842E9D81699F6
:103C200006EBC4003131C17209F13101817516987A
:103C30000328CDD15A49312201F5E16081F81E27D0
:103C40003021C1750D2101760A214176BDF80800A9
:103C5000401CADF80800BBE70020ADF808004F4F4E
:103C6000153F0AE0385CBDF8082006EBC401885413
:103C7000BDF80800401CADF8080048481538F4F7B6
:103C800002FBBDF808108842BDF80800EAD8ADF87C
:103C90000C00019890F82C0B019920F07800183056
:103CA00081F82C0B4FF4FA60C5F8700B1698C8B366
:103CB000012849D0022857D003287FF40FAFBDF860
:103CC0000C0000283FF40AAF4FF480612F48F6F74C
:103CD00078F9BDF80C102E48C1652D4801215830E7
:103CE000F5F7FCFAF0E60020ADF80800DFF8AC804C
:103CF000A8F137080DE0BDF80810BDF8082018F845
:103D0000010006EBC4018854BDF80800401CADF862
:103D1000080022483738F4F7B6FABDF80810884290
:103D2000E9D855E7FFE7BDF80C000028DAD080217C
:103D30001648F6F746F9BDF80C101548C0F8A4105F
:103D400013480121A030CBE7BDF80C000028C9D0F2
:103D500008210E48F6F735F9BDF80C100C484167FC
:103D60000B4801217030BBE7BDF80C000028B9D02A
:103D70004FF480710748F6F724F9BDF80C10044899
:103D8000C0F8BC1002480121B830A9E7000C02407D
:103D90000060024000000240A4120020D9ED01089A
:103DA000405B00202DE9F04700242DED048B804678
:103DB00089469FED1E9B25462646E2004046494621
:103DC000F4F731FAC7B22046F4F70CFC41EC110BC2
:103DD000B0EE490AF0EE690A09F002F9380907F075
:103DE0000F0100EB8000B0EE408AF0EE608A01EB3C
:103DF0004000F4F7F7FB53EC182BF4F701FB41EC10
:103E0000180B28463146F4F7FAFB53EC182BF4F75D
:103E100050FAF4F727FC641CE4B205460E46082C61
:103E2000CBD3BDEC048BBDE8F087000000000000A0
:103E30000000594070B50E4D40F2244421462846FA
:103E400008F087FD012812D1298828462A1D1188EB
:103E5000214608F01BFD0748012180F8391B064860
:103E6000D0F88C000549C0F57A70A1F84C0470BDFB
:103E700000440040A422002000600240A452002020
:103E800010B50B4C40F22441204608F062FD012899
:103E90000DD12088201D00880648012180F8451B8F
:103EA0000548406C0549C0F57A70A1F84E0410BD74
:103EB000004C0040A422002000600240A4520020D8
:103EC00010B50B4C40F22441204608F042FD012879
:103ED0000CD12088A0880748012180F8511B064892
:103EE00040690649C0F57A70A1F8500410BD000081
:103EF00000500040A422002000600240A452002094
:103F000010B50B4C40F22441204608F022FD012858
:103F10000DD12088201D00880648012180F85D1BF6
:103F20000548C06A0549C0F57A70A1F8520410BD71
:103F300000480040A422002000600240A45200205B
:103F400010B5124C10492046F5F7B2F90021204671
:103F5000F5F7C4F90E4C4021204608F0F3FC002888
:103F6000F9D080210B48F6F72EF8084C0A49183C86
:103F70002046F5F79DF901212046F5F7AFF90749ED
:103F80000120087110BD000000802020A0600240C8
:103F900000440040000C0240008800201200002075
:103FA00010B5124C10492046F5F782F90021204641
:103FB000F5F794F90E4C4021204608F0C3FC002888
:103FC000F9D008210B48F5F7FEFF084C0A49303CB0
:103FD0002046F5F76DF901212046F5F77FF90749ED
:103FE0000120087110BD0000208000207060024098
:103FF000004C0040000C0240008020101200002005
:1040000010B5124C10492046F5F752F90021204610
:10401000F5F764F90E4C4021204608F093FC002887
:10402000F9D04FF480710B48F5F7CDFF074C0A49E2
:10403000A83C2046F5F73CF901212046F5F74EF95A
:1040400006490120087110BD00800028B8600240B8
:1040500000500040000002402080001012000020AC
:1040600010B5124C10492046F5F722F900212046E0
:10407000F5F734F90E4C4021204608F063FC002887
:10408000F9D04FF480610B48F5F79DFF074C0A49C2
:10409000303C2046F5F70CF901212046F5F71EF9D2
:1040A00006490120087110BD0080001858600240C8
:1040B00000480040000C0240008800101200002060
:1040C0002DE9F047012190B0480505F093FE8648A0
:1040D000F5F70EF9402738010024CDE90540C50168
:1040E00007940894CDE9094546040C940D94DFF833
:1040F000FC917F480B94CDE90207CDE90069694640
:104100000E947948F5F79CF9012210217648F5F7CD
:1041100081F9DFF8D4A1AAF1180A5046F5F7E8F8BA
:104120004FF47A78CDE90348E811CDE905400794CA
:104130000894CDE909456F480B940C940D940096B2
:104140000E94CDE9019069465046F5F779F90121C1
:104150005046F5F7C3F8DFF890A1AAF1300A5046AF
:10416000F5F7C6F8E811CDE9054007940894CDE9C4
:1041700009450C940D94DFF8809160480B94CDE9CB
:104180000207CDE9006969460E945046F5F758F9E3
:10419000012210215046F5F73DF9DFF84CA1AAF1B4
:1041A000600A5046F5F7A4F8CDE90348E811CDE9D7
:1041B000054007940894CDE9094551480B940C94A7
:1041C0000D9400960E94CDE9019069465046F5F79E
:1041D00037F901215046F5F781F8DFF80CA10AF113
:1041E000180A5046F5F784F8E811CDE90540079420
:1041F0000894CDE909450C940D94DFF808914248E4
:104200000B94CDE90207CDE9006969460E9450464A
:10421000F5F716F9012210215046F5F7FBF8DFF803
:10422000C8A0AAF1900A5046F5F762F8CDE9034814
:10423000E811CDE9054007940894CDE909453348D4
:104240000B940C940D9400960E94CDE90190694660
:104250005046F5F7F5F801215046F5F73FF8DFF83D
:104260008890A9F148094846F5F742F80397E81104
:10427000CDE9054007940894CDE9094525480B94FC
:104280000C940D94224F00960E94CDE9017069466E
:104290004846F5F7D5F8012210214846F5F7BAF857
:1042A000DFF84490A9F178094846F5F721F8CDE9FF
:1042B0000348E811CDE9054007940894CDE9094584
:1042C00015480B940C940D9400960E94CDE9017052
:1042D00069464846F5F7B4F801214846F4F7FEFF71
:1042E00010B0BDE8F0870000A06002400444004028
:1042F000405B0020A0640020044C0040985D00203A
:104300008868002004500040F05F0020706C00209E
:104310000448004048620020587000202DE9FC410C
:104320000121084605F066FD0121042005F062FD2B
:104330000121082005F05EFD0121402005F05AFD15
:10434000DFF8FC80072205214046F5F723FE07220F
:1043500006214046F5F71EFE072208214046F5F7E4
:1043600019FE072209214046F5F714FE354F0822B1
:104370000A213846F5F70EFE08220B213846F5F7DC
:1043800009FE082202214046F5F704FE08220C210E
:104390003846F5F7FFFD02268DF8056000244FF43E
:1043A00059708DF80640012500908DF807508DF862
:1043B000046069464046F5F7B1FD8DF805604FF49D
:1043C000E0508DF8064000908DF807508DF804609D
:1043D00069463846F5F7A2FD4FF4916000908DF8DC
:1043E00006408DF8045069464046F5F797FD2802CF
:1043F00000908DF806408DF8045069461248F5F794
:104400008DFD8DF806404FF4F040104C00908DF873
:10441000045069462046F5F781FDA9032046F5F7CB
:10442000D0FD69032046F5F7CCFDA1142046F5F731
:10443000C8FDE1142046F5F7C4FDBDE8FC8100008D
:10444000000C024000080240000002400018024038
:1044500070B50024FFF762FFFFF732FE00F01EF890
:104460000C4800210170817041700121C1704FF42E
:104470007A718160084D042085F8360B04E02046EF
:1044800000F062F9641CE4B295F8360BA042F6D84D
:1044900070BD000034570020A4220020F8B5112080
:1044A0008DF8000002258DF8015001248DF802409E
:1044B0008DF80340684601F047F826208DF800008B
:1044C0008DF8014000268DF802608DF803406846A3
:1044D00001F03AF80E208DF800008DF801508DF8AB
:1044E00002408DF80340684601F02EF827208DF831
:1044F00000008DF801408DF802608DF80340684699
:1045000001F022F80F208DF800008DF801508DF891
:1045100002408DF80340684601F016F834208DF80B
:1045200000008DF801408DF802608DF80340684668
:1045300001F00AF82F208DF800008DF801508DF859
:1045400002408DF80340684600F0FEFF35208DF8EC
:1045500000008DF801408DF802608DF80340684638
:1045600000F0F2FFF8BD01B9102110F8012B10F88E
:10457000013B491E5A400904090CF8D102F07F00A2
:10458000704700002DE9FF5F14460F464FF4805638
:104590004FF480684FF4C0694FF00C0A40F2244B8E
:1045A000002580B1012830D0022851D0032871D1D4
:1045B0000121880405F042FC0097012C6DD0022CEB
:1045C00070D094B377E00121480405F037FC0097E0
:1045D000012C03D0022C06D054B10DE0ADF80460DC
:1045E000ADF8088008E0ADF80460ADF8089003E08D
:1045F000ADF80450ADF80850ADF80650ADF80C50C9
:10460000ADF80AA069463B4C5DE00121C80405F005
:1046100015FC0097012C03D0022C07D05CB10EE0F2
:10462000ADF80460ADF8088009E040E0ADF8046042
:10463000ADF8089003E0ADF80450ADF80850ADF8BF
:104640000650ADF80C50ADF80AA069462A4C3AE085
:104650000121080505F0F2FB0097012C03D0022C84
:1046600006D054B10DE0ADF80460ADF8088008E064
:10467000ADF80460ADF8089003E0ADF80450ADF873
:104680000850ADF80650ADF80C50ADF80AA06946D8
:104690001A4C18E02CE000E004E0ADF80460ADF83E
:1046A000088008E0ADF80460ADF8089003E0ADF8CC
:1046B0000450ADF80850124CADF80650ADF80C504F
:1046C000ADF80AA06946204608F07AF90121204693
:1046D00008F0DFF801225946204608F059F9102168
:1046E000204608F0D3F80122C021204608F0DBF86C
:1046F000BDE8FF9F00440040004C004000500040D7
:10470000004800402DE9FC410024CDE900446F46FB
:1047100064220023F3F756FD0E460546104619465F
:104720000A220023F3F74EFD010102F00F000818E2
:10473000385504F10104E4B228463146082CE7D389
:10474000DDE90001BDE8FC812DE9FC5FA64E4FF0DC
:1047500004098246002586F8369B00EB400101EBF8
:104760000A10A6F5805707EB0014019404F5805455
:1047700094F8710D012803D10021504600F03CF956
:1047800094F8711DBB46994A504602EB4A0707F55B
:104790008057022945D097F82C0B40F0800087F80D
:1047A0002C0B0AEB4A010BEB8107A7F5996707F57C
:1047B00000574FF0000887F8008087F8028087F8DC
:1047C000018087F803800521B96087F8308087F879
:1047D0003280012087F8310087F83300D4F86C0D5F
:1047E00000EB80004000B86394F8692DD4F8641D94
:1047F0005046A7F63837FFF7C5FE94F86A1D0AEB56
:104800000A127A4802EB0A2200EBC200009000F57F
:10481000005008291FD2DFE801F01E1012162618DA
:10482000242600224FF4E131FFF7ACFE97F82C0B61
:1048300040F0800087F82C0BB5E0052100E00F2147
:1048400080F8281207E00721FAE7D4F86C1D6422EB
:104850005143C7F8701B9BF81810D946012904D0A2
:1048600019E00321ECE74946EAE780F828820120B5
:10487000C7F8400B5E4F80213846F5F7A4FB0821AE
:104880003846F5F7A0FBB9155A48F5F79CFB3915E2
:104890003846F5F798FB4FF0A10ECB467EE0009826
:1048A00005EB051200EBC20000F50B7000F500509F
:1048B0000021017381734173C173D4F86C2D94F896
:1048C0006B7D7A4302EB820292004261019A02EB15
:1048D000051202F5805292F8967D27F0800782F843
:1048E000967D017094F86A1DA0F50B70082953D2CB
:1048F000DFE801F0520408080A0C0E44E52180F8B4
:10490000311249E07146FAE7B121F8E73121F6E7C3
:10491000F12180F8311200212BE001EB011303EBB0
:1049200001230BEBC30701EB410303EB01130BEB7B
:104930000313002003F5805915E003EB001C0CF570
:10494000805C9CF894CD92F89C8DC44509D192F876
:1049500094CD00EB001807EBC80808F5005888F85C
:10496000A3C2401CC0B299F86BCD8445E5D8491C60
:10497000C9B296F8360B8842CFD80DE0062180F8F0
:10498000311205EB0A1101EB8102C2EB811159448E
:10499000D1F86910C0F860126D1CEDB294F86B0D7F
:1049A000A8423FF67CAF002086F8370B5A4600EB52
:1049B000400101EB001102EB011101F5805191F86A
:1049C0006A3D052B09D291F86A3D33B196F8373B21
:1049D00091F86B1D194486F8371B401CC0B204289F
:1049E000E5D3BDE8FC9F0000A4220020A412002013
:1049F000000C0240000002402DE9F04105466648E7
:104A00004FF480425310066864488414C71439B1C7
:104A1000C5B1012D18D0022D18D0032D1BD117E0E0
:104A200035B1012D06D0022D06D0032D13D105E09E
:104A3000114604E0194602E0214600E03946F5F748
:104A4000C2FA08E0114604E0194602E0214600E0FF
:104A50003946F5F7B6FA642009F008FC00224FF455
:104A600016512846FFF78EFD4D4905EB450201EB37
:104A7000820000F58050002380F86A3BC0F86C3B50
:104A800005EB450000EB051001EB001101F580512D
:104A9000D1F86C4D4348C0F89844012480F8914403
:104AA000414805EB850738447724847091F86A7D86
:104AB0009721082F08D2DFE807F0070406063537EC
:104AC0000704847000E08170C5EB0511374F01EBDE
:104AD0008101C02407F8314007EBC104637008214D
:104AE000A170310EE17006F0F0011144217180785F
:104AF00060712020A07106F00F00C5EBC5010844CD
:104B0000E071802020724C2060725420A0722848EE
:104B1000284F0B2655B1012D11D0022D27D0032D82
:104B200016D12FE06F21CEE76721CCE78021F5F782
:104B300048FAC7F8A4601F480121A03006E0082108
:104B4000F5F73FFA7E671B4801217030F4F7C6FB8A
:104B5000194890F8E90328B1204600232A460B2182
:104B6000F5F754FABDE8F041642009F07FBB4FF43B
:104B700080711248F5F725FAC7F8BC600D4801218D
:104B8000B830E3E74FF48061F5F71BFAFE6509489A
:104B900001215830DAE70000187AFF1F00180240A0
:104BA000A4120020A452002040740020405B00208A
:104BB000000C024000600240A422002000000240DD
:104BC0002DE9F0438FB000278DF830708DF83470E8
:104BD0008DF83870CDE90077CDE902778DF818703F
:104BE0008DF81C708DF820708DF82470ADF8287049
:104BF0009FED950A954C0B978DED0B0A94F84A0D95
:104C0000934D4FF0010808B384F84A7DB4F8620D63
:104C1000904E3168C1F57A71884217D13068C0F57D
:104C20007A70A4F8600DA6F1040900214846F4F753
:104C300055FB89494846F4F73BFB85F800804FF463
:104C40007A70306001214846F4F748FB2878012843
:104C50007ED12F7094F8EA0C804D00EB400005EBFC
:104C6000001000F5805090F8E20B794EB61C042835
:104C700004D0052802D0062804D106E084F8568D19
:104C8000C4F8587D8DF83070D6E0B4F8601D701C03
:104C9000891FF4F7E3FAC117CDE90201B4F8601DEA
:104CA0006B48C01E0844042105F088FBDDE902239F
:104CB000C117CDE90001504059400843DED1634897
:104CC000801D80F83C7D3079ADF82800BDF82800C3
:104CD0003128D3D1B4F8600D4121183890FBF1F0A0
:104CE000C117CDE9000184F88C058DF8307091E092
:104CF0009DF8300000EB80103044017D9DF83000BD
:104D0000284400F5805080F88D159DF8300008216A
:104D100000EB801030441A3005F01CFB8DED0B0ABF
:104D200010EE100A9DF8301005EB011101F58051CD
:104D3000C1F89D059DF83000082100EB801030443B
:104D4000323005F007FB8DED0B0A10EE100A00E083
:104D500076E09DF8301005EB011101F58051C1F8A6
:104D600099059DF83000082100EB801030443A305E
:104D700005F0F0FA8DED0B0A10EE100A9DF83010D8
:104D800005EB011101F58051C1F8A1059DF8300036
:104D9000082100EB80103044423005F0DBFA8DED45
:104DA0000B0A10EE100A9DF8301005EB011101F509
:104DB0008051C1F8A5059DF8180000EB400101EBFA
:104DC00000109DF8301005EB001000EB011041F6CB
:104DD00096510844017841F080010170B4F8601DDB
:104DE0001B48401C095C9DF8180000EB001202EB08
:104DF000002005EBC0029DF8200000EB001002EB44
:104E0000C00000F5005080F868129DF83000401C8A
:104E10008DF830009DF83010DDE90023891A77EB1A
:104E20000300FFF665AF29E79DF8300037549DF881
:104E30003000401C8DF830009DF830001428F3D36A
:104E40000FB0BDE8F083000000000000A4220020A5
:104E5000CE0A00202C64024000880010A41200201A
:104E60002DE9F34FDCA185B0D1E90021CDE9012185
:104E7000DBA10026D1E90021CDE90321DA4A35463C
:104E80003746B146B2465670D84B191801F58051D5
:104E900091F83C2D042A1ED1052281F83C2D524662
:104EA00081F8EEAC91F8CC4C24F0800481F8CC4C25
:104EB000042804D0052808D006280CD101E0CC49EC
:104EC00005E0CB493122891C01E0C949491C01F5A3
:104ED000005181F8F32C00EB4001C44800EB0110B5
:104EE00000F58050804690F8E22BC248DFF808B306
:104EF000C24C4FF48071042A24D0052A7ED0062AA1
:104F00007DD10546F5F75FF84FF400712846F5F7B7
:104F10005AF898F8E11BD8F8DC0B00F0CFFA94F8B7
:104F20003C0D401C84F83C0D0698312868D045287B
:104F300065D103A958468A5D8255761CB6B2072E04
:104F4000F9D331E194F8EC2C002A58D0F5F739F870
:104F5000A64E98F8E11BD8F8DC0B00F0AFFA94F8F5
:104F6000EC0C012802D0022841D11BE094F8EB1C84
:104F700001EB8100C0EB8110304490F860909B4AB7
:104F800050F8617F02F64173C2F8217F4768C2F88A
:104F9000257F8268C6F8292F026A1A60808C988063
:104FA0000F0924E096F8209F1DE007EB470101EB75
:104FB000071106EB0112002002F5805109E002EB17
:104FC000001303F5805393F894CDCC4505D0401CD5
:104FD00080B291F86B3D8342F1D891F86B1D81420C
:104FE00005D87F1CBFB294F8360BB842DDD84846CE
:104FF0000021FFF787FB02460B4602E0E0E0C8E035
:10500000CAE006210020CDF800A004F049FE07EB1D
:10501000470000EB071006EB001707F5EC57387850
:10502000C0F381000090D6F8252F002307211846F1
:1050300006F6277604F034FE387800F0030000907E
:1050400056F8062C00230821184604F029FE38786B
:10505000C0F301100090D6F8022000230921184661
:1050600004F01EFE322004F8C70F30206070F17F7C
:1050700000EB1111A170F17F01F00F013031E170EF
:105080002D222271B17F00EB11116171B17F01F00E
:105090000F013031A171E271717F00EB11112172AA
:1050A000717F01F00F0130316172317F00EB11111E
:1050B000E172317F01F00F01303121733A216173C8
:1050C000F27E00EB1212A273F27E02F00F02303277
:1050D000E2732174B17E00EB11106074B07E00F0B9
:1050E0000F003030A074306A0021C73CA6F6277646
:1050F000FFF708FB02460B460C210020CDF800A06C
:1051000004F0CEFD0020202240F28A215F463A546E
:10511000401C80B28842FAD34FF00A0C87F800C0D6
:1051200087F801C00021002006EB4112131893F804
:105130005B3F202B03D1401C80B22028F6D31F28D0
:105140000DD20020131893F85B3F00EB451807F8C9
:105150000830401C80B22028F4D36D1CADB2491C2D
:1051600089B21429DFD30BEB451080F820C080F8FA
:1051700021C080F822C080F823C080F824C080F8C5
:1051800025C0252000EB45100004000C84F8ECAC91
:105190000BD107B0BDE8F08F01A958468A5D825552
:1051A000761CB6B2072EF9D30720154908601448BB
:1051B0000121001FF4F792F80B4981F801A0E8E7FC
:1051C00094F83C0D401C84F83C0D98F8E11BD8F88D
:1051D000DC0B00F073F9DCE701693230313030006C
:1051E0000169323045303000CE0A0020A412002080
:1051F000A802002000080240B80E0020A4220020CF
:10520000A464024070B50D4C40F224452946204666
:1052100007F09FFB002810D02946204607F036FBF8
:105220002088201D00880648012180F8491D054975
:105230000968C1F57A71A0F8621D70BD00140140C3
:10524000A42200202C64024010B5124C10492046C4
:10525000F4F72EF800212046F4F740F80E4C4021D8
:10526000204607F06FFB0028F9D04FF400710B487F
:10527000F4F7A7FE074C0A49783C2046F4F718F8E3
:1052800001212046F4F72AF806490120487010BD94
:1052900000802020A0640240001401400008024069
:1052A00000880010CE0A00202DE9F04301218FB0C4
:1052B000880504F09FFDDFF894904846F4F718F84D
:1052C0004020050103900024CDE90545C60207945E
:1052D0000894CDE909464FF020681E480B940C94C1
:1052E0000D941B4FCDF800800E94CDE901706946F6
:1052F0004846F4F7A5F8012210214846F4F78AF849
:10530000DFF84890A9F178094846F3F7F1FF4FF428
:105310007A70CDE90340CDE9054507940894CDE9BD
:1053200009460D480B940C940D94CDF800800E9412
:10533000CDE9017069464846F4F782F801214846F4
:10534000F3F7CCFF0FB0BDE8F0830000A06402408B
:1053500004140140B80E0020D00A00207CB50121C1
:10536000042004F047FD184E082206213046F4F7C9
:1053700011FE082207213046F4F70CFE02218DF8B9
:10538000051000258DF806500124C0208DF8074037
:1053900000908DF8041069463046F4F7BFFD4FF4D5
:1053A000407000908DF804408DF8065003208DF871
:1053B00005008DF8074069463046F4F7AFFD6102FD
:1053C0003046F4F7FEFD7CBD000802402DE9F041B7
:1053D0000024FFF7C3FF00214FF4E13000F06EF826
:1053E000FFF762FF00F04CF823480023037083703E
:1053F0004370C37002218160037383730126467377
:10540000C6734FF47A7141611C4A04EB440102EB0C
:10541000810000F5E850037083704670C67002EB9F
:10542000011505F58055D5F8E41B01EB8101490014
:10543000816095F8E21BA0F55060042904D005298D
:1054400002D0062912D105E0101900F5805080F82D
:10545000F33C0BE03121171907F5805787F8F31C4F
:10546000D5F8E41B64256943C0F8081D641CE4B248
:10547000052CCAD3BDE8F081EC2F0020A412002037
:1054800038B545208DF8000002208DF80100012478
:105490008DF802408DF80340684600F055F847202B
:1054A0008DF800008DF8014000208DF802008DF885
:1054B0000340684600F048F838BD00007FB50C4650
:1054C00005460121202004F0D1FC00204FF480513A
:1054D0000095012C03D0022C06D064B10FE0ADF88A
:1054E00004104FF4806103E0ADF804104FF4C06184
:1054F000ADF8081003E0ADF80400ADF80800ADF811
:105500000400ADF80600ADF80C000C200D4CADF811
:105510000A006946204607F053FA0121204607F0A9
:10552000B8F9012240F22441204607F031FA102157
:10553000204607F0ABF90122C021204607F0B3F95D
:105540007FBD00000014014030B50F23C278017800
:105550000125FAB1144A126801F1E02102F4E06277
:10556000C2F5E062C2F30722C2F10404D3404278DC
:10557000A24084781C401443220181F80024007862
:1055800000F01F018D404009800000F1E020C0F8CC
:10559000005130BD01F01F0085404809800000F136
:1055A000E020C0F8805130BD0CED00E0024A11400F
:1055B000014302480160704780FFFF1F08ED00E0D3
:1055C00010B50021074B0A46002003EBC004401C25
:1055D000C0B262548028F8D3491CC9B20829F3D359
:1055E00010BD0000437E00202DE9FE4F0026171A53
:1055F0008146701E3546A3EB010A8846002F02DD66
:105600004FF0010102E003D14FF00001019102E0EF
:10561000C7F100070190BAF1000F02DD4FF0010061
:1056200002E003D14FF00000009002E0C7F1000A51
:1056300000905046574501DD3C4600E00446601CA2
:105640004FF0000B029016E008F0FF0109F0FF0098
:105650000C9A00F015F83E445544A64202DD01992B
:10566000361B8944A54202DD00992D1B88440BF1AD
:1056700001001FFA80FB02998B45E5DBBDE8FE8F38
:1056800030B5CC0801F0070301259D40EBB2064D73
:1056900005EBC005C808285C0AB1184302E063EABC
:1056A0000000C043285530BD437E00202DE9FC4159
:1056B00001210A2004F09EFB01248DF804400026FD
:1056C0004FF4C0508DF80660032700908DF80570E8
:1056D0008DF8074069464648F4F720FC8DF80440F1
:1056E0008DF806608DF80570A5028DF80740414CD5
:1056F000009569462046F4F711FCC82008F0B6FD75
:1057000029462046F4F75DFCC82008F0AFFD294685
:105710002046F4F758FCC82008F0A8FD0021FD2021
:1057200000F054FA0021122000F050FA0021AE20BF
:1057300000F04CFA0021D52000F048FA0021A0200A
:1057400000F044FA0021A82000F040FA00213F2098
:1057500000F03CFA0021D32000F038FA002108467E
:1057600000F034FA0021402000F030FA0021A0209F
:1057700000F02CFA0021C02000F028FA0021DA20E5
:1057800000F024FA0021122000F020FA00218120EC
:1057900000F01CFA00217F2000F018FA0021D92027
:1057A00000F014FA0021822000F010FA0021DB2022
:1057B00000F00CFA0021342000F008FA0021A420A7
:1057C00000F004FA0021A62000F000FA00212020B9
:1057D00000F0FCF90021084600F0F8F9FFF7F0FEB0
:1057E0000021AF2000F0F2F900F054F8BDE8FC8190
:1057F000000C0240000402400346012000E0584330
:10580000491EC9B2FBD270472DE9F84F82460A986B
:105810000D4650436421B0FBF1F0984600F0FF0BB9
:105820004FF001090AEB02072B4600245046FAB25A
:105830001946CDF80090FFF7D7FE05EB0806F3B246
:10584000FAB2F1B25046CDF80090FFF7CDFE5246C5
:10585000F3B229461046CDF80090FFF7C5FEF3B22B
:10586000FAB2F8B22946CDF80090FFF7BDFE4F46D8
:105870000AEB0B0609E02819C3B2C1B2F2B25046D6
:105880000097FFF7B1FE641CE4B24445F3D3BDE8D2
:10589000F88F000070B50025B020294600F096F979
:1058A0000021084600F092F90021102000F08EF946
:1058B000084E002406EBC4000121405D00F086F98B
:1058C000641CE4B2802CF5D36D1CEDB2082DF0D32E
:1058D00070BD0000437E002070B50B4C05460221D0
:1058E000204604F051FC0028F9D02946204604F057
:1058F00054FC0121204604F047FC0028F9D0204642
:1059000004F049FCC0B270BD003800402DE9FC4FE6
:105910001D46884681468B460090082B0ED06807AE
:1059200000D0012000EBD500690810FB01F0C0B2E7
:10593000203A02F0FF0A0026019046E00620F7E731
:10594000082D10D00C2D14D0102D16D0182D3FD1AD
:1059500021490AEBCA0001EB80000027845DE007C3
:105960000FD00B9A10E01D490AEB4A0001EB4000F2
:10597000F3E70AEB4A001A49EDE71A4901EB0A106E
:10598000EBE70B9830B3002241464846FFF778FE1C
:105990007F1C640808F10100FFB200F0FF08082F27
:1059A000DDD309F1010000F0FF09082D0AD00099AC
:1059B000A9EB0100B0EB550F04D10BF108008946AB
:1059C00000F0FF0B761CD846F6B201988642B7D39A
:1059D000BDE8FC8F0122D7E7F400020868F4010853
:1059E00090F6010804FB01082DE9FF4F81B04FF04C
:1059F0000005DDE90F7ADDF838B05FEA030980467B
:105A00002E4612D10398F2F7EDFD41EC100B07F092
:105A10004FFA9FED331B51EC100B53EC112BF2F7A7
:105A200048FCF2F700FE00F0FF09082F00D1022524
:105A3000D94510D8BBF1000F0DD03B463022CDF830
:105A400000A040460299FFF761FF05EB570101EB0B
:105A5000080000F0FF08002431E0A9EB0B01A1428F
:105A60000DD105EB570101FB0480C0B23B462E224D
:105A7000CDF800A00299FFF749FF01261DE0001BA9
:105A8000401EC1B20A20FFF7B7FE0399CDF800A06F
:105A9000B1FBF0F00A21B0FBF1F201FB120106EBC1
:105AA0000800A1B105EB570202FB04003031C0B27F
:105AB000CAB23B460299FFF729FF641CE4B209EB26
:105AC0000600A042C9D805B04846BDE8F08F05EBF6
:105AD000570101FB0400C0B23B463022EAE7000058
:105AE000000000000000F03F2DE9FF4F81B00646A6
:105AF00000900F464FF0000A8946580700D0012059
:105B000000EBD3000490002032E0002029E00E9842
:105B1000002410F80A500AF101001FFA80FAE80781
:105B200001D00F9A02E00F9848B300223946304660
:105B3000FFF7A6FD7F1C641C6D08E4B2FFB2082CC1
:105B4000EDD3761C0098F6B2311A0398814204D145
:105B500009F10800009E00F0FF0908F101004F461E
:105B6000C0B2039980468842D1D30BF10100C0B284
:105B7000049983468842C8D305B0BDE8F08F01225E
:105B8000D4E72DE9F8431D46DDE908781646894635
:105B900004460EE03B4649462046CDF80080FFF71C
:105BA000B5FE082F0ED004EB5700C4B26D1EEDB247
:105BB000761C002D04D03278202A01D37E2AE9D920
:105BC000BDE8F883A41DE4B2F0E700002DE9F04140
:105BD000114C06464FF4006500292946204602D0A4
:105BE000F4F7F1F901E0F4F7ECF94FF48057394696
:105BF0002046F4F7E6F939460848F4F7E4F9304668
:105C0000FFF76AFE39462046F4F7DDF929462046BB
:105C1000BDE8F041F4F7D7B9000C0240000402409F
:105C20002DE9F04F4FF0000A89B05446D146ADF847
:105C300000A0ADF804A0ADF808A0ADF80CA0ADF838
:105C400010A0ADF814A0FF4D564695F8EA06A5F54C
:105C5000805B01060BF58040069002F1718002F036
:105C600075B895F8AE07022805D195F8AD0710B1C3
:105C70000720ADF81400DFF8D083BDF8141018F831
:105C80000100FA285AD1BDF8140001194046014418
:105C9000497885F8F513BDF814102144014489783A
:105CA00085F8F413BDF8141021440144C97885F82F
:105CB000F313BDF8141021440144097985F8F21357
:105CC000BDF8141021440144497985F8F113BDF859
:105CD0001410214401EB0800807985F8F00395F851
:105CE000F00395F8EA13884208D995F8F0030021EB
:105CF000FEF758F8064695F8EA0307E095F8EA0338
:105D00000021FEF74FF8064695F8F0030021FEF754
:105D100049F8301AC0B205280FD395F8F00354287B
:105D20000BD295F8F003062807D9C848D0F806101A
:105D3000016041898180F3F733FC0624BDF814002B
:105D40004746204438448079BDF814102144394432
:105D5000C97840EA0160BDF814102144394409793A
:105D6000BDF81420090422443A44527941EA022140
:105D70000843B7494A68904251D04860BDF81400C2
:105D8000204438448078BDF81410214439444978BF
:105D900040EA0126B5F87216BDF814003044801CA4
:105DA00081423CD3B5F87206BDF814103144401A54
:105DB000801EA5F87206BDF8140031463844F3F78A
:105DC00037FABDF81410314439444978BDF814202D
:105DD0003244BA5C41EA0221814241F0888795F859
:105DE000E90340B1B01C81B2BDF81400012338446E
:105DF0000422F4F70BF9BDF814002044384400796C
:105E000000F001000890BDF8140020443844807967
:105E10000023C0F34200A6F10708079013E0A5F89D
:105E2000729609B0BDE8F08F18443844C079DDE9B6
:105E30000721F3F7FFFBBDF814102144194439443E
:105E4000C8715B1C9BB2BDF8140043452044EBDBDA
:105E50003844C079012185F8AC174946C5F8B09699
:105E600085F8AE96069A82F88694C2F8889495F8DA
:105E7000AE27032A03D095F8AE27012A03D1754B2C
:105E80000122C3F888228946ADF80C1012287CD074
:105E90000CDCA0F10B00072818D2DFE810F0220B71
:105EA000900BCF0BC90B020E24009E0CA2286ED0C3
:105EB00008DC142801F01F86152801F07086A1283F
:105EC00004D140E3A3287CD0A4287BD000204946FD
:105ED000BDF8142022440244B954401C80B2052865
:105EE000F6D301F0FFBEC8464046FDE1BDF8000014
:105EF00000EB400101EB00100BEB001000F58050AF
:105F0000594690F86A0D08287ED2DFE800F07D043B
:105F10000404047DB40440468CE0BDF81400BDF8D0
:105F20000C20204410443844007A78B3012802D071
:105F3000022877D113E0BDF80000BDF8041000EB93
:105F4000400202EB00100BEB001000EB011041F6D9
:105F500096510844017821F00401017062E0BDF817
:105F6000000000EB400202EB0010BDF8042001EB42
:105F7000001000EB021041F696521044027822F015
:105F800008020270BDF8000002E0EFE34AE0EEE331
:105F900000EB400303EB0010BDF804100BEB001006
:105FA00000EB011000F58050C0F8988DBDF800108E
:105FB0000220F3F7D3FB0020DC464246BDF8001078
:105FC00001E0F9E3F9E301EB011303EB01210CEB31
:105FD000C103BDF8041001EB011103EBC101014441
:105FE00001F5005181F86B22401C80B21428E5D3E2
:105FF0000020BDF8001001EB011303EB01210CEBB5
:10600000C103BDF8041000E06BE101EB011103EBEB
:10601000C101014401F5005181F88722401C80B282
:106020000A28E6D3BDF80C00401CADF80C00BDF802
:106030000400401CADF80400BDF8000000EB400176
:106040000AE00000A4220020547400208E260020C4
:10605000180200200000404201EB00100BEB001082
:1060600000F58050594690F86B0DBDF80420904221
:106070003FF653AF35E1ADF8048021E1BDF81400DF
:10608000BDF80C20204410443844007A042805D080
:1060900005DC58B1012846D002287DD12EE1082820
:1060A0007BD010287AD0202876D1E7E1BDF8000017
:1060B00000EB001202EB002001EBC002BDF804006F
:1060C00000EB001002EBC00000F5005090F8A202B7
:1060D000102824D1BDF8000000EB001202EB0020D4
:1060E00001EBC002BDF8040000EB001002EBC000A1
:1060F00000F5005080F8A282BDF80000F32200EB0A
:10610000001303EB002001EBC003BDF8040000EB1B
:10611000001003EBC00000F5005080F83122BDF8FC
:106120000C00401CC5E0BDF80000F22200EB00139B
:1061300003EB002001EBC003BDF8040000EB0010EE
:1061400003EBC00000F5005080F83122BDF80000DC
:1061500000EB400202EB0010BDF8042001EB001040
:1061600000EB021041F696521044027822F004022D
:106170000270BDF81400BDF80C20204410443844CF
:10618000027ABDF8000000EB001303EB002001EBE6
:10619000C003BDF8040002E08DE0AFE0EFE000EBEB
:1061A000001003EBC00000F5005080F8A222002090
:1061B000BDF81420BDF80C3022441A4402443A447D
:1061C000537ABDF8002002EB021C0CEB022201EB1B
:1061D000C20CBDF8042002EB02120CEBC202024416
:1061E00002F5005282F87532401C80B20F28DFD3CE
:1061F0000020BDF81420BDF80C3022441A4402449B
:106200003A44137EBDF8002002EB021C0CEB022284
:1062100001EBC20CBDF8042002EB02120CEBC2022F
:10622000024402F5005282F88732401C80B20A28EC
:10623000DFD3BDF81400BDF80C20204410443844CE
:1062400090F82200BDF8002002EB021303EB0222BB
:1062500001EBC203BDF8042002EB021203EBC20201
:1062600002F5005282F89C020020BDF81420BDF80F
:106270000C3022441A4402443A4492F82330BDF8C8
:10628000002002EB021C0CEB022201EBC20CBDF859
:10629000042002EB02120CEBC202024402F500528F
:1062A00082F89D32401C80B20528DED3BDF80C0078
:1062B0002030ADF80C00BDF80400401CADF804001F
:1062C000BDF8000000EB400202EB001001EB0010F3
:1062D00000F5805090F86B0DBDF8042090423FF619
:1062E000CDAEBDF80000401CADF8000095F8360BAF
:1062F000BDF8001088423FF6F9ADF2E5BDF80000A8
:10630000F22200EB001303EB002001EBC003BDF809
:10631000040000EB001003EBC00000F5005080F813
:106320003122BDF8000000EB400202EB0010BDF886
:10633000042001EB001000EB021041F696521044CD
:10634000027822F004020270BDF81400BDF80C209F
:10635000204410443844027ABDF8000000EB0013DA
:1063600003EB002001EBC003BDF8040000EB0010BC
:1063700003EBC00000F5005080F8A222CFE6BDF884
:106380000000F32200EB001303EB002001EBC0033D
:10639000BDF8040000EB001003EBC00000F5005056
:1063A00080F83122BDF8000000EB400202EB001043
:1063B000BDF8042001EB001000EB021041F69652EC
:1063C0001044027822F004020270BDF81400BDF8F7
:1063D0000C20204410443844027ABDF8000000EB41
:1063E000001303EB002001EBC003BDF8040000EB39
:1063F000001003EBC00000F5005080F8A222BDF8A9
:106400001400BDF80C20204410443844427ABDF8F2
:10641000000000EB001303EB002001EBC003BDF80C
:10642000040000EB001003EBC00000F5005080F802
:106430009C220020BDF81420BDF80C3022441A44E0
:1064400002443A44937ABDF8002002EB021C0CEBA4
:10645000022201EBC20CBDF8042002EB02120CEB8D
:10646000C202024402F5005282F89D32401C80B202
:106470000528DFD3BDF80C00C01D1AE7BDF80000E9
:10648000F22200EB001303EB002001EBC003BDF888
:10649000040000EB001003EBC00000F5005080F892
:1064A0003122BDF8000000EB400202EB0010BDF805
:1064B000042001EB001000EB021041F6965210444C
:1064C000027822F004020270BDF81400BDF80C201E
:1064D000204410443844027ABDF8000000EB001359
:1064E00003EB002001EBC003BDF8040000EB00103B
:1064F00003EBC00000F5005080F8A2220020BDF898
:106500001420BDF80C3022441A4402443A44537A11
:10651000BDF8002002EB021C0CEB022201EBC20CC6
:10652000BDF8042002EB02120CEBC202024402F599
:10653000005282F89D32401C80B20428DFD3BDF89F
:106540000C00401DB5E6B01E0D2190FBF1F0C0B26D
:10655000079048461BE24846F3E1BDF80000BDF84D
:10656000041000EB400202EB0012D8460BEB0210C5
:1065700000EB011000F5805090F8960D80077DD457
:10658000BDF814000AEB8A02011902EBCA000844A4
:106590003844007A0021FDF705FCBDF80020BDF865
:1065A00004C002EB420303EB0213424608EB031361
:1065B00003EB0C1303F5805393F8943D89EA010C27
:1065C000434053EA0C0359D1BDF8000000EB001121
:1065D00001EB002002EBC001BDF8040000EB00104D
:1065E00001EBC00000F5005090F8690201287CD151
:1065F000BDF8140020443844417ABDF8000000EB97
:10660000001303EB0023BDF8040008EBC30200EB0A
:10661000001002EBC00000F5005080F83212BDF807
:10662000140020443844407BBDF814102144394400
:10663000897A40EA0161BDF8140020443844C07AE8
:10664000BDF81420000422443A44127B40EA0220A0
:106650000143BDF8000000EB001202EB0022BDF880
:10666000040008EBC20200EB001002EBC00000F5D2
:106670000050C0F83412BDF8140000E05EE1204480
:106680003844007DBDF8141021443944497C40EA67
:106690000161BDF8140020443844807CBDF814200A
:1066A000000422443A44D27C40EA02200143BDF86F
:1066B000000000EB400202EB001208EB0210BDF8F4
:1066C000042000EB021000F58050C0F8981DBDF8C2
:1066D00000100220F3F742F8BDF8000000EB400183
:1066E00001EB001108EB011000E07FE0BDF80410A1
:1066F00000EB011000F5805090F8941DBDF80000EB
:1067000000EB001202EB002208EBC20000F5005083
:1067100080F82512BDF8000000EB400101EB0011EC
:1067200008EB011000F5805090F86A0D012806D0A2
:1067300002285ED003285CD0072857D1CBE0BDF8F3
:10674000000000EB001101EB002008EBC002BDF8D7
:106750000400414600EB001002EBC00000F50050C1
:1067600090F8320220B1012840D140E0FDE331E24F
:10677000BDF8000000EB400202EB001001EB00103E
:1067800000F5805090F8700D0028BDF8000000EB77
:10679000001202EB002001EBC002BDF8040000EB88
:1067A000001002EBC00000F50050D0F8340205D014
:1067B000B0F1104F05D106E02AE3F2E0B0F5100F7A
:1067C00001D0B52200E0C322BDF8000000EB0013A9
:1067D00003EB002008EBC001BDF8040000EB001043
:1067E00001EBC00000F5005080F831229FE0B92293
:1067F000EAE7BDF8000000EB001101EB002008EB18
:10680000C002BDF80400414600EB001002EBC000DE
:1068100000F5005090F82C22BDF8000000EB0013AA
:1068200003EB002008EBC00000F5005090F82802B0
:1068300082427CD1BDF8140020443844807BBDF8EE
:106840001420000422443A44D27B40EA0222BDF8DC
:10685000140020443844007C0243BDF8000000EBE3
:10686000001303EB002001EBC003BDF8040000EBB4
:10687000001003EBC00000F50050C0F86022BDF826
:10688000140020443844427ABDF8000000EB0013A5
:1068900003EB002001EBC003BDF8040000EB001087
:1068A00003EBC00000F5005080F83222BDF8000074
:1068B000A42200EB001303EB002001EBC003BDF8A2
:1068C000040000EB001003EBC00000F5005080F85E
:1068D0002E22A32278E7BDF8000000EB400101EB77
:1068E000001008EB001000F5805090F8700D0028A3
:1068F000BDF8000000EB001202EB002008EBC00224
:10690000BDF8040000EB001002EBC00000F50050E1
:10691000D0F8340204D0B0F1104F06D003E006E006
:10692000B0F5100F01D001224EE705224CE70AF125
:106930000100079900F0FF0A8A4515D2BDF804004E
:10694000401CADF80400BDF8000000EB400101EB75
:1069500000100BEB001000F5805090F86B0DBDF8A7
:10696000042090423FF6F9ADBDF8000000EB400175
:1069700001EB00110BEB011000F5805090F86B0D4E
:10698000BDF8041088427CD8BDF80000401CADF86A
:10699000000095F8360BBDF8001088423FF6DBADDD
:1069A000ABE4484648E0ADF80490D84621E0BDF895
:1069B000140020443844007A0021FDF7F3F9BDF8B3
:1069C000002002EB420303EB021308EB0312BDF8B5
:1069D000043002EB031202F5805292F8942D89EAFA
:1069E000010342401A4330D0BDF80400401CADF80A
:1069F0000400BDF8000000EB400101EB001108EBC2
:106A0000011000F5805090F86B0DBDF8041088421D
:106A1000CDD8BDF8000000EB400101EB001108EB00
:106A2000011000F5805090F86B0DBDF804108842FD
:106A3000B6D8BDF80000401CADF8000095F8360B44
:106A4000BDF800108842AED857E4BDF80000BDF88C
:106A5000042000EB400101EB0010414608EB001060
:106A600000EB021000F5805090F8942DBDF8000066
:106A700000EB001303EB002008EBC00000F5005012
:106A800000E06DE180F82522BDF8000000EB400237
:106A900002EB001008EB001000F5805090F86A0D32
:106AA000012806D0022806D0032839D00728B0D103
:106AB0007CE0CA227BE0BDF8000000EB001202EB94
:106AC000002001EBC002BDF8040000EB001002EB57
:106AD000C00000F5005090F82C22BDF8000000EB3B
:106AE000001303EB002001EBC00000F5005090F80C
:106AF000280282428DD1BDF80000AA2200EB0013CB
:106B000003EB002001EBC003BDF8040000EB001014
:106B100003EBC00000F5005080F82E22A32246E0CF
:106B2000BDF8000000EB001202EB002001EBC002F8
:106B3000BDF8040000EB001002EBC00000F50050AF
:106B400090F82C22BDF8000000EB001303EB0020AE
:106B500001EBC00000F5005090F82802824225D1D8
:106B6000BDF80000AA2200EB001303EB002001EBAC
:106B7000C003BDF8040000EB001003EBC00000F5FB
:106B8000005080F82E22BDF80000A32200EB001375
:106B900003EB002001EBC003BDF8040000EB001084
:106BA00003EBC00000F5005080F831220422BDF84C
:106BB000000000EB001303EB002008EBC001BDF860
:106BC000040000EB001001EBC00000F5005080F85D
:106BD00031221EE7484648E0ADF80490D84621E04F
:106BE000BDF8140020443844007A0021FDF7DAF89B
:106BF000BDF8002002EB420303EB021308EB031283
:106C0000BDF8043002EB031202F5805292F8942D85
:106C100089EA010342401A4330D0BDF80400401C09
:106C2000ADF80400BDF8000000EB400101EB0011DD
:106C300008EB011000F5805090F86B0DBDF80410C2
:106C40008842CDD8BDF8000000EB400101EB0011F7
:106C500008EB011000F5805090F86B0DBDF80410A2
:106C600088427DD8BDF80000401CADF8000095F8C2
:106C7000360BBDF800108842AED891E6BDF8000092
:106C8000BDF8042000EB400101EB0010414608EB89
:106C9000001000EB021000F5805090F8942DBDF824
:106CA000000000EB001303EB002008EBC00000F530
:106CB000005080F82522BDF8000000EB001202EB26
:106CC000002008EBC002BDF8040000EB001002EB4E
:106CD000C00000F5005090F82C22BDF8000000EB39
:106CE000001303EB002001EBC00000F5005090F80A
:106CF00028028242A6D1BDF8140020443844407ACC
:106D0000BDF81420000422443A44927A40EA022258
:106D1000BDF8140020443844C07A0243BDF8000096
:106D200000EB001303EB002001EBC003BDF80400EF
:106D300000EB001003EBC00000F50050C0F860222B
:106D4000BDF8000000EB400202EB001001EB001068
:106D500000F5805090F86A0D0828BFF473AF00E08A
:106D6000BEE3DFE800F0040519192E04044169E7C9
:106D7000BDF80000B22200EB001303EB002008EB8B
:106D8000C001BDF8040000EB001001EBC00000F5ED
:106D9000005080F82E2255E7BDF80000A52200EB38
:106DA000001303EB002001EBC003BDF8040000EB6F
:106DB000001003EBC00000F5005080F82E22A32243
:106DC00013E0BDF80000B52200EB001303EB002038
:106DD00001EBC003BDF8040000EB001003EBC000A2
:106DE00000F5005080F831220222BDF8000000EBCF
:106DF000001303EB002008EBC001BDF8040000EB1A
:106E0000001001EBC00000F5005080F8312219E7B6
:106E1000BDF8140020443844007A05287DD2BDF81E
:106E2000140020443844007A002876D0BDF81400BD
:106E300020443844007A401EADF800000020494646
:106E4000BDF8002002EB420303EB02120BEB02122F
:106E500002EB001202F5805282F8941DBDF800206A
:106E600002EB420C0CEB02120BEB021202EB0012D3
:106E700002F5805282F8951DBDF8002002EB420C0D
:106E80000CEB02120BEB021202EB001202F5805225
:106E900082F89C1D401C80B21028D1D3BDF814008C
:106EA00020443844807B89460021FCF77BFF08435F
:106EB0007DD0BDF8140020443844407ABDF8141049
:106EC000000421443944897A40EA0120BDF81410B5
:106ED00021443944C97A0843C117FCF763FFBDF860
:106EE0000010D84601EB410202EB01120BEB02113C
:106EF00001F58051C1F8640DBDF8140020443844F8
:106F0000007B0021FCF74EFFBDF8001001EB4102B1
:106F100002EB011208EB021100E0FAE101F58051E9
:106F200081F8680DBDF8140020443844407B0021EE
:106F3000FCF738FFBDF8001001EB410202EB011233
:106F400008EB021101F5805181F8690DBDF81400BC
:106F500020443844807B0021FCF724FFBDF800105A
:106F600001EB410202EB011200E0FDE308EB02112C
:106F700001F5805181F86A0DBDF8140020443844B1
:106F8000C07B0021FCF70EFFBDF8001001EB4102B1
:106F900002EB011208EB021101F5805181F86B0D33
:106FA000BDF8140020443844007C002100E0F1E0EA
:106FB000FCF7F8FEBDF8001001EB410202EB0112F4
:106FC00008EB021101F58051C1F86C0DBDF81400F9
:106FD00020443844407C0021FCF7E4FEBDF800105A
:106FE00001EB410202EB011208EB021101F58051A5
:106FF00081F8700DBDF8000000EB400101EB0011BD
:1070000008EB011000F5805090F86A0D06284846FC
:107010005DD0ACE0BDF81400BDF804102044084475
:107020003844807C0021FCF7BDFEBDF8042003211C
:10703000B2FBF1F2BDF8001001EB410303EB0113C9
:1070400008EB031101EB021101F5805181F8940D59
:10705000BDF81400BDF80410204408443844C07C36
:107060000021FCF79FFEBDF804200321B2FBF1F2E2
:10707000BDF8001001EB410303EB011308EB031112
:1070800001EB021101F5805181F8950DBDF8140056
:10709000BDF80410204408443844007D0021FCF76A
:1070A00081FEBDF804200321B2FBF1F2BDF800100F
:1070B00001EB410303EB011308EB031101EB021198
:1070C00001F5805181F89C0DBDF80400C01CADF89D
:1070D0000400BDF8000000EB400101EB001108EBDB
:1070E000011000F5805090F86B0DBDF8041000EB16
:1070F000400088428ED84DE0BDF81400BDF8041061
:10710000204408443844807C0021FCF74BFEBDF845
:10711000001001EB410202EB011208EB0211BDF875
:107120000420520801EB021101F5805181F8940D01
:10713000BDF81400BDF80410204408443844C07C55
:107140000021FCF72FFEBDF8001001EB410202EB1D
:10715000011208EB0211BDF80420520801EB0211E4
:1071600001F5805181F8950DBDF80400801CADF843
:107170000400BDF8000000EB400101EB001108EB3A
:10718000011000F5805090F86B0DBDF80410B1EBC4
:10719000400FB1D3BDF80400123086427ED9BDF84D
:1071A000000000EB400101EB00100BEB001000F5BC
:1071B0008050594690F86A0D012837D0BDF800007C
:1071C00000EB400202EB001001EB001000F58050D4
:1071D00090F86A0D032829D0BDF8000000EB4002AA
:1071E00002EB001001EB001000F5805090F86A0DE2
:1071F00002281BD0BDF8000000EB400202EB00109B
:1072000001EB001000F5805090F86A0D07280DD0B2
:10721000BDF8000000EB400202EB001001EB001093
:1072200000F5805090F86A0D04285CD1BDF8140078
:107230003044384410F8020C00F00F00042813D238
:10724000BDF8000000EB400202EB0010BDF8142076
:1072500001EB001032443A4412F8023C00F5EC50C5
:10726000027863F301020270BDF814003044384420
:1072700010F8012C0420B0EB121F16D9BDF8000045
:1072800000EB400202EB0010BDF8142001EB0010EF
:1072900032443A4412F8012C130900E023E000F5CF
:1072A000EC50027863F383020270BDF8140030449E
:1072B000384410F8010C00F00F00042813D2BDF878
:1072C0000000BDF8141000EB400202EB00100BEBC5
:1072D00000103144394411F8012C00F5EC500178CC
:1072E00062F305110170BDF800100220F2F736FAC2
:1072F000BDF80000C0B2FDF727FABDF8000001217B
:1073000000EB40020BEB820000F5805080F8B916CC
:10731000CBE0BDF8140020443844007A05287CD125
:10732000BDF8140020440930ADF80C00BDF80C0085
:10733000385C85F8D80BBDF80C00401CADF80C008B
:10734000ADF80090D846A3E0BDF80C00385C0021F1
:10735000FCF728FDBDF8001001EB410208EB02111B
:1073600001F5805181F8E30BBDF80C00401CADF82D
:107370000C00BDF80C00385C0021FCF713FDBDF8D3
:10738000001001EB410208EB021101F5805181F878
:10739000E20BBDF80C00401CADF80C00BDF80C0071
:1073A000385CBDF80C1000043944497840EA0120EB
:1073B000BDF80C10394489780843C117FCF7F2FC7A
:1073C000BDF8001001EB410208EB021101F58051FC
:1073D000C1F8DC0BBDF80C00C01CADF80C00BDF80A
:1073E0000C00385C0021FCF7DDFCBDF8001001EB5F
:1073F000410208EB021101F5805181F8E00BBDF864
:107400000C00401CADF80C00BDF80C00385C0021ED
:10741000FCF7C8FCBDF8001000E046E001EB4102BB
:1074200008EB021101F5805181F8E10BBDF80C0069
:10743000401CADF80C00BDF80C00385C0021FCF7D6
:10744000B1FCBDF8001001EB410208EB021101F59F
:107450008051C1F8E40BBDF80C00401CADF80C00E5
:10746000BDF80C0038444078BDF80C10795C40EA57
:107470000120BDF80C10891CADF80C10BDF80C10E3
:107480000844ADF80C00BDF80000401CADF8000049
:1074900095F8D80BBDF8001088423FF655AF002193
:1074A0000A20F2F75BF9FDF791FFBDF8000000EB51
:1074B000400101EB00100BEB001000F5805090F83C
:1074C000710D02280CD1BDF80000A32200EB0013BF
:1074D00003EB00200BEBC00000F5005080F82922E0
:1074E000DEE2BDF8140020443844007A85F8EF034A
:1074F000BDF8140020443844407A85F8EE03BDF806
:10750000140020443844807A85F8ED03BDF8140057
:1075100020443844C07A85F8EC03BDF814002044B8
:107520003844007B85F8EB03BDF814002044384450
:10753000407B85F8EA0305F2EA35F2F731F8F1F716
:10754000F3FF2878A5F2EA35FF282FD1F1F7A2FF43
:10755000BDF8140020443844007A85F8EF03BDF8E4
:10756000140020443844407A85F8EE03BDF8140036
:1075700020443844807A85F8ED03BDF81400204497
:107580003844C07A85F8EC03BDF814002044384430
:10759000007B85F8EB03BDF8140020443844407BA1
:1075A00085F8EA03F1F7FCFFF1F7BEFFDBF85800BE
:1075B00008B10F2000E00E2085F8B00792E31020FC
:1075C00085F8B007BDF8140020443844007A85F8E7
:1075D000EF03BDF8140020443844407A85F8EE03E8
:1075E000BDF8140020443844807A85F8ED03BDF8D6
:1075F000140020443844C07A85F8EC03BDF8140028
:1076000020443844007B85F8EB03BDF81400204487
:107610003844407B85F8EA0305F57B75F1F7C0FF38
:1076200002F092FCE860E868E868A5F57B7559E32C
:107630000E2085F8B00785F8E19153E34A46ADF88E
:10764000009059463EE0ADF8042016E0BDF8000079
:1076500000EB400303EB0010BDF8043001EB001019
:1076600000EB031000F5805090F8960DC00714D180
:10767000BDF80400401CADF80400BDF8000000EBAC
:10768000400303EB001001EB001000F5805090F870
:107690006B0DBDF804309842D8D8BDF8000000EB5F
:1076A000400303EB001001EB001000F5805090F850
:1076B0006B0DBDF80430984208D8BDF80000401C9E
:1076C000ADF80000BDF800000428BCD3BDF80000F0
:1076D000042878D390461046FE4A5070FE4B012095
:1076E000C3F88802C3F8880295F8E701E8B30D20D3
:1076F00085F8B007BDF8140020443844407ABDF83E
:10770000143023443B441B7A40EA0320ADF80800C0
:10771000BDF8140020443844C07ABDF81430234426
:107720003B449B7A40EA0320508000204FF4007CC9
:10773000BDF814102144014439440B7B0BEB0001CC
:1077400001F5805181F8E831401C80B26045EFD3EB
:10775000E048408800F2FF3081B20120F1F7F4F9EF
:1077600018B185F8E18101E040E029E0D94841887D
:1077700064225143BDF80820B1FBF2F185F8E01115
:1077800001218BF808104188491C41804088BDF8D0
:107790000810884214D995F8DC0140F0010085F802
:1077A000DC0195F8DC0120F00600801C85F8DC0186
:1077B000BDF80800A5F8DE0100210120F1F7CEFF99
:1077C000404668E1FFE7102085F8B00795F8DC0136
:1077D00040F0800085F8DC0184E2BDF8140020440C
:1077E0003844007A85F8E1011120E5E64946ADF814
:1077F0000090DC463EE0ADF8041016E0BDF8000055
:1078000000EB400202EB0010BDF804200CEB00106E
:1078100000EB021000F5805090F8960DC00714D1CF
:10782000BDF80400401CADF80400BDF8000000EBFA
:10783000400202EB00100CEB001000F5805090F8B5
:107840006B0DBDF804209042D8D8BDF8000000EBC5
:10785000400202EB00100CEB001000F5805090F895
:107860006B0DBDF80420904208D8BDF80000401C04
:10787000ADF80000BDF800000428BCD3BDF800003E
:107880000428A9D3DFF84C82894688F80110924970
:107890000120C1F88802C1F8880295F8E701E0B339
:1078A000BDF8140020443844007A042835D812204A
:1078B00085F8B007BDF8140020443844007A85F8F4
:1078C000E10195F8E101401EADF800000020BDF88F
:1078D00014102144014439444A7ABDF8001001EBE8
:1078E000410303EB01110CEB0111014401F580513F
:1078F00081F8722D401C80B20A28E8D3BDF814002C
:1079000020443844007DBDF8141021443944C97C1A
:1079100040EA0120ADF8080000E06BE0BDF814007B
:1079200020443844807DBDF8141021443944497DF9
:1079300040EA0120A8F8020000204FF40072BDF8D0
:107940001410214401443944CB7D0BEB000101F5B7
:10795000805181F8E831401C80B29042EFD3B8F8F2
:107960000200BDF8001000EB8120401E81B2032010
:10797000F1F7EAF8F0B3B8F8021040466422514338
:10798000BDF80820B1FBF2F185F8E01101215A465B
:107990008BF80810B8F80210491CA8F80210B8F8C3
:1079A0000210BDF80830994245D9002041F69D5398
:1079B000BDF8001001EB410C0CEB011102EB0111C1
:1079C00001EB0011194491F800C04CF0010C81F852
:1079D00000C0401C80B21028EAD3BDF8000000EBC4
:1079E000400101EB001002EB001041F67C5108440D
:1079F000037800E04EE043F001030370BDF800009F
:107A000000EB400303EB001002EB00100844017888
:107A100021F00601891C0170BDF80810BDF80000B6
:107A200000EB400303EB00100BEB001000F580505F
:107A3000A0F87E1D29E0408801282BD1002041F6C6
:107A40009D53BDF8001001EB410C0CEB011102EB52
:107A5000011101EB0011194491F800C02CF0010C48
:107A600081F800C0401C80B21028EAD3BDF80000A5
:107A700000EB400101EB00100BEB001041F67C51D4
:107A80000844017821F001010170BDF800100220C6
:107A9000F1F764FE48461049C1F88802C1F888022F
:107AA00020E1DBF858000A21B0FBF1F0BDF814101A
:107AB00021443944097A88421CD1BDF8140020447D
:107AC0003844007A50B1DBF858100A39CBF8581016
:107AD00009E000001802002000004242CBF8589054
:107AE000102085F8B00700210520F1F737FE0120AE
:107AF0008BF80800F6E000212022DC4600200CEB89
:107B0000411303EB000888F85B2F401C80B220284B
:107B1000F7D3491C89B21429F0D3142085F8B00793
:107B2000BDF8141021443944097AADF80810BDF8A5
:107B3000141021443944497AADF81010BDF80810EA
:107B4000142901D9ADF80800BDF81000202801D98A
:107B5000ADF81020002119E000200CEB41180FE0D7
:107B6000BDF81420BDF8103001FB032223181A447D
:107B70003A44927A08EB000383F85B2F401C80B2F2
:107B8000BDF810209042EBD3491C89B2BDF8080023
:107B90008142E1D300210720F1F7E0FDA2E01520AA
:107BA00085F8B007BDF8140020443844017A5846DF
:107BB0008BF8201FBDF8141021443944097BBDF80F
:107BC000142022443A44527A41EA0261BDF814205A
:107BD00022443A44927ABDF81430120423443B44C0
:107BE000DB7A42EA03221143C0F8251FBDF81410C6
:107BF00021443944097CBDF8142022443A44527B84
:107C000041EA0261BDF8142022443A44927BBDF857
:107C10001430120423443B44DB7B42EA0322114329
:107C2000C0F8211FBDF8141021443944497CBDF827
:107C30001420090422443A44927C41EA0221BDF80E
:107C4000142022443A44D27C1143C0F8291FBDF8C5
:107C5000141021443944097D80F8461FBDF81410E2
:107C600021443944497D80F8451FBDF81410214452
:107C70003944897D80F8441FBDF8141021443944EB
:107C8000C97D80F8431FBDF8141021443944097E92
:107C900080F8421FBDF8141021443944497E80F811
:107CA000411F202E1BD9BDF8141021443944497FAF
:107CB000BDF8142022443A44927E41EA0261BDF8A4
:107CC000142022443A44D27EBDF8143012042344D6
:107CD0003B441B7F42EA03221143C0F8471F0220A6
:107CE00085F8EC0CB5F8720650B300201BE00020BC
:107CF0004946BDF8142022440244B954401C80B2C5
:107D00000528F6D3A5F8721609B0BDE8F08FBDF8C6
:107D100014103144014439448978BDF814200244D8
:107D2000B954401C80B2B5F872168142EFD8B5F84C
:107D30007206494602E03954401C80B22828FAD322
:107D4000B5F8720600287DF48CAFDDE795F8AE0734
:107D50004FF47A7430B101287DD002287CD00328FA
:107D60007BD12DE295F8EA06C0F3C3000E2874D249
:107D7000DFE800F0EE0713ED1F2B2B374D7A9FAB9A
:107D8000ECEFF8A1F84806F011FC002865D095F852
:107D9000EA0620F078001030E5E0F4A1F24806F0A1
:107DA00005FC0028F2D095F8EA0620F0780018309B
:107DB000D9E0EFA1EC4806F0F9FB0028E6D095F8F1
:107DC000EA0620F078002830CDE0E9A1E64806F088
:107DD000EDFB0028DAD095F8EA0620F0780038307C
:107DE000C1E0E3A1E04806F0E1FB0028CED09BF81B
:107DF0000100182805D995F8EA0620F078005030DF
:107E0000B1E095F8EA0620F078004030ABE0D9A167
:107E1000D54806F0CBFB0028B8D05A464B469119FE
:107E200001F5805181F83337761CB6B2142EF6D3A3
:107E3000CD4C0021431823441E79531803F5805379
:107E400083F83867491C89B20F29F3D30021032036
:107E5000F1F784FC02E08EE040E175E095F8EA0677
:107E600020F07800483019E2C4A1BF4806F09EFB1C
:107E700000288BD05A464946931903F5805383F85E
:107E8000EC16761CB6B2142EF6D3B74C002143186C
:107E900023445E79531803F5805383F8F166491C37
:107EA00089B20F29F3D395F8EA0620F07800503014
:107EB000F4E1AFA1AC4806F079FB00288AD095F830
:107EC000EA0620F0780058304DE095F8B20758B136
:107ED00095F8EA0620F07800603085F8EA06C5F8E3
:107EE0008896012085F88606A6A19F4806F05EFBCD
:107EF000002829D0C5F88896012185F886169A4C65
:107F00002044417900793039303841EA0010C117F6
:107F1000FBF748FF85F8B2079CA1204606F046FB18
:107F2000002811D021184A78302A06D34978205CDD
:107F30003038303941EA001001E0205C3038C11798
:107F4000FBF730FF85F8B307B9E102E0A9E14DE1A5
:107F500046E187A1844806F029FB00280AD095F85D
:107F6000EA0620F0780085F8EA06C5F88896012030
:107F700085F88606A3E195F8EA06C0F3C3000D284C
:107F80004CD2DFE800F0081825303B66078890EDFA
:107F90004B96A10035E776A1734806F007FBE8B3DE
:107FA000C5F88896012085F8860695F8EA0620F03F
:107FB0007800083072E176A19DE0C5F8889601202E
:107FC00085F8860695F8EA0620F07800103065E11D
:107FD00067A1654806F0EAFA00B3C5F88896012063
:107FE00085F88606B6E06BA15F4806F0DFFAA8B117
:107FF00095F8EA0620F078002030B4E75FA15A48EF
:1080000006F0D4FA50B15A464B46911901F5805109
:1080100081F8EC36761CB6B2142E00E042E0F4D3C0
:10802000514E0021441834446779541804F58054A3
:1080300084F8F176491C89B20F29F3D3C5F8883644
:10804000012085F8860695F8EA0620F078002830A9
:1080500024E14CA1444806F0A9FA18B395F8B217E8
:1080600031B195F8EA1621F07801303185F8EA1639
:10807000C5F88896012185F886163B490844417960
:1080800000793039303841EA0010C117FBF78AFE19
:1080900085F8B20713E136A1334806F087FA0028C5
:1080A0007FF478AF0BE195F8EA0620F078004830CD
:1080B00059E72FA12C4806F079FA10B395F8EA0693
:1080C00020F0780060304EE729A1274806F06EFACC
:1080D000B8B195F8EA0620F07800DFE095F8EA06F6
:1080E000C0F3C30005280CD2DFE800F003040CDB6A
:1080F000580055E71EA11C4806F058FA00287FF4E6
:108100005CAFDCE0C5F88896012085F88606164C41
:10811000A07961793038303940EA0110C117FBF796
:1081200041FE85F8B20719A1204606F03FFA88B152
:1081300021184A78302A06D34978205C3038303903
:1081400041EA001001E0205C3038C117FBF72AFE3D
:1081500085F8B30795F8EA0620F0780018309DE01E
:10816000A5E0000061000000547400206F6B000067
:108170004F4B0000494D45493A00000049434349EF
:10818000443A00004353513A000000002C00000024
:1081900022000000524541445900000095F8EA06CB
:1081A00020F0800085F8EA0695F8EA0620F07800CD
:1081B00085F8EA06069981F88694C1F888947EE0ED
:1081C00095F8EA06C0F3C300092878D2DFE800F08A
:1081D0000807060E051145566900EAE5DDE5D0E51C
:1081E00095F8EA0620F078000830BCE6AFF280018E
:1081F000FAE638A1394806F0D9F968B34F46C5F810
:1082000088964FF0010885F88686344A5C468119C5
:1082100011440B79A11901F5805181F8B437761C0E
:10822000B6B2142EF3D32CA12D4806F0BFF950B1ED
:1082300000210A18224402F5805282F8B377491CC3
:1082400089B20229F5D395F8EA0620F0780030309B
:1082500085F8EA0684F8088031E0AFF2EC011F48A7
:1082600006F0A4F958B3C5F88896012085F886066B
:1082700095F8EA0620F0780038300FE0AFF21011E0
:10828000164806F093F9D0B1C5F88896012085F814
:10829000860695F8EA0620F07800403085F8EA0670
:1082A0000DE0AFF234110D4806F080F938B195F8C1
:1082B000EA0640F0800085F8EA06C5F88C46494693
:1082C000A5F87296054A00201154401C80B264281B
:1082D000FAD319E5444843502C00000054740020A0
:1082E000582A00202DE9F74F86B0002001908146E2
:1082F0000090FF4D00212954401C80B26428F8D31F
:10830000FC4890F88614A0F5405431B394F8AD17AA
:1083100019B3002180F8861494F8EA0620F0800052
:1083200084F8EA0694F8AE0728B101280ED0022896
:1083300006D0032811D194F8EA0620F078000AE06C
:1083400094F8EA0620F07800203004E094F8EA0679
:1083500020F07800583084F8EA0694F8EA06DFF84E
:1083600098B300067ED594F8AE0601287BD194F828
:10837000AC07012877D10020E04F804600EB400198
:1083800001EB081007EB0010039000F58050002669
:10839000029061E0039800EB061505F5805595F80D
:1083A000960D000655D595F8960D40F0040085F819
:1083B000960D95F8960D00074BD595F8960D20F083
:1083C000080085F8960D0020C7F8390008EB081161
:1083D00001EB082007EBC00006EB061100EBC10A19
:1083E000C64842F24D2151441022293005F69455D9
:1083F000EFF72BFF0AF5085050F8451FC7F81D107E
:108400004068C7F821002878387742F2602050F899
:108410000A00C7F82500BA480168C7F83D108088EF
:10842000A7F841006868C7F84300B86D81B2022020
:10843000F0F78AFB00210620F1F790F9B86D798BEF
:10844000884202D2B86D401CB86500210520F1F7C2
:1084500085F9761C0298B6B290F86B0DB04299D8A7
:10846000414601E0FEE31AE00220F1F777F908F156
:10847000010080B28046042880D394F8AE07032818
:1084800003D094F8AE07012803D19E490020C1F81B
:108490008802002084F8AC070B2084F8B007944EC3
:1084A00000203A3E307000980DE001F04DFDC4F818
:1084B000F803D4F8F803C0F300400190D4F8F803AF
:1084C000C0F3420000900028EFD094F8AE070228D5
:1084D00011D194F8AD0770B1854855214FF00709C7
:1084E0000170FD214170AA2181700021C1700171CC
:1084F0006122427181717E49FA2201F8092094F8C3
:10850000EF2301EB09000290427094F8EE23827091
:1085100094F8ED23C27094F8EC23027194F8EB23E5
:10852000427194F8EA2382710020D4F8F823C0F154
:108530000301C900CA406E4909EB000319444A729D
:10854000401C80B20428F0D394F8AD0720B16D48E8
:10855000D0F80802A8B905E002990898487309F113
:108560000E0533E06548007858B194F8AE0703284B
:1085700007D094F8AE07012803D0012084F8AE0696
:10858000F3E35E495A4A00200B1803F5805393F831
:10859000335709EB000313445D73401C80B2142869
:1085A000F2D300200B1803F5805393F8F45709EB2E
:1085B0000003134483F82150401C80B20A28F1D3F1
:1085C0000299089881F82B0009F12C05002DD7D0CD
:1085D000089884F86F0608981021FF2212287CD092
:1085E00009DCA0F10B0007281BD2DFE800F01A1A03
:1085F000FD0DFC1BFB00A22813DA4FF059021428D2
:1086000001D015280DD1B1E384F8B0173E4A38499E
:1086100000202E18135C8B55401C80B20A28F8D31A
:108620000A35A8E394F8DC01C00760D0012080F38C
:108630001388BFF34F8F35480168354A01F4E06174
:1086400011430160BFF34F8FFEE700EB40012B4F5A
:1086500001EB0A1007EB0016049606F5805696F813
:108660006A0D032818D096F86A0D012814D096F8E0
:108670006A0D022810D096F86A0D04280CD096F8DE
:108680006A0D072808D096F86A0D05287ED096F85E
:108690006A0D06287BD068E1154901204855ED1C7C
:1086A000A8B2022205900A54401C80B21D220A542E
:1086B000401C85B20020B5E0049800EB081101F5DC
:1086C000805191F8940D0A4A50556D1C91F8963DD1
:1086D000A8B21354401C85B200E048E291F8960D10
:1086E00040071BD491F8960D000717D412E03FE124
:1086F00052020020A4520020BC640240A4120020B8
:108700008E26002000004042BCE601080CED00E08F
:108710000400FA0591F8960D800766D50020D1F87F
:10872000983DC0F10307FF00FB404719D355401C9B
:1087300080B20428F3D32D1DABB20AEB0A1505EB6A
:108740000A210CEBC10508EB081105EBC1010391EF
:10875000002001F50051D1F84552C0F10307FF0098
:10876000FD40C718D555401C80B20428F3D31B1D0B
:108770009BB20020D1F84952C0F10307FF00FD4031
:10878000C718D555401C80B2042801E05CE091E098
:10879000F0D31B1D9BB20020D1F86052C0F102073C
:1087A000FF00FD40C718D555401C80B20328F3D305
:1087B000DB1C9FB20025039901F50050D0F84D0253
:1087C00001F50051D1F85112C5F10502D200EFF7C1
:1087D0002AFDFA49EA1988546D1CADB2062DEAD378
:1087E000B81D03E06CE1FFE14AE118E087B2002523
:1087F000039901F50050D0F8550201F50051D1F868
:108800005912C5F10502D200EFF70DFDEB49EA1947
:1088100088546D1CADB2062DEAD3B81D85B208F19F
:10882000010080B2DFF898C396F86B1D8046414581
:108830003FF642AF0598E149059A281A1144030A08
:1088400001F8023D487090E0DFF870C302200CF898
:108850000500ED1CADB22E46002220E0531C0CF8A2
:1088600005306D1CB91801F58051A8B291F88D152D
:108870000CF80010401C81B2002007EB02152A18EA
:1088800002F5805292F8992500EB01080CF80820B7
:10889000401C80B21028F2D310318DB29AB294F8F5
:1088A0008C059042DAD80CEB0600002100F8021D7E
:1088B000A91B59E0C14B03205855ED1CA8B2022159
:1088C00080461954401C80B20E211954401C85B2B8
:1088D0000021BE463DE0049800EB0110A0F51B709E
:1088E00000F5005002785A556D1CAAB285789D5447
:1088F000521C807895B2400729D50AEB0A1C0CEB74
:108900000A220EEBC20201EB0117002002EBC702A4
:10891000171807F5005797F86B7200EB050C03F872
:108920000C70401C80B20A28F2D30A35ADB2002088
:10893000171807F5005797F8847200EB050C03F839
:108940000C70401C80B20228F2D3AD1CADB2491CA1
:1089500089B296F86B0D8842BDD803EB0800002160
:1089600000F8021DA5EB080141700AF1010080B278
:1089700094F8361B824651453FF667AE94F8D80B03
:1089800000287CD0002176E0DFF8348201EB410042
:1089900008EB001202F5805292F8E20B042810D185
:1089A000864B58556D1CA8B201251D5408EB0105D6
:1089B00005F58055401C95F8415D80B21D54401C62
:1089C00085B292F8E20B06280CD001EB410000EBD7
:1089D000011008EB001000F5805090F86A0D052892
:1089E00035D046E0754F062078556D1C94F88C25DF
:1089F000A8B23A54401C80B212223A54401C85B2AC
:108A000000231FE05E1C7E5508EB030202F5805236
:108A10006D1C92F88D25A8B23A54401C82B20020F9
:108A200008EB03152B1803F5805393F8993500EBE9
:108A3000020C07F80C30401C80B21028F2D3103220
:108A400095B2B3B294F88C059842DBD811E05B4A3A
:108A5000052050556D1CA8B20123135408EB0103E7
:108A600003F58053401C93F8413D80B21354401CE1
:108A700085B2491C89B294F8D80B884284D87AE12F
:108A80007078401C70707078052803D294F8DC016F
:108A9000C00706D084F8B01794F8DC01C00704D0F2
:108AA00005E00D2084F8B00701E084F8E02170882B
:108AB000010A42484155718828444170AD1C5AE171
:108AC00084F8B01794F8E1013C4F78550022DFF8A4
:108AD000F0C06D1C3CE094F8E10102EB021600EBE3
:108AE000001101EB00200CEBC00000EBC60000F50C
:108AF000805090F81C0A012828D194F8E10100EB7D
:108B0000400101EB00100CEB001000EB021000F52F
:108B1000805090F8640C78556D1CABB2002094F82E
:108B2000E11101EB011505EB01210CEBC10101EB9A
:108B3000C601014401F5805191F81D1A1D1879559F
:108B4000401C80B20A28EAD30A339DB2521C92B26A
:108B500094F8E10100EB400101EB00100CEB001078
:108B600000F5805090F83B0C9042B4D803E1707847
:108B7000401C7070707805280ED294F8E10100EB6B
:108B8000400303EB00130E4800EB031000F5805088
:108B900090F84C0CC00715D084F8B01794F8E10198
:108BA00000EB400101EB0011054800EB011000F55E
:108BB000805090F84C0CC00708D009E05202002009
:108BC000A4120020122084F8B00701E084F8E0210C
:108BD00094F8E111FC48415571882844090A417014
:108BE00071888170ED1CC6E0F84801210172816D29
:108BF0000A22B1FBF2F2F4494A55806D6D1C0A2835
:108C000001D90A2201E0F148826D002003909246CA
:108C10004A5522206D1C485500266D1C9DE0DFF84A
:108C2000AC83D8F8580038B1D8F85800801B401EE3
:108C300081B20220EFF71CFF98F81C00E24948556A
:108C40006D1CAAB20020D8F81D30C0F10305ED005C
:108C5000EB4085184B55401C80B20428F3D3121DFD
:108C600092B200E0D1E00020D8F82130C0F1030535
:108C7000ED00EB4085184B55401C80B20428F3D31F
:108C8000121D92B20020D8F82530C0F10205ED0087
:108C9000EB4085184B55401C80B20328F3D3D21CFF
:108CA00097B20025414651F8290F4968C5F10502E0
:108CB000D200EFF7B8FAC449EA1988546D1CADB276
:108CC000062DEFD3BF1DBFB200258846BF4951F81E
:108CD000310F4968C5F10502D200EFF7A4FAEA198D
:108CE00008F802006D1CADB2062DEFD3B749BF1DC9
:108CF000B8B291F84230424608F80030401C91F872
:108D0000413080B208F80030401C91F8403080B209
:108D100008F80030401C91F83F3080B208F800306D
:108D2000401C91F83E3080B21354401C91F83D3005
:108D300080B21354401C83B20020D1F84350C0F1DC
:108D40000307FF00FD40C718D555401C80B204281A
:108D5000F3D31B1D761C9DB2B6B2039A0020B6EB6E
:108D60000A019041FFF65BAF05E0D9E084F8B01747
:108D7000954842556D1C0298A5EB0906320ADFF8AA
:108D80004882C2710298067200230BE009EB0301CE
:108D900001EB0807787BDDE90021F0F75BFC7873D5
:108DA0005B1C9BB29E42F1DC94F8E90328B1B1B29E
:108DB000002304220298F1F729F9B1B2464602983D
:108DC000F0F736FA010A71556D1CA9B27054491CAE
:108DD00094F8AE078DB202280DD194F8AD0750B1CA
:108DE000681F010AF170307181B2701D01F0F3F952
:108DF00070556D1CADB2CBF8005001217448F0F7EE
:108E00006DFA09B02846BDE8F08F94F8AE07714BB3
:108E1000714F42F21076A3F18509A3F1870CA3F1FB
:108E20000B08A3F1720A30B1012877D0022876D05E
:108E3000032875D13EE394F8EA06C0F3C3000E2878
:108E40006ED2DFE800F0071422303E4D5C6E7D8C60
:108E50009BDEEBFE00261F4603E0B85DA855761C9E
:108E6000B6B25C48EFF70FFAB042F6D83CE3002404
:108E700004E019F804002855641CA4B2554885384C
:108E8000EFF701FAA042F4D8C8E30024664603E0F5
:108E9000305D2855641CA4B24E488738EFF7F3F9CB
:108EA000A042F5D8BAE3002404E018F804002855DD
:108EB000641CA4B247480B38EFF7E5F9A042F4D898
:108EC000ACE3444E00241C3E03E0305D2855641C96
:108ED000A4B240481C38EFF7D6F9A042F5D89DE37C
:108EE0003C4E00242D3E03E0305D2855641CA4B2A6
:108EF00038482D38EFF7C7F9A042F5D88EE3324E47
:108F00000024323E03E0305D2855641CA4B22E4894
:108F10003238EFF7B8F9A042F5D87FE39FE0DEE101
:108F2000C4E02C4E00243C3E03E0305D2855641C18
:108F3000A4B228483C38EFF7A6F9A042F5D86DE373
:108F4000244E0024163603E0305D2855641CA4B27C
:108F500020481630EFF797F9A042F5D85EE31D4E92
:108F600000240A3603E0305D2855641CA4B2194879
:108F70000A30EFF788F9A042F5D84FE394F8AD072F
:108F8000144E643E022811D00020315C2954401C4C
:108F900080B20D28F9D33846EFF775F9002250EA70
:108FA000020129D000211346084C20E0002403E0F0
:108FB000305D2855641CA4B206486438EFF763F9A5
:108FC000A042F5D82AE3000052020020A41200209B
:108FD000B86402407BEE0108A5290020661806F55A
:108FE000805696F801676F187E73491C89B20E1A75
:108FF00073EB0206F2DBFDE2FB48EFF744F984B2C3
:109000000CE30024F94E03E0305D2855641CA4B243
:10901000F648EFF738F9A042F6D8FFE2DFF8CC8344
:109020000027A8F19A0805E00BE018F80700E855BA
:109030007F1CBFB2ED489A38EFF725F9B842F4D853
:1090400012E2002704E01AF80710E9557F1CBFB2AE
:10905000E6489338EFF717F9B842F4D804E294F8E9
:10906000EA06C0F3C3000D2820D2DFE800F0072095
:109070002F3C4B5A69788796F3F1F000DB4F0026BE
:109080008C3F03E0B85DA855761CB6B2D7488C3843
:10909000EFF7F9F8B042F5D8CBF800600121D448D9
:1090A000F0F71CF94FF47A70C4F88C06CAE2CF4E80
:1090B0000024B63603E0305D2855641CA4B2CB48CA
:1090C000B630EFF7E0F8A042F5D8A7E20024C94E89
:1090D00003E0305D2855641CA4B2C648EFF7D3F80E
:1090E000A042F6D89AE2C34E0024A53E03E0305DCC
:1090F0002855641CA4B2BF48A538EFF7C4F8A042B5
:10910000F5D88BE2BB4E00249A3E03E0305D285533
:10911000641CA4B2B7489A38EFF7B5F8A042F5D866
:109120007CE2B44E00248F3E03E0305D2855641C81
:10913000A4B2B0488F38EFF7A6F8A042F5D86DE298
:10914000AC4E0024863E03E0305D2855641CA4B27A
:10915000A8488638EFF797F8A042F5D85EE2A54E0A
:109160000024773E03E0305D2855641CA4B2A1487A
:109170007738EFF788F8A042F5D84FE29D4E0024EB
:10918000593E03E0305D2855641CA4B29948593813
:10919000EFF779F8A042F5D840E294F8AD07954C86
:1091A0004C3C022816D00020215C2954401C80B27F
:1091B0001428F9D33846EFF766F8044600268EA146
:1091C000384605F0F3F954EA060135D00021431E74
:1091D0008A4A17E0002603E0A05DA855761CB6B2C7
:1091E00084484C38EFF74FF8B042F5D828E05718CC
:1091F00007F5805797F8017705EB010C8CF8147090
:10920000491C89B29942F2DB22212B18D974641CC3
:1092100046F1000108E0131803F5805393F8003776
:109220002F183B75401C80B2031B76EB0103F2DB69
:1092300073A16D48EFF71BF86B48EFF724F886B27F
:10924000CBF8006001216A48F0F748F8FAE12FE016
:109250000FE0FFE7674E00241C3E03E0305D285519
:10926000641CA4B263481C38EFF70DF8A042F5D88F
:10927000D4E1D4F88C1640F2E930814207D194F859
:10928000EA0620F07800603084F8EA0601E0C4F8CD
:109290008C06564E00249E3E03E0305D2855641C2B
:1092A000A4B252489E38EEF7EEFFA042F5D8B5E1E1
:1092B000504F00260B3F03E0B85DA855761CB6B2B0
:1092C0004C480B38EEF7DFFFB042F5D8CBF8006022
:1092D00001214748F0F702F843F69820E4E694F8B5
:1092E000EA06C0F3C30005287DD2DFE800F00314CE
:1092F000608ED100002084F8AF07044604E018F81F
:1093000004002855641CA4B238482C38EEF7BBFF83
:10931000A042F4D882E1002184F8AF17084629540E
:10932000401C80B26428FAD384F8AF172F4900207C
:109330005B310A5C2A54401C80B20828F9D3DFF85C
:10934000BC9041F26F71002709EB010809E009EBBD
:10935000070000F5805090F86F07E91908727F1C2C
:10936000BFB24046EEF78FFFB842F0D82C20E91983
:10937000087209371FFA87F841F29771002709EB45
:10938000010A0AE009EB070000F5805090F89717F2
:1093900008EB0702A9547F1CBFB25046EEF773FFDB
:1093A000B842EFD816A11048EEF761FF6BE00F4FFF
:1093B0000026A13703E0B85DA855761CB6B20B486D
:1093C000A130EEF760FFB042F5D8CBF80060012184
:1093D0000748EFF783FF94F8EA0620F0780018308A
:1093E00084F8EA060EE0E9E0520200209CEE010853
:1093F000B864024001F001082C000000A412002013
:109400000D0A00004FF4FA604EE694F8AD07DFF85D
:109410003C8202284FF0000018D000212954401C43
:1094200080B26428FAD384F8AF17002018F800102F
:109430002954401C80B20E28F8D33846EEF723FF9B
:109440000104090C1FD00020814A19E084F8AF07FD
:10945000002704E018F80710E9557F1CBFB27B48CD
:10946000EEF711FFB842F5D8CBF80070E4E013181E
:1094700003F5805393F801372F18BB73401C80B25B
:109480008842F4D38EE77348EEF7FDFE5946D2E0EA
:10949000DFF8B881002708F1350804E018F8070064
:1094A000E8557F1CBFB269483530EEF7ECFEB84294
:1094B000F4D8D9E794F8EA06C0F3C30009287DD2AE
:1094C000DFE800F005202D3B4958679EAF000026DD
:1094D0001F4603E0B85DA855761CB6B25B489938C4
:1094E000EEF7D1FEB042F5D8CBF8006001215A4822
:1094F000EFF7F4FE94F8EA0620F07800083084F8DC
:10950000EA06CFE5002404E019F804002855641C9D
:10951000A4B25248EEF7B7FEA042F5D87EE0002490
:10952000664603E0305D2855641CA4B24B48801E9B
:10953000EEF7A9FEA042F5D870E0002404E018F888
:1095400004002855641CA4B244487A30EEF79BFE10
:10955000A042F4D862E03D4E0024443E03E0305D7A
:109560002855641CA4B239484438EEF78CFEA0425A
:10957000F5D853E0354E0024353E03E0305D2855E4
:10958000641CA4B231483538EEF77DFEA042F5D810
:1095900044E094F8AD072D4E6E3E022812D0002014
:1095A000315C2954401C80B20F28F9D33846EEF7BD
:1095B0006AFE0104090C3FF41FAD00E042E0002008
:1095C000234A15E0002403E0305D2855641CA4B252
:1095D0001E486E38EEF757FEA042F5D81EE013186D
:1095E00003F5805393F801372C18E373401C80B2C5
:1095F0008842F4D3AFF2F8111648EEF738FEFBE4D8
:10960000124E00242B3E03E0305D2855641CA4B2AA
:109610000E482B38EEF737FEA042F5D8CBF80040C5
:1096200010E600201AF800102954401C80B20728C8
:10963000F8D35946401E086001210748EFF74EFE57
:10964000C4F88C6609B00020BDE8F08F14EF010863
:10965000A412002052020020B8640240F6ED010876
:1096600070B5164C40F224452946204603F071F9A6
:10967000002821D02946204603F008F9104D00218A
:109680002846EFF72BFE61102846EFF711FE0D4933
:10969000012081F8AF072088A088281D0268C2F544
:1096A000FA62A1F872264FF4FA6101602846BDE81B
:1096B00070400121EFF712BE70BD000000100140A4
:1096C00088640240A422002010B5074C05492046BA
:1096D000EFF7EEFD00212046EFF700FE03490120E1
:1096E000087010BD00800028B864024018020020F5
:1096F0002DE9F04301218FB0880500F07BFBDFF8F6
:1097000094904846EFF7F4FD4020050103900024B3
:10971000CDE90545C60207940894CDE909464FF006
:1097200000681E480B940C940D941B4FCDF80080DC
:109730000E94CDE9017069464846EFF781FE01229B
:1097400010214846EFF766FEDFF84890A9F130098E
:109750004846EFF7CDFD4FF4FA60CDE90340CDE97F
:10976000054507940894CDE909460D480B940C94DF
:109770000D94CDF800800E94CDE9017069464846FD
:10978000EFF75EFE01214846EFF7A8FD0FB0BDE8F8
:10979000F0830000B864024004100140520200202F
:1097A000547400207CB50121032000F023FB164EE9
:1097B000072206213046F0F7EDFB0722114630461E
:1097C000F0F7E8FB02218DF8051000258DF8065012
:1097D0000124C0208DF8074000908DF804106946E0
:1097E0003046F0F79BFB202000908DF804408DF868
:1097F000065003208DF805008DF807406946304675
:10980000F0F78CFB7CBD000000040240F0B589B08D
:109810000025FFF7C7FFFFF76BFF4FF4E13000F0C3
:109820000FF900F0EFF80121402000F0FBFA0120D1
:1098300000F07CFB4FF47A77384604F017FD5F4C5C
:109840000B2084F82C01002684F828612676A67661
:109850006676E676276284F82860012384F82A3049
:1098600084F8293084F82B30F80020632670A37028
:109870006370E370A7602673A3736373E3730011CF
:10988000606104F538510E708E704B70CB704EF6DF
:1098900060278F604A4A42F6F82CA1F28441A4F274
:1098A000846405EB450002EB8000A0F6481000F54B
:1098B0000050067086704370C670C0F808C06D1CFA
:1098C000042DEED394F8AB07000706D094F8AB074D
:1098D00000F00F00401E84F8AD0794F8AB070009B4
:1098E00006D094F8AB07FF2303EB101084F8AE0703
:1098F00084F8B26794F8AE0768B1324B01280DD0F6
:10990000022808D0032811D147F23050C1F88C0446
:10991000C3F888620AE0C1F88C7407E0C1F88C745F
:10992000C3F8886243F69820C4F88C062648274975
:10993000006808602448001D00684860224808301C
:10994000006888600020131803F5805383F833679C
:10995000401C1428F7D3087A04AFCD7A8B7A4A7A60
:1099600087E82D000879CD798B794A798DE82D002B
:1099700012488B780A7816A1AF3003F089F80021DD
:109980000320EFF7EBFE10B11C48C0F8886294F892
:10999000AD171B4800294FF0200104D009B0BDE8E5
:1099A000F040F0F70EBBF0F70EFB94F8EA0640F03B
:1099B000800084F8EA0609B0F0BD000028290020E4
:1099C000A412002000004042107AFF1F247C0020D7
:1099D000253032782530327825303278253032788B
:1099E000253032782530327825303278253032787B
:1099F00025303278253032782500000000004242C0
:109A00000004024038B546208DF8000002208DF891
:109A1000010001248DF802408DF803406846FBF7F1
:109A200093FD25208DF800008DF8014000208DF871
:109A300002008DF803406846FBF786FD38BD000044
:109A40001FB504460121102000F010FA0020ADF8E7
:109A500004000094ADF80600ADF80800ADF80C0065
:109A60000C200D4CADF80A006946204602F0A8FF14
:109A70000121204602F00DFF012240F22441204640
:109A800002F086FF1021204602F000FF0122C021D3
:109A9000204602F008FF1FBD001001402DE9FC47E1
:109AA0000121592000F0A6F943F6F8700024DFF8F0
:109AB000A0A000908DF8044002268DF8076069464A
:109AC0005046F0F72BFAFC20DFF8889000908DF8D4
:109AD000044001258DF8075069464846F0F71EFA04
:109AE000DFF874804FF440478DF8044000978DF8FC
:109AF000075069464046F0F711FA8DF804408DF89A
:109B000007600720154E009069463046F0F706FAC8
:109B100007213046F0F755FA39464046F0F753FA38
:109B20004FF47C515046F0F74EFAF8215046F0F7CA
:109B300048FAFC214846F0F746FA0948D0F82812BE
:109B40000848012902D00470BDE8FC870570FBE7D6
:109B50000010024000180240000C024000000240C9
:109B600000004242A412002070B5FFF797FF642066
:109B700004F07CFB2048D0F83C3201221F492048E9
:109B80000024E3B180F8AD47D1F814021D4978B341
:109B90000C761D48D0F81C22D0F81832120142EA87
:109BA000C302D0F8143242EA8302D0F81032D0F85F
:109BB0000C0242EA4302024318324A7070BDD1F8E7
:109BC00018328BB180F8AD27D1F80832D1F80C5299
:109BD00043EA4503DB4380F8AE3790F8AE3703F035
:109BE000030380F8AE37CFE7022380F8AD37EBE709
:109BF000FFE70A76CDE700000080414200004342C3
